:020000040800F2
:100000000000011011FD0308F1B1030869D70008D1
:1000100015FE030815FE030815FE03080000000086
:10002000000000000000000000000000F9B103081B
:10003000F5B1030800000000EDB10308ADED0008C4
:1000400015FE030815FE030815FE030815FE030838
:1000500015FE030815FE0308919D0008BD9E0008CB
:10006000819E0008459E0008099E0008C5BC000846
:10007000B5BC0008A5BC000895BC000885BC0008FC
:1000800071BC00085DBC000815FE030815FE0308DE
:1000900015FE030815FE030815FE0308CD9D000894
:1000A00055DE0008C5DE000815FE0308D5DE000891
:1000B000B5DE0008A5DE000895DE0008A5C2000830
:1000C000ADC2000899C20008A1C2000815FE0308CD
:1000D00015FE0308E99200084D92000839EE000869
:1000E000559D000815FE03087D2D030815FE030825
:1000F00065DE000815FE030875DE000849BC00082F
:1001000015FE030815FE030885DE000815FE03082A
:1001100015FE030815FE030841E1010825E1010869
:1001200035BC000821BC00080DBC0008F9BB000864
:10013000E5BB000815FE030815FE030815FE0308BD
:1001400015FE030815FE030815FE03083D270308E6
:10015000D1BB0008BDBB0008A9BB000815FE030801
:100160008DC2000895C2000815FE030815FE03089D
:1001700015FE030815FE030815FE030815FE030807
:0801800015FE030815FE03083B
:08018800A8F8030001000000CB
:10019000160008009C250020A42500200000000077
:1001A0006806000803000100242C00202C2C0020ED
:1001B00000000000000000001D0001003C2C002099
:1001C000CC2C00200000000070060008270004006E
:1001D0005C2C0020D02C00200000000072060008DB
:1001E0000A020A000C2E00201C2E00200000000035
:1001F000760600082C001000C0340020B034002027
:1002000000000000210502082B002400F434002027
:10021000D034002000000000F10402080312330073
:100220003B3700200837002000000000800600084F
:1002300025005A0054360020AE3600200000000091
:1002400000000000F6110C00483600203C3600206B
:1002500000000000B40600081B00F400BC370020BA
:100260003C390020000000001DB402082F001100DE
:1002700020390020303A002000000000C0060008AD
:1002800003010600943A0020D03A0020000000004C
:10029000D20600080B201000003E0020383E00204F
:1002A00000000000D80600081F000E00703B002070
:1002B000483E002000000000E8060008050201009A
:1002C000C43B0020583E002000000000F606000855
:1002D00001010400143F0020184E0020000000001F
:1002E0000000000008020900564D00201C4E0020AE
:1002F000000000001F82000806020C00CC4D002008
:10030000284E0020000000007D9000080702020037
:10031000F04D0020344E002000000000F8060008D8
:10032000FF010100064E0020384E002000000000B2
:10033000FA06000802000C00D84D00203C4E0020B8
:100340000000000000000000F7010600504D0020F2
:10035000484E002000000000FC06000801020500D5
:1003600084530020E057002000000000D12D030836
:1003700000020500504E0020E85700200000000059
:10038000000000001E00040090510020F0570020E3
:10039000000000000207000822000C001451002099
:1003A000F45700200000000006070008F9010400CF
:1003B000AC5D0020206600200000000011820008D3
:1003C00018102C007C5D0020246600200000000036
:1003D000C90E0208FB010100545D00205066002098
:1003E00000000000A1C30008FC010900205C0020FF
:1003F00054660020000000006DC300080A101200BF
:10040000F45B002060660020000000001207000876
:1004100006001600C458002074660020000000008A
:10042000E143030829005000FC68002070690020A7
:10043000000000000000000014000200F868002026
:10044000C06900200000000024070008100003001D
:10045000EC680020C46900200000000026070008A6
:1004600028000C00E0680020C8690020000000009F
:100470002A07000823001000D0680020D46900205B
:10048000000000003DFC010819000500C8680020BC
:10049000E46900200000000036070008F8110100A0
:1004A000C4680020EC690020000000003C07000840
:1004B00000010400C0680020F06900200000000076
:1004C0003E070008340010003C7C0020107D002016
:1004D000000000007D4303080D002400187C00206C
:1004E000207D002000000000CD9E030812100C00AB
:1004F000FC7B0020447D0020000000004207000833
:100500000C020100F87B0020507D0020000000005C
:100510004E070008020203000C7C0020547D0020DE
:10052000000000000000000011000C00846A0020A0
:10053000587D00200000000041880008FD011E00D9
:10054000646A0020647D002000000000A181000892
:10055000FE010800506A0020847D00200000000099
:10056000A9C3000804008000E0A2002060A40020CD
:1005700000000000000000000902010044A5002066
:100580009CA5002000000000500700080C0024007B
:1005900002A50020A0A5002000000000DD9B0208AD
:1005A00001200800E4AD0020ECAD002000000000B8
:1005B000520700081A000800C8AD0020F4AD002062
:1005C000000000005A0700082A0060005CAE00200E
:1005D000FCAD00200000000055430308150070002A
:1005E00054A70020BCAE0020000000000000000066
:1005F0000E20EA00BEAF0020DCBD0020000000009D
:10060000C143030813000400ECB00020C8BE002062
:10061000000000006407000802010300A9AF0020E9
:10062000CCBE002000000000059C0208050006006A
:100630005CBF0020D4C00020000000006807000854
:10064000F5116200F4BE0020DCC0002000000000B4
:100650007D3B020826000E0050C1002040C1002052
:0806600000000000717703089F
:10066800C409000019012828000020030000000028
:100678004A01B400D601000000000000000000009C
:100688000000000000000000000000000000000062
:100698000000000000000000000000000000000052
:1006A8000000000000000000000001000000000041
:1006B8000000000000000000000000000000000032
:1006C800000000000000000000000401010000001C
:1006D8002B21231E64010100000001000A012900EA
:1006E80000000000000001000000000500000000FC
:1006F800013C000023010000000000000100C800C8
:10070800141E010064002C01280000300100005A6A
:100718000000000090012C01C800640003000001E3
:1007280005000000000100000000000000000000BB
:1007380028010000040090010000000000010005ED
:1007480042524634000001001300E8036400040A22
:1007580000017E05EA05B4053200000008044400E3
:0607680020000200010068
:10076E000100000050010000070000000200000020
:10077E000000000000000000010203040607080943
:10078E0001010000745A04083886040800000000B5
:10079E0000000000845A04088C5A0408000000006F
:1007AE0001200000905A0408985A04080000000026
:1007BE00014000009C5A0408387404080000000030
:1007CE0001200000A85A0408B45A040800000000D2
:1007DE0004000000B85A0408289304080000000022
:1007EE0004000000C45A0408DC8F04080000000056
:1007FE000100000002010000685E0C00FF00000016
:10080E000000803F0000803F01010000BD01020892
:10081E000000000000000000010000000060024027
:10082E001060024000000000000B000000002000DD
:10083E00000000000000000000600240286002403E
:10084E0000000000060C0000000020000000000068
:10085E000000000000600240406002400000000006
:10086E00100D00000000200000000000000000003D
:10087E00006002405860024000000000160E0000AA
:10088E000000200000000000000000000060024098
:10089E007060024000000000200F000000002000E9
:1008AE00000000000000000000600240886002406E
:1008BE0000000000261000000000200000000000D4
:1008CE000000000000600240A06002400000000036
:1008DE0030110000000020000000000000000000A9
:1008EE0000600240B860024000000000362F000099
:1008FE000000200000000000000000000064024024
:10090E0010640240000000000038000000004000AB
:10091E000000000000000000006402402864024055
:10092E00000000000639000000004000000000003A
:10093E00000000000064024040640240000000001D
:10094E00103A00000000400000000000000000000F
:10095E00006402405864024000000000163B000094
:10096E000000400000000000000000000064024093
:10097E007064024000000000203C000000004000B7
:10098E000000000000000000006402408864024085
:10099E00000000002644000000004000000000009F
:1009AE000000000000640240A0640240000000004D
:1009BE003045000000004000000000000000000074
:1009CE0000640240B8640240000000003646000099
:1009DE00000040000000000000000000FFFFFFFFCD
:1009EE0000000101FFFF000000FFFF0000000000FB
:1009FE00AA5505010000AA550701000000000000DD
:100A0E00010203040102030406070809AA550B019B
:100A1E000000000001000000C01201AA5503009F53
:100A2E00AA5509020000000009024300020100C09D
:100A3E003209040000010202010005240010010524
:100A4E002401000104240202052406000107058288
:100A5E00030800FF09040100020A00000007050157
:100A6E00024000000705810240000000FF00000068
:100A7E00284504080508040000000000EC56040890
:100A8E00CC42040814450408000000005445040834
:100A9E0005080A0000000000EC560408CC420408C9
:100AAE009457040800000000E00100000000803FA1
:100ABE0008000000FFFF0100303030302D30312DA6
:100ACE0030315430303A30303A30300000010101CC
:100ADE000800000004030904120100020202004093
:100AEE00830440570002010203010000B196020880
:100AFE00B19502082D97020801880208FD8B0208A5
:100B0E00118802082D880208D9870208C9870208B1
:100B1E0000000000000000000000803F0101010005
:100B2E003C9204080F0000009163030800000000CF
:100B3E0000000000400500200092040800000000A4
:100B4E0000000000000000000000000038860408CD
:100B5E000000000000000000CC0500200400000092
:100B6E008C9104080D000000B96A0308E00900200A
:100B7E0000000000309604080D000000896A03088A
:100B8E00D409002000000000209204080800000094
:100B9E0000000000C80900200400000010920408A4
:100BAE000D000000A1690308BC0900200000000030
:100BBE00A49004080300000071C50308A4090020D6
:100BCE0000000000189204080300000071C503081D
:100BDE008C09002000000000A8900408010000000D
:100BEE0000000000000000000000000000000000F7
:100BFE000E000000000000000000000000000000D9
:100C0E000092040800000000000000000000000038
:100C1E0000000000388604080000000000000000FC
:100C2E00CC050020040000003091040803000000F1
:100C3E00456903087409002008000000109204089A
:100C4E000D000000A1690308BC090020000000008F
:100C5E00A49004080300000071C50308A409002035
:100C6E0000000000189204080300000071C503087C
:100C7E008C09002000000000A8900408010000006C
:100C8E000000000000000000000000000000000056
:100C9E000E00000000000000000000000000000038
:100CAE002892040800000000000000000000000070
:100CBE00000000003886040800000000000000005C
:100CCE00CC05002004000000389104080300000049
:100CDE0071C50308EC09002000000000A89004086C
:100CEE0001000000000000000000000000000000F5
:100CFE00000000000E0000000000000000000000D8
:100D0E000000000020700020702D72002D202D2D6F
:100D1E00202D2D2D2D202D2D2D2D0000000000001D
:100D2E000000000000000000000000002D202D2D0E
:100D3E00202D2D2D2D202D2D2D000000000000002A
:100D4E000000000000000000000000004AAF00207C
:100D5E0088130C17010000004CAF002088130C17ED
:100D6E00000000007C90040800000000000000005D
:100D7E0000000000000000008C9004080800000035
:100D8E0000000000F8050020040000009890040800
:100D9E000800000000000000EC050020000000002C
:100DAE00A4900408040000008569030800000000F8
:100DBE0000000000A89004080100000000000000E0
:100DCE000000000000000000000000000E00000007
:100DDE0000000000000000000000000048AF0020EE
:100DEE0088130C170100000046AF002088130C1763
:100DFE0000000000E09004080F000000E963030803
:100E0E00000000000000000004060020EAB00020F0
:100E1E0001000000AC56040845AF002001000000A0
:100E2E00B8560408C63A002002000000C056040856
:100E3E00A6A300200000000000000000A4A30020D4
:100E4E000000000000000000A2A30020000000002F
:100E5E0000000000A0A30020000000000000000021
:100E6E009EA3002000000000000000009CA30020B4
:100E7E000000000000000000B8020020000000008A
:100E8E000000000044AF002002000000CC56040811
:100E9E00E8900408000000000000000000000000C0
:100EAE00000000008C900408080000000000000004
:100EBE008806002004000000989004080800000036
:100ECE00000000007C06002000000000A490040832
:100EDE0004000000C96303080000000000000000C9
:100EEE00A8900408010000000000000000000000AF
:100EFE0000000000000000000E00000000000000D6
:100F0E000000000000000000F8900408000000003F
:100F1E00000000000000000000000000089104081E
:100F2E000D000000296A0308C4060020040000001A
:100F3E00149104080D0000000D640308B80600208B
:100F4E0004000000209104080D000000E969030868
:100F5E00AC060020000000002C91040803000000E5
:100F6E006569030894060020080000003891040803
:100F7E000300000071C50308EC090020000000000A
:100F8E00A89004080100000000000000000000000E
:100F9E0000000000000000000E0000000000000035
:100FAE000000000000000000409104080000000056
:100FBE00000000000000000000000000489104083E
:100FCE0004000000E96A03080000000000000000B1
:100FDE00A8900408010000000000000000000000BE
:100FEE0000000000000000000E00000000000000E5
:100FFE0000000000000000009491040800000000B2
:10100E00000000000000000000000000B081040895
:10101E000D00000000000000240700200400000066
:10102E00A49104080800000000000000180700202A
:10103E0004000000B0910408080000000000000049
:10104E000C07002004000000B891040808000000FE
:10105E00000000000007002004000000C0910408FA
:10106E000800000000000000F4060020040000004C
:10107E00C89104080800000000000000E8060020E7
:10108E0004000000D09104080800000000000000D9
:10109E00DC06002004000000D891040808000000BF
:1010AE0000000000D006002004000000A8900408F4
:1010BE000100000000000000000000000000000021
:1010CE00000000000E000000000000000000000004
:1010DE0000000000E09104080F000000D96303082F
:1010EE00000000000000000030070020E891040816
:1010FE000F000000000000000000000000000000D3
:10110E00A8070020F09104080F0000000000000066
:10111E00000000000000000048080020E9B0002098
:10112E0004000000D856040840AF0020E0150C174C
:10113E000000000043AF002008000000CC4204086D
:10114E0042AF002005000000EC560408F891040898
:10115E000F00000000000000000000000000000072
:10116E0098080020010000003C7F040800000000E9
:10117E0000000000199C0208A08601000400000077
:10118E000000000000000000000000000000000051
:10119E00000000000000000000000000AC960408F3
:1011AE00907E0408000000004D5901087D000000EB
:1011BE00060000000000000000000000000000001B
:1011CE000000000000000000000000000000000011
:1011DE004493040800000000000000006DD90308CD
:1011EE00E803000003000000000000000000000003
:1011FE0000000000000000000000000000000000E1
:10120E00000000004C9304080000000000000000E5
:10121E00F144030810270000030000000000000046
:10122E0000000000000000000000000000000000B0
:10123E0000000000000000002495040800000000DB
:10124E00C9030208753A0108204E0000050000008F
:10125E000000000000000000000000000000000080
:10126E00000000000000000000000000B080040834
:10127E00000000000000000029D403081027000021
:10128E00010000000000000000000000000000004F
:10129E000000000000000000000000000000000040
:1012AE0058930408000000000000000039C3000835
:1012BE00E803000005000000000000000000000030
:1012CE000000000000000000000000000000000010
:1012DE0000000000649304080000000000000000FD
:1012EE00419E0208204E0000030000000000000096
:1012FE0000000000000000000000000000000000E0
:10130E0000000000000000007493040800000000BC
:10131E0000000000499C0208204E0000030000005F
:10132E0000000000000000000000000000000000AF
:10133E00000000000000000000000000849304087C
:10134E000000000000000000B9D10308400D0300AA
:10135E00030000000000000000000000000000007C
:10136E00000000000000000000000000000000006F
:10137E00F07F0408000000000000000059AD0308D3
:10138E001027000001000000000000000000000017
:10139E00000000000000000000000000000000003F
:1013AE0000000000AC7E04080000000000000000F9
:1013BE00E5C4020810270000030000000000000032
:1013CE00000000000000000000000000000000000F
:1013DE0000000000000000009C7E040800000000D9
:1013EE00000000009539010850C300000100000004
:1013FE0000000000000000000000000000000000DF
:10140E00000000000000000000000000C092040870
:10141E000000000000000000FD340108A86100007B
:10142E0001000000000000000000000000000000AD
:10143E00000000000000000000000000000000009E
:10144E0094930408000000000000000045380308D3
:10145E00A086010001000000000000000000000056
:10146E00000000000000000000000000000000006E
:10147E0000000000B880040800000000000000001A
:10148E00D5EE0008A00F00000100000000000000D3
:10149E00000000000000000000000000000000003E
:1014AE000000000000000000A093040800000000EF
:1014BE000000000049400208102700000100000053
:1014CE00000000000000000000000000000000000E
:1014DE00000000000000000000000000188004085A
:1014EE00000000000000000061870008A00F00004F
:1014FE0001000000000000000000000000000000DD
:10150E0000000000000000000000000000000000CD
:10151E00009B04080000000000000000CD770308C7
:10152E001A41000001000000000000000000000051
:10153E00000000000000000000000000000000009D
:10154E00000000001C8104080000000000000000E4
:10155E009571020810270000010000000000000035
:10156E00000000000000000000000000000000006D
:10157E0000000000000000000885040800000000C4
:10158E000000000099C603081A4100000100000087
:10159E00000000000000000000000000000000003D
:1015AE00000000000000000000000000AC930408E2
:1015BE000000000000000000A99E0308400D03007B
:1015CE00000000000000000000000000000000000D
:1015DE0000000000000000000000000000000000FD
:1015EE00B49304080000000000000000659E03088C
:1015FE00400D03000000000000000000000000008D
:10160E0000000000000000000000000000000000CC
:10161E0000000000BC930408000000000000000061
:10162E0049A00208A086010003000000000000008F
:10163E00000000000000000000000000000000009C
:10164E000000000000000000698B0208218B0208D8
:10165E00718A020800000000A5870208A589020809
:10166E00458A02080D8902080000000000000000F3
:10167E0099870208011E0308FD1D0308F91D0308C2
:10168E00ED1D0308E91D0308F51D0308F11D0308F0
:10169E00751E0308691E0308411E0308551E030824
:1016AE002D1E0308191E0308051E03085C9B040863
:1016BE000F0000000000000000000000000000000D
:1016CE00D4220020FFFFFFFFFA00000001000000FF
:1016DE0001000000EC930408F49304084091040800
:1016EE0000000000000000000000000000000000EC
:1016FE00E293040804000000D7680308000000000D
:10170E0000000000A8900408010000000000000086
:10171E000000000000000000000000000E000000AD
:10172E000000000000000000000000004AA400209D
:10173E000100C4090000000048A400200100C409F3
:10174E000000000046A400200100C40900000000B3
:10175E0044A400200100C4090000000040A40020A1
:10176E000100C4090000000042A400200100C409C9
:10177E00000000003EA400200100C409000000008B
:10178E003CA400200100C409000000005AAF002054
:10179E000100C8000100000058AF00203200307573
:1017AE003200000057AF0020055A050052AF00204E
:1017BE0000FF010056AF002001000000740F002052
:1017CE0054AF0020020000000457040851AF00205F
:1017DE0000FF010055AF002001000000740F002033
:1017EE0053AF002002000000045704081C940408A4
:1017FE000F000000000000000000000000000000CC
:10180E007C0F0020903A00209CFF2C01000000006D
:10181E00BE0300200A000000945704083CAF0020CD
:10182E00E0150C1700000000BD03002008000000AA
:10183E00CC420408BC03002005000000EC5604084E
:10184E003EAF002002000000AC570408DAB00020C2
:10185E000100FF7F01000000D8B000200200000050
:10186E00B8570408B2AF002003000000C8570408A0
:10187E00B1AF002003000000C8570408B0B000202C
:10188E000000F40101000000AEB000200000F401E1
:10189E0001000000ACB000200000F40101000000C7
:1018AE00AAB000200000F40101000000A8B0002042
:1018BE0000FF0100C4B00020E803D0070A000000BA
:1018CE00C2B00020006401000A000000C3B0002076
:1018DE00006401000A000000BCB00020006401009A
:1018EE000A000000C1B00020006401000A000000E0
:1018FE00C0B00020006401000A000000BFB000204C
:10190E00006401000A000000BBB0002000FF0100CF
:10191E000A000000BAB0002000FF01000A0000001B
:10192E00BAAF00200000F40101000000B8AF0020A3
:10193E000000F40101000000B6AF00200000F40129
:10194E0001000000B4AF00200000F401010000000F
:10195E00B7B0002000C80100B6B0002000C80100DA
:10196E00B5B0002000C80100B4B000200064010032
:10197E000A000000B3B0002000FF01000A000000C2
:10198E00CFB0002000C80100CEB0002000C801007A
:10199E00CDB0002000C80100CCB0002000C801006E
:1019AE00CBB0002000C80100CAB0002000C8010062
:1019BE00C9B0002000C80100C8B0002000C8010056
:1019CE00C7B0002000C801002494040800000000E5
:1019DE000000000000000000000000003494040825
:1019EE00090000000000000020100020040000008C
:1019FE003C940408090000000000000014100020B0
:101A0E0004000000C4990408090000000000000052
:101A1E000810002004000000F483040809000000F0
:101A2E0000000000FC0F0020040000004494040895
:101A3E000900000000000000F00F0020040000006C
:101A4E004C9404080900000000000000E40F002080
:101A5E000400000054940408090000000000000077
:101A6E00D80F0020040000005C9404080900000058
:101A7E0000000000CC0F002004000000A890040815
:101A8E000100000000000000000000000000000047
:101A9E00000000000E00000000000000000000002A
:101AAE000000000034950408000000000000000053
:101ABE0000000000000000009092040807000000E3
:101ACE0000000000441000200000000044950408AF
:101ADE000800000000000000381000200000000088
:101AEE005095040808000000000000002C10002093
:101AFE0000000000A8900408010000000000000093
:101B0E000000000000000000000000000E000000B9
:101B1E0000000000000000000000000058950408BE
:101B2E0000000000000000000000000000000000A7
:101B3E00689504080D0000000000000080100020D1
:101B4E0000000000709504080D0000000000000069
:101B5E0074100020000000007895040807000000B3
:101B6E00000000006C1000200000000080950408AA
:101B7E000D000000000000006010002000000000BA
:101B8E00889504080D00000000000000541000208D
:101B9E0000000000909504080700000000000000FF
:101BAE004C10002000000000A89004080100000066
:101BBE000000000000000000000000000000000017
:101BCE000E000000000000000000000000000000F9
:101BDE0098950408000000000000000000000000BE
:101BEE0000000000909204080C00000000000000AD
:101BFE005CAF002000000000AC9504080C00000053
:101C0E00000000005EAF002000000000BC9504083C
:101C1E000C0000000000000094AF00200000000047
:101C2E00CC9504080C0000000000000088AF0020D6
:101C3E0000000000E09504080C0000000000000009
:101C4E0060AF002000000000EC9504080C000000BE
:101C5E000000000062AF002000000000F4950408B0
:101C6E000C0000000000000064AF00200000000027
:101C7E00089604080C0000000000000066AF00206B
:101C8E0000000000109604080C0000000000000088
:101C9E0068AF002000000000189604080C00000039
:101CAE00000000006AAF0020000000002496040827
:101CBE000C000000000000006CAF002000000000CF
:101CCE00BC8404080C000000000000006EAF002071
:101CDE00000000002C9604080C000000000000001C
:101CEE0070AF002000000000389604080C000000C1
:101CFE000000000072AF002000000000A492040853
:101D0E000C0000000000000074AF00200000000076
:101D1E00449604080C0000000000000076AF00207E
:101D2E0000000000509604080C00000000000000A7
:101D3E0078AF0020000000005C9604080C00000044
:101D4E00000000008CAF0020000000006496040824
:101D5E000C000000000000008AAF00200000000010
:101D6E006C9604080C0000000000000098AF0020E4
:101D7E0000000000789604080C000000000000002F
:101D8E009AAF002000000000849604080C000000AA
:101D9E0000000000A0AF002000000000C092040868
:101DAE000C000000000000007AAF002000000000D0
:101DBE00109204080C0000000000000082AF00200A
:101DCE0000000000909604080C00000000000000C7
:101DDE007CAF0020000000009C9604080C00000060
:101DEE00000000007EAF002000000000A89604084E
:101DFE000C0000000000000080AF0020000000007A
:101E0E00B09604080C0000000000000084AF002013
:101E1E0000000000107F04080C000000000000000D
:101E2E008EAF002000000000BC9604080C000000DD
:101E3E000000000086AF0020000000006C84040843
:101E4E000C0000000000000096AF00200000000013
:101E5E00C89604080C0000000000000090AF00209F
:101E6E0000000000D09604080C00000000000000E6
:101E7E0092AF002000000000D89604080C0000006D
:101E8E00000000009CAF002000000000E096040857
:101E9E000C000000000000009EAF002000000000BB
:101EAE00A8900408010000000000000000000000DF
:101EBE0000000000000000000E0000000000000006
:101ECE000000000000000000E8960408000000007A
:101EDE00000000000000000000000000F89604085A
:101EEE000500000000000000B0AF00200000000060
:101EFE00A89004080100000000000000000000008F
:101F0E0000000000000000000E00000000000000B5
:101F1E000000000000000000009704080000000010
:101F2E0000000000000000000000000038860408D9
:101F3E000000000000000000AC05002004000000BE
:101F4E00F08304080D0000001D690308E010002056
:101F5E00000000008C9104080D0000003D63030892
:101F6E00D410002000000000309604080D00000080
:101F7E0009630308C8100020000000002092040826
:101F8E000800000000000000BC100020040000004B
:101F9E00109204080D000000F5620308B010002036
:101FAE00000000000C97040809000000000000006B
:101FBE00A410002004000000A490040803000000F8
:101FCE0071C503088C10002000000000A8900408C2
:101FDE0001000000000000000000000000000000F2
:101FEE00000000000E0000000000000000000000D5
:101FFE00000000001497040800000000000000001C
:10200E000000000000000000249704080D000000EE
:10201E0000000000F8100020000000002C970408BB
:10202E000A00000000000000F0B0002000000000D8
:10203E00389704080A00000000000000F8B00020E5
:10204E0000000000409704080A0000000000000095
:10205E0000B10020000000004897040808000000AE
:10206E0000000000EC10002000000000A890040802
:10207E000100000000000000000000000000000051
:10208E00000000000E000000000000000000000034
:10209E00000000005097040800000000000000003F
:1020AE000000000000000000649704080D0000000E
:1020BE0000000000101100200000000074970408BA
:1020CE0004000000B56B03080000000000000000D3
:1020DE007C9704080D000000000000000411002091
:1020EE00000000009097040804000000916B0308A4
:1020FE000000000000000000A8900408010000008D
:10210E0000000000000000000000000000000000C1
:10211E000E000000000000000000000000000000A3
:10212E009897040800000000000000000000000066
:10213E0000000000AC97040807000000000000003B
:10214E004C11002000000000B897040808000000A1
:10215E00000000004011002000000000C497040899
:10216E0008000000000000003411002000000000F4
:10217E00D09704080800000000000000281100207D
:10218E0000000000DC9704080800000000000000BA
:10219E001C11002000000000A8900408010000009F
:1021AE000000000000000000000000000000000021
:1021BE000E00000000000000000000000000000003
:1021CE00E89704080000000000000000A7050020AA
:1021DE0000000000F49704080B000000000000004F
:1021EE00B411002000000000FC9704080B00000052
:1021FE0000000000A811002000000000089804084C
:10220E000B000000000000009C11002000000000E8
:10221E00149804080B00000000000000901100202C
:10222E0000000000209804080B00000000000000D1
:10223E0084110020000000002C9804080B00000000
:10224E0000000000781100200000000034980408FF
:10225E000B000000000000006C11002000000000C8
:10226E00409804080B0000000000000060110020E0
:10227E00000000004C980408080000000000000058
:10228E005411002000000000A89004080100000076
:10229E000000000000000000000000000000000030
:1022AE000E00000000000000000000000000000012
:1022BE005898040800000000000000000000000014
:1022CE00000000006C9804080800000000000000E8
:1022DE00E4110020000000007898040808000000B7
:1022EE0000000000D81100200000000084980408AF
:1022FE000800000000000000CC11002000000000CB
:10230E00909804080800000000000000C011002092
:10231E0000000000A890040801000000000000006A
:10232E000000000000000000000000000E00000091
:10233E000000000000000000000000009898040853
:10234E000000000000000000A405002000000000B6
:10235E00A89804080B0000000000000014120020D2
:10236E0000000000B49804080B00000000000000FC
:10237E000812002000000000C098040807000000AA
:10238E00000000000012002000000000CC9804089D
:10239E000700000000000000F811002000000000FF
:1023AE00D89804080700000000000000F01100207B
:1023BE0000000000A89004080100000000000000CA
:1023CE000000000000000000000000000E000000F1
:1023DE00000000000000000000000000E498040867
:1023EE000000000000000000A40500200000000016
:1023FE00F0980408070000000000000060120020A2
:10240E0000000000F898040807000000000000001B
:10241E005812002000000000009904080700000078
:10242E00000000005012002000000000089904086F
:10243E00070000000000000048120020000000000D
:10244E001099040807000000000000004012002050
:10245E0000000000189904080700000000000000AA
:10246E003812002000000000209904080700000028
:10247E00000000003012002000000000289904081F
:10248E0007000000000000002812002000000000DD
:10249E003099040807000000000000002012002000
:1024AE0000000000A89004080100000000000000D9
:1024BE000000000000000000000000000E00000000
:1024CE000000000000000000000000003899040821
:1024DE000F00000000000000096603080000000065
:1024EE0068120020AEAF002017000000D857040875
:1024FE00ADAF00200A320100ACAF002001FA01009E
:10250E00A8AF002000C80100A6AF0020E803D00746
:10251E0001000000424545524F544F5246340000D0
:10252E0050AF0020000301004FAF00200003010058
:10253E00409904080F0000002D6503080965030883
:10254E0000000000441300204C9904080F00000006
:10255E00D16403089164030800000000BC1300203E
:10256E00589904080F0000006965030851650308B7
:10257E000000000070140020649904080F00000091
:10258E001F66030800000000616B03086817002037
:10259E006C9904080F00000055620308000000004B
:1025AE0000000000B8170020749904080F00000006
:1025BE00A96C03087D680308796803089418002045
:1025CE007C9904080F000000456603080000000017
:1025DE000000000034190020849904080F00000048
:1025EE00E9660308B966030800000000C019002060
:1025FE008C9904080F00000065670308AD67030897
:10260E0000000000601A0020B8B000200103010095
:10261E00989904080F0000008566030859660308A0
:10262E0000000000501B0020A09904080F000000BD
:10263E0019670308D96B030800000000DC1B00209B
:10264E00AC9904080F000000DD670308256C030831
:10265E00000000007C1C0020B2B00020010301002D
:10266E00B499040800000000000000000000000003
:10267E0000000000C09904080800000000000000DF
:10268E00A81D002000000000C899040807000000E3
:10269E0000000000A01D002000000000D8990408D2
:1026AE000700000000000000981D00200000000040
:1026BE00E49904080700000000000000901D0020AF
:1026CE0000000000F09904080D000000000000005A
:1026DE00841D002000000000FC9904080300000087
:1026EE0071C503086C1D002000000000A8900408AE
:1026FE0001000000000000000000000000000000CB
:10270E00000000000E0000000000000000000000AD
:10271E0000000000049A0408000000000000000001
:10272E000000000000000000149A04080A000000D7
:10273E0000000000D05A0408000000001C9A040893
:10274E000A00000000000000545A040800000000B7
:10275E00249A04080A00000000000000D0B00020F7
:10276E00000000002C9A04080A000000000000007F
:10277E00B41D002000000000A89004080100000015
:10278E00000000000000000000000000000000003B
:10279E000E0000000000000000000000000000001D
:1027AE00349A040800000000000000000000000041
:1027BE0000000000409A04080300000071C50308E1
:1027CE00001E0020000000005099040803000000C5
:1027DE0071C50308E81D002000000000449904089C
:1027EE000300000071C50308D01D0020000000008A
:1027FE004C9A040805000000000000004EAF0020B7
:10280E0000000000549A04080700000000000000B9
:10281E00C81D002000000000609A04080700000098
:10282E0000000000C01D002000000000A890040859
:10283E000100000000000000000000000000000089
:10284E00000000000E00000000000000000000006C
:10285E00000000006C9A0408000000000000000058
:10286E000000000000000000CC92040803000000ED
:10287E0071C50308481E002000000000809A04085D
:10288E000300000071C50308C00300200000000013
:10289E00889A04080300000071C50308301E00204A
:1028AE0000000000909A04080300000071C50308A0
:1028BE00181E002000000000A8900408010000006F
:1028CE0000000000000000000000000000000000FA
:1028DE000E000000000000000000000000000000DC
:1028EE009C9A040800000000000000000000000098
:1028FE0000000000A89A040807000000716C03088D
:10290E00F81E002000000000AC9604080300000032
:10291E0071C50308E01E002000000000B49A0408F0
:10292E000300000071C50308C81E0020000000004F
:10293E00BC9A04080300000071C50308B01E0020F5
:10294E0000000000C49A040807000000556C03083C
:10295E00A81E002000000000A8910408030000003B
:10296E0071C50308901E002000000000D09A0408D4
:10297E000300000071C50308781E0020000000004F
:10298E00DC9A04080300000071C50308601E0020D5
:10299E0000000000A89004080100000000000000E4
:1029AE000000000000000000000000000E0000000B
:1029BE00000000000000000000000000E89A04087B
:1029CE000F000000C56503088165030800000000C4
:1029DE00001F0020F09A04080F0000004D68030845
:1029EE000000000000000000B41F0020FC9A040844
:1029FE000F0000007564030859640308000000000E
:102A0E0040200020049B04080F000000000000007E
:102A1E000000000000000000F4200020149B0408B9
:102A2E000F000000256803088D6C030800000000ED
:102A3E00802100201C9B0408000000000000000004
:102A4E000000000000000000888A04080300000057
:102A5E0071C50308BC22002000000000089B04087A
:102A6E000300000071C50308A4220020000000002E
:102A7E00009B04080300000071C503088C2200208F
:102A8E0000000000289B04080300000071C5030825
:102A9E007422002000000000349B04080300000094
:102AAE0071C503085C220020000000003C9B040856
:102ABE000200000085C403080000000000000000B2
:102ACE00449B04080200000085C4030801000000B6
:102ADE0000000000509B04080200000085C403089B
:102AEE000200000000000000000000000E000000C8
:102AFE0000000000000000000000000001000000C7
:102B0E004300000000000000000000000000000074
:102B1E0000000000000000000000000000000000A7
:102B2E004300000000000000000000000000000054
:102B3E000000000000000000000000000000000087
:102B4E004300000000000000000000000000000034
:102B5E000000000000000000000000000000000067
:102B6E004300000000000000000000000000000014
:102B7E000000000000000000000000000000000047
:102B8E0043000000000000000000000000000000F4
:102B9E000000000000000000000000000000000027
:102BAE0043000000000000000000000000000000D4
:102BBE000000000000000000000000000000000007
:102BCE0043000000000000000000000000000000B4
:102BDE0000000000000000000000000000000000E7
:102BEE0079000408B9FE0308000000002E9D0408B9
:102BFE00DD930408135F0408135F0408135F0408D1
:102C0E00135F0408135F0408135F0408135F0408BE
:102C1E00135F0408135F0408FFFFFFFFFFFFFFFFB2
:102C2E00FFFFFFFFFFFF0000010041534349490032
:102C3E000000000000000000000000000000000086
:102C4E00000000000000000000004153434949000D
:102C5E000000000000000000000000000000000066
:102C6E000000000000000000000000001025002001
:102C7E000000000000000000000000000000000046
:102C8E000000000000000000000000000000000036
:102C9E000000000000000000000000000000000026
:102CAE000000000000000000000000000000000016
:102CBE000000000000000000000000000000000006
:102CCE0000000000000000000000000000000000F6
:042CDE0001000000F1
:1080000070B4EFF31186502383F31288436B1A6820
:10801000D20720D45D686DB9446A826A944217D051
:1080200081691144D9600ED9A21A5A608462002273
:1080300080F858201A6842F00102F1B21A6081F308
:10804000118870BC704701698A1A5A608562EEE730
:10805000012380F85830F3B283F3118870BC704765
:10806000436A8269D154436A0169426B01338B428E
:1080700028BF00234362002A2FD0EFF31182502340
:1080800083F31288436B1968C9072CD470B45E68F7
:108090006EB9456A816A8D4217D084690C44DC60F0
:1080A0000ED9691A59608562002180F85810196844
:1080B00041F00101D2B2196082F3118870BC70479F
:1080C0000469611A59608662EEE7012380F858302E
:1080D000D2B282F3118870BC7047426DD36843F00E
:1080E0008003D3607047D2B282F31188704700BF1B
:1080F000026B10B462B1836CC2684469D11A013B4F
:10810000615C5DF8044B08BF13468364C8B27047D6
:10811000016A4369C4685B5C0131A14228BF114612
:1081200001625DF8044BD8B2704700BF436B13B1D6
:1081300090F858007047836A406A181AB0FA80F0C5
:1081400040097047416A836A99420AD3CB1A416B4E
:10815000026961B14968501E0B4483420AD2C01AB9
:10816000704702691144CB1A416B0029F2D1501EAD
:10817000C01A704700207047036B43B1826C5B6884
:1081800093422FBF981AC0689B1AC0187047C269E3
:10819000036A9A422FBFD01AC0688018C01A70476D
:1081A0000A4B30B503F10C0493F900205D78072ADF
:1081B000C8BF143A811804338D7213F8025C8554D9
:1081C00013F8012C0A75A342EED130BD74260408C1
:1081D00003682DE9F041DF691FB13B46BDE8F0417E
:1081E0001847002A164611DD04460D460E4400E0ED
:1081F00023689B68204698470028F9D0236815F823
:10820000011B1B6820469847AE42F1D1BDE8F081C2
:1082100000232422027043708370C370704710B52E
:10822000074B03F10C0193F900205C78845402445D
:108230009C78D470DC78947104338B42F3D110BDF8
:1082400080260408F0B5846814B12568A4886C837E
:1082500041F08001446840F2E93501E0002D58D03A
:108260002689013D16F0020FADB2F7D089B2A18187
:1082700040F2E93101E0002960D02589013915F08B
:10828000010F89B2F7D0A189A1894FF0000C4FF4FA
:108290007A714FF6FF764FF0FF0E634502D131E061
:1082A000B1421BD02589013915F0020589B2F7D0FA
:1082B000A4F80CE04FF47A7102E0B9B2B1420DD0EB
:1082C000258915F0010501F1FF37F6D0A589ADB27A
:1082D0000AB1157001320CF1010CDEE7244B9C420F
:1082E00008D0A3F578439C423CD003F580639C42C0
:1082F00008D102251F4B03EB05156B8901339BB297
:108300006B816B89836813B11A689B881383012082
:10831000F0BD17498C4208D0A1F578418C4223D09A
:1083200001F580618C42AFD10225124901EB0515A0
:108330006989013189B269816989A5E70C4DAC422F
:1083400007D00D498C4211D001F580618C429BD140
:108350000221084D05EB01114D890135ADB24D816A
:10836000498991E70125C5E70125DEE70121F0E70D
:10837000003001400CC400200038004030B4846854
:1083800014B12368A5885D83436840F2E93001E0B9
:10839000002833D01D89013815F0020F80B2F7D0C4
:1083A00089B2998140F2E93101E0002950D0188961
:1083B000013910F0010F89B2F7D0998940F2E93103
:1083C00001E000292FD01889013910F0020F89B27D
:1083D000F7D092B29A8140F2E93201E0002A4BD004
:1083E0001989013A11F0010F92B2F7D09B8914B1AB
:1083F0002368A2881A83012030BC70472C498B4225
:1084000008D0A1F578418B424CD001F580618B42B8
:10841000D4D10220274901EB00104189013189B2F2
:1084200041814189CAE7224A934208D0A2F57842A5
:10843000934235D002F580629342D8D102211D4B80
:1084400003EB01114B8901339BB24B814B89CEE782
:108450001748834207D018498B4227D001F5806125
:108460008B42ABD10221134800EB01114889013046
:1084700080B248814989A1E70D498B4207D00E4A55
:10848000934211D002F580629342B0D10222094B8F
:1084900003EB0212538901339BB253815389A6E740
:1084A0000121CCE70120B5E70122F0E70121DAE75D
:1084B000003001400CC4002000380040002870B596
:1084C0001EDB0928044620DD012303EB83035B0048
:1084D000B0FBF3F2092AF8D87BB10E4EB4FBF3F0EF
:1084E0000928CCBF57223022A6FB03E5024403FB38
:1084F0001044EB0801F8012BF0D100230B7070BD84
:108500002D230B7040420131DBE7303001F8010BC5
:10851000F3E700BFCDCCCCCC884230B44FF001049F
:108520002ED301FB04F4B0FBF4F58D42F9D284B1F3
:10853000AAB901E0B0FBF4F5092DCCBF57223022D7
:108540002A4404FB150003F8012BB4FBF1F4002CC2
:10855000F0D100221A7030BC7047B0FBF4F5092D41
:10856000CCBF372230222A4404FB150003F8012B2C
:10857000B4FBF1F4002CF0D100221A7030BC70472B
:108580000546002AEBD1D7E703685A1C0260197030
:10859000704700BF2DE9F047089C2578002B8046E6
:1085A00089460CBF4FF0200A4FF0300A661C35B3E5
:1085B000002A29DD334601E0024698B113F8011B79
:1085C000501E0029F8D1971E60B13D46013D51462D
:1085D0004046C8476B1C002BF8DC257827EAE7707B
:1085E000013055B1041B29464046C847301916F8DA
:1085F000015B002DF7D1BDE8F087BDE8F087002AC8
:1086000004DC2846BDE8F0870020EBE7571EDCE7D6
:1086100083684268D0ED037A00EB83010133934213
:1086200081ED040A836004BF0023836000EB8303B1
:1086300093ED047A036870EE277A9A42C0ED037ACC
:1086400077EEC77AC0ED037A0CDA013307EE103A01
:10865000F8EEC76AB7EE007A87EEA60A036030EE3E
:10866000070A704707EE102AB8EEC77A87EE870A26
:10867000704700BF90ED057A90ED004AD0ED066A94
:10868000D0ED014AD0ED047A90ED035AD0ED025AB4
:10869000A4EE007AB0EE406AB0EE470AB0EE667A19
:1086A000A6EE247A67EEC07AA0EE457AE6EE257A49
:1086B00080ED057AC0ED067A704700BFD0ED057AEF
:1086C00090ED013AD0ED003AD0ED064A90ED024A25
:1086D00090ED077A90ED035A90ED086AD0ED045AB8
:1086E000C0ED067AF0EE406A27EE830AC0ED056A17
:1086F000A3EEA60A80ED087AA4EE240AA5EE470AA6
:10870000A5EEC60A80ED070A704700BFD0ED007ADB
:1087100090ED017A30EE670AE7EE007AB0EE670A74
:10872000C0ED007A704700BF704700BF0A44914215
:1087300014D030B40139551E41F2210211F8014F15
:10874000082380EA042004044CBF82EA4000400071
:10875000013B80B2F7D18D42F0D130BC704700BFF1
:108760002B4B1B7813B12B4B1B7803B970472DE9AA
:10877000F04329490B7803F0FF0E002B46D1274D1B
:108780002B68C31A002B41DB254B264E1A786C68E8
:10879000254BDFF8A890013A570007EB020806EBDB
:1087A00048083A4403EB040C06EB4206B8F80430E0
:1087B0009CF818C07288A9FB03830134DB086C6045
:1087C0000E2C03FB0CF310440C7888BFC5F804E0B2
:1087D00003442B6034B1154803680A780133002A3A
:1087E000FBD10360124A1348134B126800681C8ABD
:1087F000012500230D705460436203889BB22B4314
:10880000038013682B431360BDE8F083BDE8F08359
:10881000044E0020054E0020826A002074250020AE
:10882000846A00203C28040874260408E8750020A7
:108830009025002094250020906A0020CDCCCCCC3F
:1088400070B40F4C0F4E054607CC0023AA60344687
:1088500028606960012200E0A27912F0200F04F183
:10886000180404D101330A2BF6D170BC704703EB16
:10887000430306EBC3031B79EB7270BC704700BF68
:108880009C2604084047040810B4037B01681F2B92
:1088900009D9203B20224C6802FA03F31C4214D170
:1088A0005DF8044B704720220C6802FA03F31C4267
:1088B000F6D00C4A40680024147002685DF8044B3E
:1088C00022F0010202608B607047064A4068002473
:1088D000147002685DF8044B22F001020260CB6064
:1088E000704700BF826A00202DE9F04FDFF81CB20C
:1088F000DFF81CE2BBF80020DEF80860BBF90430AA
:10890000BBF90250BBF90A80C2EB261404FB04F445
:1089100024135200C2EBE60203FB04F305FB02F250
:108920009B1303EBE223B3F5FA364FEAE37589B004
:1089300045F1FF373246A6FB0645CDE9024502FB6D
:1089400007F205EB4202CDE90467029EBBF908403D
:10895000039208FB02FC4FEAE87906FB09CC3A4691
:10896000A8FB0689049ECBF81830E51704FB02F239
:1089700006FB0522A4FB0667E14417444FEA1822D0
:1089800042EA096200924FEA292201923D03DDE9A1
:108990000078340345EA16553F19BBF80660069087
:1089A00048EB05083C1C48F5004503EB8302A4FB9B
:1089B000068906FB0599803213124FEA69064FEAD1
:1089C000E977079356EA07038A4600F09280DDE9CB
:1089D0000489BBF90E20DEF80C40BBF910004946B3
:1089E000C4F5801ED317DDE9024502FB01F108FB47
:1089F0000311A2FB08230B444FEA43492B46C1173E
:108A000000FB03F304FB0133A0FB0401BBF90C40A2
:108A10001944E30001937346DC170023009349EAED
:108A2000D2394FEA4248DDE9002310EB080041EB60
:108A30000901E50712184FEACE744B4145EA5E057D
:108A4000A41A65EB0305221945EB050312196B41C6
:108A500099019001801841EA926159418B0082008E
:108A600043EA9073101943EB05018B00820043EA3F
:108A7000907310460019194632463B46694136F05C
:108A800073FFBBF916204C13450B45EAC14502FBA9
:108A900004F6D31705FB0366A2FB05233344BBF999
:108AA000146002FB04F405FB034406FB01FEA2FB79
:108AB0000523F717234400FB07EE540EA6FB0067BF
:108AC000774444EAC3144FEAD64800194FEA636575
:108AD00048EA473869414FEAE74918EB0008BBF913
:108AE000124049EB01094FEA182646EA09662001BF
:108AF0003618069B0BB1360A1E60BAF1000F02D081
:108B0000079BCAF8003009B0BDE8F08F506900201B
:108B100074250020704700BF704700BF50F8043C28
:108B2000012280F84520103803B11847704700BF74
:108B30004FF4006383827047BFF34F8F0549064BA4
:108B4000CA6802F4E0621343CB60BFF34F8F00BFEB
:108B5000FDE700BF00ED00E00400FA05F8B5057B75
:108B6000466903681F2D29D9A5F120045F682021DB
:108B7000A1400F422A4613D01022A240D960DA60E9
:108B80005A68E240D10703D5012202FA04F4DC60FE
:108B900004463046FFF734FA227B23681F2A20D987
:108BA000A2F1200008215A688140114200D0D9600A
:108BB0000422596882400A4221D1F8BD20211C6854
:108BC000A9400C422A460CD01022AA4099609A6013
:108BD0001A68EA40D207DBD5012202FA05F59D604A
:108BE000D6E7082118689140014200D0996004211D
:108BF000186801FA02F2024203D09A60F8BDDA6006
:108C0000F8BDF8BD70B4037B04681F2B08D9203B66
:108C10002021626801FA03F31A421CD170BC70472C
:108C20002021226801FA03F31A42F7D0426914495D
:108C3000582000FB021251685689CD6808682968DF
:108C400021F001012960828992B222EA0602828122
:108C5000A36070BC704742690949582000FB0212AA
:108C600051685689CD680868296821F0010129609A
:108C7000828992B222EA06028281E36070BC704768
:108C8000EC58002030B4094B1C786CB1084A002520
:108C900002EBC404116893884D628889083203434B
:108CA0009BB2A2428B81F5D130BC7047AC5B0020F7
:108CB000B05B002010B4037B01681F2B09D9203B57
:108CC00020224C6802FA03F31C4214D15DF8044BD5
:108CD000704720220C6802FA03F31C42F6D00C4ABB
:108CE00040680024147002685DF8044B22F0010211
:108CF00002608B607047064A406800241470026866
:108D00005DF8044B22F001020260CB60704700BFA7
:108D1000BF380020F0B5C40022189200AE498B582D
:108D20005B689D8AADB2EEB2F7070A445CD4B70720
:108D300032D5BFF35F8F167EF6B2012E00F0C780EA
:108D4000A64D1A8BBFF35F8F221801EB8202167EAD
:108D5000022E00F0D580221801EB8202167E032E2F
:108D600000F088809A8895F9106092B242F480628F
:108D70009A80221801EB8202127E013296425BD168
:108D8000AA7C00266E74002A40F09580204401EBF6
:108D9000800000234375F0BD77074ED416F04006DF
:108DA00000F0C9808D4D1E8A95F910E0176AF6B261
:108DB00007F80E605FFA8EFE0EF1010C4FFA8CFC84
:108DC000177E85F810C00CF103029742664600F04A
:108DD0001C81221801EB8202127E9445C9D10EF14A
:108DE000020676B22E74C4E71E887C4D26F4006617
:108DF0003604360C1E801E88B6B246F480661E808D
:108E0000967E00272F74002E48D06E7C002E42D014
:108E1000221801EB82020126127E6E74022A00F0F3
:108E2000B980221801EB8202927D42F001021A827F
:108E3000204401EB8000037EF0BD684D967E012743
:108E4000AF74002E73D06E7C002E7BD1221801EB04
:108E50008202527E002A00F0A3801A882E7C92B2F1
:108E6000013642F4007276B21A802E741A88D20546
:108E7000FCD47EE7927E002A3FF474AF6A7C002A1D
:108E80003FF470AF9A8895F9106022F48062120462
:108E9000120C9A806DE7D27DFF2AB9D0221801EB1F
:108EA0008202967D06F0FE061E82D37DFF2BBFD088
:108EB000FF232B74BCE79A8822F4407212042044EA
:108EC000120C01EB80009A8000234375F0BD927E66
:108ED000424D002A3FF435AF6A7C002A3FF431AF9F
:108EE0001A8822F480621204120C1A80BFF35F8F7A
:108EF0001A8B1A88AE7492B242F400721A8031E76B
:108F0000927E002A3FF427AF6A7C002A3FF423AF09
:108F10001A8895F9106022F480621204120C1A80EB
:108F20009A8822F480621204120C9A8021E76A7CEB
:108F3000002A8BD091E715F0800F284D3AD195F992
:108F4000106016E7167ED2F820E01F88022E95F9F1
:108F5000106045D927F480673F043F0C1F801F8AAB
:108F6000FFB20EF806701F88D2F820E0BFB247F4B7
:108F700000771F80F2B21F8A561C76B2FFB20EF83D
:108F800006709F88961CBAB276B242F480622E7444
:108F90009A806BE71A8892B242F400621A8040E726
:108FA0001A8895F9106092B242F4807201271A80F3
:108FB0006F745BE795F91070B7F1FF3F2CD0D6695D
:108FC000F65D1E8292F818E001377AB29645164691
:108FD0002A747FF4CEAEA3E7604D002074250020F4
:108FE000BFB247F400771F801F8AFFB20EF80670E9
:108FF000F6B21F8AD2F820E0721C52B20336FFB2DA
:1090000076B20EF802702E7430E79A8822F48062ED
:109010001204120C9A80DCE6D77D1F822E74957E96
:109020001DB9127E002A7FF403AF9A8822F4806271
:109030001204120C9A80FBE670B5044682B0083028
:10904000656A06236A463B21A847A8B19DF804003B
:109050009DF800609DF801109DF802509DF80320D6
:109060009DF8053041EA062143EA002342EA052241
:10907000E18222836383012002B070BD0023262297
:10908000036002702722C2700122436083608271F4
:1090900043727047F8B50468C4F30D0405460E46E4
:1090A00004B32F681DF07AFB092840F08880454CF6
:1090B000236923F440732361236943F4007323611C
:1090C000236943F0010323613E601DF067FB2369C0
:1090D000092823F00103236171D12B6804332B602D
:1090E0000020F8BD384B394A93422BD902F5804213
:1090F000934226D902F5804293422AD902F5804252
:10910000934228D902F58032934226D902F50032E3
:10911000934224D902F50032934222D902F500325B
:10912000934220D902F5003293421ED902F58022E3
:1091300093421CD9B3F1016F1BD3052005F0EEF863
:10914000FBE708241DF02AFB092814D04FF0FF305C
:10915000F8BD1024F6E71824F4E72024F2E72824C9
:10916000F0E73024EEE73824ECE74024EAE748242F
:10917000E8E75824E6E7134F3B6923F440733B616B
:109180003B6943F400733B613B6923F0F8033B61A7
:109190003B6943F002031C433C613B6943F4803369
:1091A0003B611DF0FBFA3B6923F002033B613B6925
:1091B000092823F0F8033B613FF473AFC6E76FF073
:1091C0000100F8BD003C024000400008FF3F0008DD
:1091D000F8B504460D468E180027B54201D1206926
:1091E000F8BDE368591CE160234415F8012B1A729D
:1091F0000429F2D1206918B9A1682046FFF74AFF77
:109200002061E760E9E700BF70B582B004466946B7
:10921000143027F007FCB0B19DF805009DF80160FF
:109220009DF802109DF803509DF804209DF806302B
:1092300041EA062143EA002342EA0522A187E287A8
:10924000A4F84030012002B070BD00BF38B5254BF6
:109250005C68236B73B1636D626BCAB1998A1A88BB
:10926000C90592B201D5D20700D438BD4FF6F772C6
:109270001A8038BD636D99891A88890692B2EBD538
:109280009206E9D5E26ACAB1988880B29047E2E7CF
:1092900099891A880D0692B2E0D51006DED5A26A29
:1092A000616A8A4219D0A1692569885C9880013277
:1092B000B2FBF5F105FB1122A262CFE79B88E269C0
:1092C0006169DBB28B54E269E068636D0132B2FB25
:1092D000F0F100FB1122E261BEE7DA6822F08002C1
:1092E000DA60BBE7384D002038B5254B1C68236B8E
:1092F00073B1636D626BCAB1998A1A88C90592B25B
:1093000001D5D20700D438BD4FF6F7721A8038BDA8
:10931000636D99891A88890692B2EBD59206E9D5D0
:10932000E26ACAB1988880B29047E2E799891A88C0
:109330000D0692B2E0D51006DED5A26A616A8A42B5
:1093400019D0A1692569885C98800132B2FBF5F1DA
:1093500005FB1122A262CFE79B88E2696169DBB25B
:109360008B54E269E068636D0132B2FBF0F100FBFF
:109370001122E261BEE7DA6822F08002DA60BBE720
:10938000384D002003685B6A03B11847704700BF7F
:1093900003681B6A03B11847704700BF03682DE9D3
:1093A000F041DF691FB13B46BDE8F0411847002A94
:1093B000164611DD04460D460E4400E023689B6806
:1093C000204698470028F9D0236815F8011B1B6830
:1093D00020469847AE42F1D1BDE8F08103689B6911
:1093E000184700BF03685B69184700BF03681B6923
:1093F000184700BF0368DB68184700BF03689B6815
:10940000184700BF03685B68184700BF03681B6804
:10941000184700BF014B1868F8E700BF80C3002061
:1094200038B50C46097849B1054601342B68284601
:109430001B68984714F8011B0029F7D138BD00BFFD
:10944000064B53F820302BB11A689B8851690B42A8
:1094500001D1138370475383704700BFB0CD002004
:1094600003682DE9F04F03F13F4404F57E04604E9C
:10947000A40A0125345D04F01F066409032C05FAD3
:1094800006F500F0AF80042C00F0A780022C54D029
:109490008588B5FA85F0C0F11F0080B2C40803EBDF
:1094A000840400F00700266A80000F27874026EA20
:1094B00007062662276A01F0030602FA00F0721E10
:1094C0003843012AC1F3810CC1F300182062C1F3B3
:1094D000411137D90024224601274FF0030E03E043
:1094E000102A04F1020426D007FA02F0A84302F180
:1094F0000102F5D1D3F800C00EFA04F0C04300EA2F
:109500000C0CC3F800C0D3F8008006FA04FC4CEA47
:10951000080CC3F800C0D3F80CC000EA0C00D860F7
:10952000D3F80CC001FA04F040EA0C00102AD8600D
:1095300004F10204D8D1BDE8F08F2E4C666C35439F
:109540006564A5E7002002464FF0010E4FF00309C5
:1095500004E00132102A00F102003CD00EFA02F7BA
:1095600037EA0504F5D1D3F800A009FA00F4E44382
:109570000AEA040AC3F800A0D3F800B006FA00FA19
:109580004AEA0B0AC3F800A0D3F808A004EA0A0AC2
:10959000C3F808A0D3F808B00CFA00FA4AEA0B0A9C
:1095A000C3F808A0D3F804A02AEA07075F60D3F83D
:1095B00004A008FA02F747EA0A075F60DF683C4048
:1095C000DC60DF6801FA00F401323C43102ADC6001
:1095D00000F10200C2D1BDE8F08F064C266B354386
:1095E000256355E7034C266C3543256450E700BFDF
:1095F0005C48040800380240026802F13F4303F56A
:109600007E032DE9F04F9B0A544DEB5C03F01F05E0
:109610005B090124032B04FA05F400F09980042B64
:1096200000F09180022B3ED001F00306731E012B47
:10963000C1F3810CC1F300188588C1F3411137D9FA
:109640000024234601274FF0030E03E0102B04F102
:10965000020426D007FA03F0A84303F10103F5D171
:10966000D2F800C00EFA04F0C04300EA0C0CC2F8B5
:1096700000C0D2F8008006FA04FC4CEA080CC2F8DC
:1096800000C0D2F80CC000EA0C00D060D2F80CC0C8
:1096900001FA04F040EA0C00102BD06004F102043F
:1096A000D8D1BDE8F08F2E4B5D6C2C435C64BBE7DA
:1096B000002003464FF0010E4FF0030904E0013390
:1096C000102B00F102003CD00EFA03F737EA050434
:1096D000F5D1D2F800A009FA00F4E4430AEA040A3A
:1096E000C2F800A0D2F800B006FA00FA4AEA0B0A63
:1096F000C2F800A0D2F808A004EA0A0AC2F808A03A
:10970000D2F808B00CFA00FA4AEA0B0AC2F808A02C
:10971000D2F804A02AEA07075760D2F804A008FA92
:1097200003F747EA0A075760D7683C40D460D76818
:1097300001FA00F401333C43102BD46000F1020025
:10974000C2D1BDE8F08F064B1D6B2C431C636BE749
:10975000034B1D6C2C431C6466E700BF5C48040887
:109760000038024010B50409013C032C17D80D4BFA
:1097700033F8142000F00F0042FA00F313F0010355
:109780000DD0012303FA00F00138104036F03CF907
:10979000054A064B125D104403EBC00010BD0020CB
:1097A00010BD00BF085A0408045A040824CC002045
:1097B0002DE9F04F4A484B494B4B4C4C4FF0010AB6
:1097C0004FF002094FF004084FF0080C4FF0100E54
:1097D00020274026802530F8022B12F0010F03D0FD
:1097E0001960A3F804A0083312F0020F03D0196027
:1097F000A3F80490083312F0040F03D01960A3F803
:109800000480083312F0080F03D01960A3F804C0D5
:10981000083312F0100F03D01960A3F804E00833E6
:1098200012F0200F02D019609F80083312F0400F11
:1098300002D019609E80083312F0800F02D01960A8
:109840009D80083312F4807F05D04FF4807B19602F
:10985000A3F804B0083312F4007F05D04FF4007B66
:109860001960A3F804B0083312F4806F05D04FF4E8
:10987000806B1960A3F804B0083312F4006F05D0B0
:109880004FF4006B1960A3F804B0083312F4805F42
:1098900005D04FF4805B1960A3F804B0083312F4CC
:1098A000005F05D04FF4005B1960A3F804B00833E3
:1098B00012F4804F05D04FF4804B1960A3F804B028
:1098C0000833D20B04D04FF4004219609A80083359
:1098D00001F58061A1427FF47EAFBDE8F08F00BF4B
:1098E000085A04080000024024CC00200010024066
:1098F00000286AD003682DE9F04F03F13F4404F5D6
:109900007E045F4EA40A0125345D04F01F0664093D
:10991000032C05FA06F559D0042C00F0AC80022C7B
:1099200059D08588B5FA85F0C0F11F0080B2C4080F
:1099300003EB840400F00700266A80000F278740AD
:1099400026EA07062662276A01F003068240701E97
:109950003A430128C1F3810CC1F300182262C1F31C
:1099600041113DD90024224601274FF0030E03E0A8
:10997000102A04F1020426D007FA02F0A84302F1EB
:109980000102F5D1D3F800C00EFA04F0C04300EA9A
:109990000C0CC3F800C0D3F8008006FA04FC4CEAB3
:1099A000080CC3F800C0D3F80CC000EA0C00D86063
:1099B000D3F80CC001FA04F040EA0C00102AD86079
:1099C00004F10204D8D1BDE8F08F70472D4C266C0D
:1099D00035432564A5E72B4C666C35436564A0E7E9
:1099E000002002464FF0010E4FF0030904E001325F
:1099F000102A00F102003CD00EFA02F737EA050403
:109A0000F5D1D3F800A009FA00F4E4430AEA040A05
:109A1000C3F800A0D3F800B006FA00FA4AEA0B0A2D
:109A2000C3F800A0D3F808A004EA0A0AC3F808A003
:109A3000D3F808B00CFA00FA4AEA0B0AC3F808A0F7
:109A4000D3F804A02AEA07075F60D3F804A008FA55
:109A500002F747EA0A075F60DF683C40DC60DF68C6
:109A600001FA00F401323C43102ADC6000F10200EC
:109A7000C2D1BDE8F08F034C266B3543256350E718
:109A80005C48040800380240002855D0026802F102
:109A90003F4303F57E032DE9F04F9B0A544DEB5CE9
:109AA00003F01F055B090124032B04FA05F444D0DD
:109AB000042B00F09780022B44D001F00306731EA4
:109AC000012BC1F3810CC1F300188588C1F341114A
:109AD0003DD90024234601274FF0030E03E0102B4D
:109AE00004F1020426D007FA03F0A84303F10103AE
:109AF000F5D1D2F800C00EFA04F0C04300EA0C0C15
:109B0000C2F800C0D2F8008006FA04FC4CEA080C47
:109B1000C2F800C0D2F80CC000EA0C00D060D2F845
:109B20000CC001FA04F040EA0C00102BD06004F1E4
:109B30000204D8D1BDE8F08F70472E4B1D6C2C432A
:109B40001C64BAE72B4B5D6C2C435C64B5E70020CA
:109B500003464FF0010E4FF0030904E00133102BD0
:109B600000F102003CD00EFA03F737EA0504F5D104
:109B7000D2F800A009FA00F4E4430AEA040AC2F8A1
:109B800000A0D2F800B006FA00FA4AEA0B0AC2F8BE
:109B900000A0D2F808A004EA0A0AC2F808A0D2F885
:109BA00008B00CFA00FA4AEA0B0AC2F808A0D2F888
:109BB00004A02AEA07075760D2F804A008FA03F7BE
:109BC00047EA0A075760D7683C40D460D76801FA73
:109BD00000F401333C43102BD46000F10200C2D1E9
:109BE000BDE8F08F034B1D6B2C431C6365E700BF82
:109BF0005C4804080038024010B1036882885A8328
:109C0000704700BF10B1036882881A83704700BF95
:109C100038B5027B04681F2A44D9A2F12003656885
:109C200020219940294230D02F4D30492B6823F014
:109C300001032B600B899D07FCD52C4B1989090664
:109C4000FCD41B89DD0743D429490B681F2A23F064
:109C500001030B6043D9203A202303FA02F2E260A9
:109C6000224A938823F0030301461B0421481B0C5E
:109C700093800068FFF7C6FF0A7B1F4B0C6800202B
:109C80001F2A187013D9A2F12003102261689A408C
:109C9000114200D0E2600822616802FA03F30B422D
:109CA00014D138BD2023216893400B42BCD110232E
:109CB00021689340194207D10823216803FA02F270
:109CC0000A420BD0A26038BDA360F5E7E36038BD5F
:109CD000064B99891989C907FBD4B5E738BD2023FC
:109CE00003FA02F2A260BBE710600240003C0040B1
:109CF00088600240F07B0020554E002018B10368B8
:109D0000828809B95A8370471A83704710B40A4B86
:109D10000A4A1C7801238340234052F8200029B9C5
:109D2000B3FA83F149095DF8044BE7E7191C18BF42
:109D300001215DF8044BE1E7ACCD0020B0CD00205F
:109D400030B1036882881B691A4214BF01200020C9
:109D5000704700BF2DE9F0410B4E346873691C4019
:109D60000FD0DFF828800127B4FA84F3C3F11F0372
:109D700007FA03F558F8230003689847AC43756168
:109D8000F2D1BDE8F08100BF003C0140F469002041
:109D90002DE9F0410B4E346873691C400FD0DFF899
:109DA00028800127B4FA84F3C3F11F0307FA03F5EF
:109DB00058F8230003689847AC437561F2D1BDE8B9
:109DC000F08100BF003C0140F46900202DE9F04122
:109DD0000B4E346873691C400FD0DFF828800127D0
:109DE000B4FA84F3C3F11F0307FA03F558F823000C
:109DF00003689847AC437561F2D1BDE8F08100BFBC
:109E0000003C0140F46900202DE9F0410B4E34681C
:109E100073691C400FD0DFF828800127B4FA84F35F
:109E2000C3F11F0307FA03F558F8230003689847A6
:109E3000AC437561F2D1BDE8F08100BF003C014048
:109E4000F46900202DE9F0410B4E346873691C4021
:109E50000FD0DFF828800127B4FA84F3C3F11F0381
:109E600007FA03F558F8230003689847AC43756177
:109E7000F2D1BDE8F08100BF003C0140F469002050
:109E80002DE9F0410B4E346873691C400FD0DFF8A8
:109E900028800127B4FA84F3C3F11F0307FA03F5FE
:109EA00058F8230003689847AC437561F2D1BDE8C8
:109EB000F08100BF003C0140F46900202DE9F04131
:109EC0000B4E346873691C400FD0DFF828800127DF
:109ED000B4FA84F3C3F11F0307FA03F558F823001B
:109EE00003689847AC437561F2D1BDE8F08100BFCB
:109EF000003C0140F4690020084A094808B5536C49
:109F000043F4804353640021402238F0FEFA054BAD
:109F10004FF0FF321A60C3F8032008BD003802403A
:109F2000F4690020346A00202DE9F0410446184607
:109F30000D461646984635F04DF82768E6722844D7
:109F4000A07229467D69434632462046AC46BDE8AC
:109F5000F0416047036810B504461B6898472368C2
:109F600020469B689847A37B0133A37310BD00BFB5
:109F700010B5036804469B689847FF23012263736A
:109F8000227310BD08B5FFF7EDFB38B12C228271AA
:109F90000022C2712021BDE8084075E508BD00BF60
:109FA000144B984224D003F58063984220D0028855
:109FB00022F040021204120C0280028822F03803C0
:109FC0001B041B0C59B141F48071002991FAA1F2D4
:109FD000B2FA82F108BF4FF0FF310139C9000B43DB
:109FE0009BB2038003889BB243F040030380704719
:109FF0004908DCE70038004038B5044690F85900BD
:10A00000002857D104F11405A0694FF48071FFF7BF
:10A01000C7FF236E80226B2128469847642004F0F6
:10A0200027FE236E0322682128469847642004F007
:10A030001FFE236E01226B21284698470F2004F053
:10A0400017FE94F85320236E032A8CBF1A2218227D
:10A050001B21284698470F2004F00AFE236E182281
:10A060001C21284698470F2004F002FE236E94F826
:10A0700052201A21284698470F2004F0F9FD236E3C
:10A0800094F85420192128469847642004F0F0FDE4
:10A09000236E10223721284698470F2004F0E8FD50
:10A0A0002846236E382101229847A0690821BDE87F
:10A0B000384075E7FFF756FB0546FFF741FE0146BE
:10A0C00000289FD1D5B12023E871AB712846FFF756
:10A0D000DBFC21460F4B41F8103F284626F038FCA8
:10A0E000AB88B3FA83F3C3F11F03012212FA03F31F
:10A0F00088D009490A6813430B6083E72946FFF7B4
:10A10000C3FC2146034B41F8103F284626F020FCB3
:10A1100078E700BF1D8B0008003C0140F8B5050141
:10A12000684C694B625961199A4204EB050704BFF8
:10A1300001230B730646387A33F026FF3B7A03F08F
:10A140001F015B090122032B02FA01F26DD0042BDF
:10A1500066D0022B5CD0631901361879FFF702FB39
:10A16000F6B2074610B11223C6718371631958798C
:10A17000FFF7F8FA10B11323C67183716319987948
:10A18000FFF7F0FA10B11423C671837166190A2122
:10A19000F2793846FFF7ACFB7079FFF7E3FAF27912
:10A1A0000A21FFF7A5FBB079FFF7DCFAF2790A2163
:10A1B000FFF79EFB6359454A934247D0424A934278
:10A1C00050D0434A934259D0424A934262D0424AC5
:10A1D00093426BD0414A93422CD02C44227BE2B96B
:10A1E00001200222198801F4415141F445710A43CA
:10A1F00002431A809A8B22F400621204120C072187
:10A200009A8319821A8892B242F040021A80F8BDED
:10A21000334B596A0A435A629DE700200246E1E740
:10A220002F4B19690A431A6195E72D4B196A0A43A6
:10A230001A6290E702F564424FF40010536A43F447
:10A24000001353621CF0A2F96359C6E702F5843289
:10A250004FF48050536A43F4805353621CF096F9D4
:10A260006359BAE702F500324FF48040136A43F4B1
:10A27000804313621CF092F96359AEE702F5FE3297
:10A280004FF40040136A43F4004313621CF086F954
:10A290006359A2E702F582324FF40050536A43F447
:10A2A000005353621CF072F9635996E702F5684255
:10A2B0004FF48010536A43F4801353621CF066F924
:10A2C00063598AE70CC40020003800400030014088
:10A2D000003C004000340140005001400054014067
:10A2E00000380240427A02B9704710B5044603684C
:10A2F000406804F10A0198470023637210BD00BF53
:10A30000437A5A1C0344D2B242729972037A93423E
:10A3100000D802B9704710B504460368406804F1DC
:10A320000A0198470023637210BD00BF302828D06F
:10A33000312828D0322828D0332828D0342828D0D3
:10A34000352828D0202828D0212828D0102828D007
:10A35000112828D0122828D0132828D0142828D033
:10A36000152828D0162805D0172808BF0F2202D09C
:10A37000002070470E22114B03EB420393F8350087
:10A3800070470022F7E70122F5E70222F3E70322F4
:10A39000F1E70422EFE70522EDE70622EBE70722CB
:10A3A000E9E70822E7E70922E5E70A22E3E70B22CB
:10A3B000E1E70C22DFE70D22DDE700BF7426040889
:10A3C00070B5448806460D46C4F30B0422460021AE
:10A3D000284638F09AF83369094A934209D3094A62
:10A3E000934206D2224628461946BDE8704035F011
:10A3F00075BD23B121462846BDE87040184770BDA1
:10A40000680600086E070008064B07498B4202D316
:10A410000023184670471A88C2F30B029042F8D006
:10A420001433F3E79001000868060008024A136835
:10A4300023EA000010607047ECB00020F8B5174D1B
:10A440002B78A32B28D16B78BE2B25D1022229464D
:10A450004FF6FF70FEF76AF9114FAC1C22884AB123
:10A46000A618BE4218D2052A16D92146FEF75EF973
:10A470003446F3E721460222FEF758F90222A118DA
:10A48000FEF754F90634074B641B1C8041F60F534A
:10A49000C31A58425841F8BD0020F8BD00400008DA
:10A4A000008000082E3500202DE9F04FDFF84C9198
:10A4B0004D4F8BB00326A7EB09071822002104A8F3
:10A4C00038F023F8494BCDF8109005971A69002A07
:10A4D00004DA474A5A6002F188325A6001228DF844
:10A4E0002420F322DA60434B434C1B88ADF8003044
:10A4F0000222694604A8FEF76BFE022269464FF667
:10A50000FF70FEF713F9DFF8F8A080464FF0000B5C
:10A51000544539D30AAC002524F8245D0222214693
:10A5200004A8FEF755FE022221464046FEF7FEF83B
:10A5300040BAC043ADF80800022202A904A8FEF701
:10A5400047FE079878B106ABC0F1040229461844CB
:10A5500037F0DBFF089818B9069904A8FEF79AFDB2
:10A560000023089007939DF82430089A23B11F49CF
:10A570000B6943F000430B61013E2DD0002A9CD1B2
:10A58000FFF75CFF50B32CE065888DF80DB0C5F384
:10A590000B05AB1DADF808302388C3F30B02ADF8F3
:10A5A0000A201B0B062202A904A88DF80C30FEF726
:10A5B0000FFE062202A94046FEF7B8F86168804601
:10A5C0002A4604A8FEF704FE616840462A46FEF7C4
:10A5D000ADF8143480469BE7002AD1D0052003F063
:10A5E0009DFE0BB0BDE8F08F00800008003C0240EB
:10A5F00023016745C82604089001000800400008B0
:10A60000680600080378202B024600F10100F9D00B
:10A61000092BF7D02D2B2CD02B2B03BF5378B7EE63
:10A62000000A0246B7EE000AA3F13001C8B20928B9
:10A630009FED467A10D8F2EE046A07EE901AF8EE13
:10A64000E77A12F8013FE7EE267AA3F13001C8B2AB
:10A650000928B0EE677AF0D92E2B4CD003F0DF0337
:10A66000452B0BD0F7EE007A67EE276A20EE260A1C
:10A6700070475378BFEE000A0246D5E710B4517810
:10A680002D2959D02B290ABF9178501C901C0024E9
:10A69000A1F13003092B53D8002303EB830301EB13
:10A6A000430310F8011FA1F13002092AA3F130037E
:10A6B000F3D9B3F59A7F28BF4FF49A73072B42D989
:10A6C000DFED236A1A46F7EE007A083A072A67EEAA
:10A6D000A67AFAD803F007032BB1F2EE046A013B25
:10A6E00067EEA67AFBD124B3C7EE276A5DF8044B68
:10A6F00020EE260A70475378A3F13001C8B209282A
:10A7000002F10102AAD8F2EE046AF0EE665A07EEF0
:10A71000901AF8EEE77A12F8013F87EEA66AA3F1E5
:10A720003001C8B2092866EEA56A37EE067AEED97E
:10A7300094E767EE276AD9E7901C91780124A7E790
:10A74000F7EE007ACFE7F7EE007AC5E700000000E9
:10A7500020BCBE4CB5EEC00ADFED317AF1EE10FA46
:10A76000CCBF30EE270A30EE670ADFED2E7A20EEFE
:10A77000270A30B5FDEEC07A87B017EE904A05463D
:10A7800084EAE470002303A9A0EBE4700193009332
:10A79000029323F0DDFE002CACBF20232D2303A861
:10A7A0008DF8003034F016FC012803A924D00228CB
:10A7B0002DD0032805BF3023684668468DF8013048
:10A7C00037F0C9FE684634F005FC0338C4B22246AF
:10A7D0006946284637F01DFF00232B55284634F0E4
:10A7E000F9FB2E22431C2A540DEB0401E81837F024
:10A7F000CFFE284607B030BD302368468DF80130C3
:10A800008DF802308DF8033037F0A5FEDAE73023FB
:10A8100068468DF801308DF8023037F09CFED1E7A4
:10A820006F12033A00007A442DE9F04106461546BE
:10A830000846B6FBF2F43CB905FB1464124B1B5DF1
:10A8400000F8013BBDE8F081B4FBF2F767B90E4BAD
:10A8500005FB174705FB1464DA5D00F8012B1B5D4F
:10A8600000F8013BBDE8F081B7FBF2F8B8F1000F4A
:10A8700002D04046FFF7D8FF05FB1878024B13F8CB
:10A88000082000F8012BE3E7105A040830B40268EE
:10A890001146531C036011F8024B0160D31C517820
:10A8A00003609378151D05601B0443EA0123D078EB
:10A8B000234343EA006030BC704700BF0368591C63
:10A8C0001A46016012F8021B0260587841EA002023
:10A8D000704700BF03685A1C02601878704700BFB9
:10A8E00038B504460068154635F0F8FA22682A445F
:10A8F000226038BD036810B40A0E5C1C04601A7034
:10A9000003680A0C5C1C04601A7003680A0A5C1C69
:10A9100004601A7003685A1C026019705DF8044BD9
:10A92000704700BF036810B40A0A5C1C04601A7008
:10A9300003685A1C026019705DF8044B704700BF31
:10A9400003685A1C026010B4197003680A0A5C1C80
:10A9500004601A7003680A0C5C1C04601A700368B7
:10A96000090E5A1C026019705DF8044B704700BF55
:10A9700003685A1C026019700368090A5A1C0260B5
:10A98000197070472DE9F047002488B080460F46C3
:10A990001E46A14605AD531C0393117839B32529F2
:10A9A00033D1931CCDF810900393507830284ED0BB
:10A9B0004FF0000AA0F13003DBB2092B42D96C281A
:10A9C00019D0642800F0938024D825281CD063D99E
:10A9D000582876D063281BD131784046B847039A6F
:10A9E000531C03931178043601340029D7D1204633
:10A9F00008B0BDE8F087039B5A1C03921B78642BB8
:10AA00007CD02AD8252B54D1252140460134B84783
:10AA1000039AC0E7732833D044D975284FD106F183
:10AA2000040E30682B4600220A217646FDF774FD9D
:10AA3000049A0095534639464046FDF7ABFD039A0C
:10AA40000444A8E704AA03A926F07EFDB7E7D31CB7
:10AA5000039390784FF0010AACE7732B10D05BD9C9
:10AA6000752B3AD0782B96D1A3F15802B2FA82F224
:10AA7000306852092B4610210436FDF74DFDD7E70B
:10AA80003368049A0093394600234046FDF782FD5F
:10AA900004360444039A7EE70028B9D1204608B062
:10AAA000BDE8F0876E28B3D1039A336804361C6082
:10AAB00071E72AD9582BD7D0632B8DD06BE7782834
:10AAC000A6D1A0F15802B2FA82F2306852092B46A0
:10AAD0001021FDF721FD0436AAE706F1040E3068C7
:10AAE0002B4600220A217646FDF716FDA0E7331D0E
:10AAF000306829461E46FDF7E1FC99E7331D3068B2
:10AB000029461E46FDF7DAFC92E7002B7FF443AF9F
:10AB1000204608B0BDE8F0876E2BC6D03BE700BFEB
:10AB20000EB400B584B005AB019053F8042B064970
:10AB3000039301A8FFF726FF019B00221A7004B0BF
:10AB40005DF804EB03B07047898500080FB430B599
:10AB500083B006AB0A490B4853F8042B0968006818
:10AB60000193FFF70FFF084C05462068FEF73AFCFB
:10AB70000028FAD0284603B0BDE8304004B0704742
:10AB80002C4D0020304D002080C30020DFED2B7ABB
:10AB9000B4EEE70AF1EE10FA4ADDDFED296A9FED27
:10ABA000297A01E0B0EE670AB4EEC70AF1EE10FAB6
:10ABB00070EE667AF6DC9FED247AF4EEC77AF1EE59
:10ABC00010FA38D5DFED1E6A9FED207A01E0F0EE35
:10ABD000407AF4EEC77AF1EE10FA37EEA60AF6D410
:10ABE000DFED1B7AB4EEE70AF1EE10FA14DDDFEDCB
:10ABF000137A37EEC00A60EE006A9FED166A9FED89
:10AC0000167ADFED167AA6EE867A20EE266AE6EE52
:10AC1000877AA6EE270A7047DFED117AB4EEE70ACD
:10AC2000F1EE10FA44BFDFED087A37EEC00AE2E732
:10AC3000F0EE407ABFE7B0EE670AD1E7DB0F49409C
:10AC4000DB0FC940E4CB1641DB0F49C0E4CB16C192
:10AC5000DB0FC93F92E741B99730083C15A82ABEDF
:10AC6000DB0FC9BF80EAE073A3EBE0738B4205DB27
:10AC7000002801DD401A704702D17047002070475C
:10AC80000844704709B909E0194690FBF1F301FB4C
:10AC900013030846002BF7D1084670470146FBE72F
:10ACA000F0EEC07AB0EEE07AB4EEE77AF1EE10FAA8
:10ACB000B4BFB0EE676AB0EE476AB5EE406AF1EE37
:10ACC00010FA46D0B4EEE77AF1EE10FA8CBFF0EE4F
:10ACD000675AF0EE475AC5EE866A9FED1F3A9FED20
:10ACE0001F6A9FED1F4A9FED1F5ADFED1F3ADFEDF0
:10ACF0001F4ADFED1F5AA6EEC36AE6EEA34AA6EE90
:10AD0000864AB7EE006AA6EE845AA6EEA46AE6EE7C
:10AD1000855AC5EE866AB4EEE77AF1EE10FA48BFBE
:10AD2000DFED147AF5EEC00A48BF77EEE66AF1EE81
:10AD300010FA48BFDFED107AB5EEC00A48BF77EED3
:10AD4000E66AF1EE10FA48BFF1EE666AB0EE660A06
:10AD50007047DFED076ADEE739094E3DE3B59E3EF9
:10AD600088FA163E45FE7F3F99FB243F69A2163EB6
:10AD7000A7DFA834DB0FC93FDB0F4940DFED317A95
:10AD800030EE277AFDEEC76A16EE903A2033402B5C
:10AD900002D99FED2D0A7047B4EEE70AF1EE10FAE2
:10ADA0004DDD9FED2A6ADFED2A6A01E0B0EE677A99
:10ADB000B4EEE67AF1EE10FA77EE467AF6DC9FED25
:10ADC000257AF4EEC77AF1EE10FA35D5DFED1F6A79
:10ADD0009FED217A01E0F0EE407AF4EEC77AF1EED1
:10ADE00010FA37EEA60AF6D4DFED167AB4EEE70ACB
:10ADF000F1EE10FA1BDCDFED197AB4EEE70AF1EEA2
:10AE000010FA44BFDFED137A37EEC00A60EE006A35
:10AE10009FED136A9FED137ADFED137AA6EE867A23
:10AE200020EE266AE6EE877AA6EE270A7047DFED67
:10AE30000F7A37EEC00AE9E7B0EE670AD4E7F0EE22
:10AE4000477ABCE7DB0FC93F00000000DB0FC940B9
:10AE5000E4CB1641DB0F49C0E4CB16C1DB0FC9BF01
:10AE600092E741B99730083C15A82ABEDB0F49404C
:10AE7000FDEEC07A17EE903A2033402B51D8DFED2B
:10AE80002D7AB4EEE70AF1EE10FA50DDDFED2A6A12
:10AE90009FED2A7A01E0B0EE670AB4EEC70AF1EE40
:10AEA00010FA70EE667AF6DC9FED257AF4EEC77A3A
:10AEB000F1EE10FA38D5DFED206A9FED227A01E03D
:10AEC000F0EE407AF4EEC77AF1EE10FA37EEA60A09
:10AED000F6D4DFED1D7AB4EEE70AF1EE10FA1BDCD2
:10AEE000DFED1A7AB4EEE70AF1EE10FA44BFDFEDB7
:10AEF000147A37EEC00A60EE006A9FED156A9FED86
:10AF0000157ADFED157AA6EE867A20EE266AE6EE51
:10AF1000877AA6EE270A7047DFED067A37EEC00A79
:10AF2000E9E79FED0E0A7047B0EE670AD1E7F0EE51
:10AF3000407AB9E7DB0F4940DB0FC940E4CB16414B
:10AF4000DB0F49C0E4CB16C1DB0FC93FDB0FC9BF24
:10AF500092E741B99730083C15A82ABE00000000CE
:10AF600010B507EE901A2DED028BB8EE678ADFED73
:10AF7000217A28EE008A044628EE278AB0EE480A95
:10AF800035F002FAF0EE408AB0EE480A35F05EF98C
:10AF9000F7EE007A9FED187AF0EE675AE8EE875ADE
:10AFA0000023A361B0EE676AC7EEA56A63612362FE
:10AFB000E361A8EEC76ABDEC028B77EEC07AB6EE0D
:10AFC000007AF8EE005A27EE877A20EE250A27EE5F
:10AFD000267A26EE266A67EEA67A20EE260A84ED09
:10AFE000046AC4ED017A84ED007A84ED027A84ED7E
:10AFF000030A10BD27D4D236F304353F10B44C09F0
:10B00000012250F8243001F01F0102FA01F10B4334
:10B0100040F824305DF8044B704700BF4B0901F045
:10B020001F0150F82320012303FA01F1114214BF3C
:10B0300018460020704700BF2DE9F84F294A1378C1
:10B0400003F0FF04002BFAD1DFF8A880264FD8F8D0
:10B050000000DFF8A490254D01233B70FEF7CCFDE6
:10B06000052033F061F8204633F05EF8062033F017
:10B070005BF8204633F058F899F80060042046F059
:10B08000010633F051F8304633F04EF82B8893B177
:10B09000DFF868A0164E1AF804B0072033F044F821
:10B0A000584633F041F81AF804202B883255013401
:10B0B000A4B2A342EFD8072033F036F8FF2033F0D4
:10B0C00033F899F80040042033F02EF8204633F08E
:10B0D0002BF8D8F80000FEF795FD00233B70BDE883
:10B0E000F88F00BF554E00208153002048030020F8
:10B0F00098530020F07B002089530020584E0020F8
:10B100002DE9F041474E3068FEF776FD464B1B783F
:10B11000012B78D05FD3022B0AD1DFF82C810823D2
:10B1200088F800300D254FF4C373404F3B8010E08A
:10B13000DFF814813D4F98F8003003F04003002BF6
:10B1400014BF4FF4F0734FF4C3733B8014BF10254A
:10B150000D25002404F11000C0B232F0E5FF0134E7
:10B16000012032F0E1FFA3B2AB42F3D398F80040E4
:10B170002F4D002032F0D8FF204632F0D5FF2D4B66
:10B180001C78022032F0D0FF204632F0CDFF2A4B4F
:10B190001C78032032F0C8FF204632F0C5FF274B51
:10B1A0001C780420044332F0BFFF204632F0BCFF7D
:10B1B0003068FEF727FD3A882148002137F0A5F9CD
:10B1C0002B7833B11F4B1B7833B300232B70BDE8B2
:10B1D000F081BDE8F081A02032F0A6FF002032F01F
:10B1E000A3FF00F00603022BDFF85C8007D000F01D
:10B1F0000500012803D1482388F8003008E008231F
:10B2000088F800308EE7DFF84080482388F8003067
:10B2100010254FF4F07388E7FFF70EFF00232B7023
:10B22000BDE8F081F07B0020087C0020480300206E
:10B23000000000200F7C0020107C0020895300209B
:10B240009853002081530020500300200C4B98425B
:10B2500013D0A3F5806398420FD003F58043984242
:10B260000BD003F58063984207D003F580639842C2
:10B2700003D0044B186840087047024B18687047A9
:10B28000000401400C7D0020F0B5774B774A87B071
:10B290001968914200AF00F0DB800023744A3B60E4
:10B2A0007B60136843F48033136003E03B68B3F5BD
:10B2B000A04F09D0136803F400337B603B6801336F
:10B2C0003B607B68002BF1D0694B1B6813F40033A3
:10B2D00018BF01237B607B68012B7BD0654D644BDD
:10B2E000654AEA606549586F654A0860AA605E6B06
:10B2F000644C654A654826F080065E635E6F46F0E2
:10B3000080765E67196B0C431C63596B5963996BAC
:10B310009963196C41F05B5141F47B1141F41F6159
:10B3200041F00F011964596C07F118040A4348F2FF
:10B33000FF715A6444F8101D002621460123FB7357
:10B340003E737E73BE731AF0FFFF21464FF6FF7304
:10B350004F48BB601AF0F8FF4FF6FF7321464D4887
:10B36000BB601AF0F1FF21464B481AF0EDFF214671
:10B370004A481AF0E9FF214649481AF0E5FF2146FC
:10B3800048481AF0E1FF214647481AF0DDFF214600
:10B3900046481AF0D9FF20461BF0B6F9444B454CFD
:10B3A0001B68BA6844484549A4FB03439B09A0FBBA
:10B3B0000202013B920CB3F1807F0A6007D2404A3F
:10B3C000F0200721536085F82300966011601C3738
:10B3D000BD46F0BD264B3B4C1A6C3B4942F08052B7
:10B3E0001A6420688A684D68C96840F4404020604B
:10B3F000986898609868120640F40040986042EAA5
:10B400008512986842F48002490842F00802013926
:10B4100042EA014240F4A05098605A601A6842F033
:10B4200080721A601A689201FCD52849104A40F2CD
:10B4300005700860996821F003019960996841F0EE
:10B4400002019960936803F00C03082BFAD145E7D9
:10B4500000221A6062B61E4B1B6883F308881D4BDE
:10B460001B689847FEE700BFFCFF0120EFBEADDE82
:10B470000038024000ED00E00005FA05A85D00205C
:10B4800000000008FF916700335F070000000240E2
:10B490000004024000080240000C0240001002407C
:10B4A0000014024000180240001C0240002002402C
:10B4B0000C7D0020D34D621083DE1B4308C40020A6
:10B4C00010E000E00070004000000020003C02405E
:10B4D0000000FF1F0400FF1F08B5054B1B6803B1E8
:10B4E0009847044B044A1A6072B6FDF725FB00BF6B
:10B4F000A8300020FCFF0120EFBEADDE08B5034BF5
:10B500001B6803B1984772B6FDF716FBA830002000
:10B51000084B10B507281B68C8BF143818440C46E0
:10B52000007DFEF71FF920B12146BDE81040FEF76F
:10B53000E5BB10BD606A002030B50446406D617106
:10B540008389A26823F400531B041B0C838185B0FC
:10B55000A379009213F0040230D04FF4805213F01C
:10B560000203ADF8042056D1ADF806304FF48063E5
:10B570000022ADF8083011F00103ADF80C2028D1FD
:10B58000ADF80A3008238D07694648BFADF80A3088
:10B590001BF050F9A279636DD10724D412F0080F83
:10B5A0009A8A1BD122F008021204120C9A829A89FC
:10B5B00092B242F400529A8105B030BD13F00203FA
:10B5C000ADF8042024D04FF400551346ADF80650D2
:10B5D000CEE70423ADF80A300C23D4E792B242F050
:10B5E00008029A82E3E70D498B420FD0A1F54C4146
:10B5F0008B4209D00A498B42D0D102200121FFF7AA
:10B6000087FFA279636DC9E70120F7E70020F5E71E
:10B61000ADF80630ACE74FF40053A5E70010014049
:10B620000048004010B50446406DA160838923F4B2
:10B6300000531B041B0C8381A37984B013F0040214
:10B64000009135D04FF4805213F00203ADF804207E
:10B6500056D1ADF806304FF480636279ADF808300A
:10B66000D1074FF00003ADF80A30ADF80C3045BFFC
:10B670000423ADF80A3008230C236946920748BF1B
:10B68000ADF80A301BF0D6F8A279636DD1071FD44C
:10B6900012F0080F9A8A16D122F008021204120C36
:10B6A0009A829A8992B242F400529A8104B010BDF3
:10B6B00013F00203ADF804201FD04FF400511346DD
:10B6C000ADF80610C9E792B242F008029A82E8E7A4
:10B6D0000D498B420FD0A1F54C418B4209D00B494B
:10B6E0008B42D5D102200121FFF712FFA279636DB1
:10B6F000CEE70120F7E70020F5E7ADF80630ACE72C
:10B700004FF40053A5E700BF00100140004800407F
:10B7100038B50D4B07281B68CCBFA0F114040446B4
:10B7200023440546187DFEF71DF858B10134272241
:10B73000C47182710121FEF7A7F928460021BDE8F6
:10B740003840E5E638BD00BF606A0020064A0023A5
:10B750005168814202F11C0204D00133102BF7D151
:10B7600000207047D8B27047BC00002070B50F4C65
:10B770000F4DC0EBC00004EB8004286B26693043FA
:10B78000286382B09209667BA1600025012101A88F
:10B7900063618DF804608DF805208DF806508DF8F2
:10B7A00007101BF00FF802B070BD00BFBC000020F6
:10B7B00000380240074BC0EBC00030B403EB800000
:10B7C000054C0569236B2B4323630176427630BC1D
:10B7D000704700BFBC000020003802402DE9F04156
:10B7E0008B4BDD7A98B045B11B78022B0BD0032B25
:10B7F00000F0F780012B00F0E180864B00221A70E8
:10B8000018B0BDE8F081844C844BC4F8543B00264A
:10B810004FF41B7318224AF29E37626004F1140041
:10B8200031461A46A7602670236136F06EFE284620
:10B8300025F000FB7A4FC36802683A600646002B89
:10B8400000F0B6802846FDF78DFF764B186018B1E2
:10B85000292200238271C371327A4A21FEF748F807
:10B8600000222921307DFFF7A5FF0023C0226E4969
:10B87000307DFFF77BFF386802F0F2FC32F084FB8A
:10B880003D686A4AA188284602FB01F1FFF7DEFC09
:10B890008142034640F2B580002218A9284621F8CB
:10B8A0005C2D00250132B3FBF2F3A268B3FBF2F387
:10B8B000C3F34E029BB2A2810293ADF80C50ADF8D7
:10B8C00006508DF80E5025F06BFA0695ADF81C5019
:10B8D000ADF81E50ADF82050ADF82250F379ADF818
:10B8E00012506022ADF810205A07ADF8145000F144
:10B8F000848001214FF48072ADF81210ADF8202041
:10B90000002503F00203ADF81C30069504AA7179F6
:10B910003868DFF8308102F065F87179386825F011
:10B920000FFA3A68F068B2F84430C8F800006FEADD
:10B9300043436FEA53439BB2A2F84430036823F0B9
:10B94000010303601AF08AFD09A81AF049FD3B685B
:10B95000707922693169364C0D92343303444022A8
:10B960000A934FF4806309910B9409A90C920F93E9
:10B970004FF480424FF40033D8F800000E954FF496
:10B98000805412951192139310941AF03BFD737921
:10B9900039680C2B9CBF274A32F813508B89D8F892
:10B9A00000209BB21D438D81136843F01003136088
:10B9B000184B01221A7025F09DFA21E7164C1E49FA
:10B9C00023701E4EC4F8541B4FF43473182704F12F
:10B9D00014001A4600216760A660236136F095FDC9
:10B9E00025E70D4C164BC4F8543BC823122749F2E7
:10B9F000704604F114001A46ECE70422ADF8142056
:10BA00007EE700EB5102B2FBF1F2013A92B244E759
:10BA1000846A0020044E0020906A0020CC2604088E
:10BA200094250020982500208988000840420F00B6
:10BA3000A46A0020E0460408D0260408CE070700C8
:10BA4000D4260408902500202DE9F04F534C54F8DB
:10BA5000204083B0002C00F09C80E56D002D00F0AC
:10BA60009A8017464E4A9846064604F162032869B2
:10BA7000226004F262226361A2614FF400736A687B
:10BA8000A160E36023616265A24668B1FFF75EFED4
:10BA9000721CD2B20C21FFF78DFE636DA9682A6972
:10BAA00022630433A1632365E868A0B1FFF74EFE6B
:10BAB000721C8146D2B20B21FFF77CFE2346EA7F3F
:10BAC00038494846FFF752FE636DA968EA68626329
:10BAD0000433E163E36494F86100FDF743FE8146BB
:10BAE00094F86000FDF73EFE8346287F00284DD184
:10BAF00018F0080F36D1BA070DD5B9F1000F0AD0EA
:10BB00000B22731C89F8062089F8073048466A7FA3
:10BB10002221FDF7EDFEFB0715D4A36B7BB995F849
:10BB20002020A97F8DF8063001A8930901228DF805
:10BB300005308DF804108DF807201AF043FE5046AA
:10BB400003B0BDE8F08FBBF1000FE6D001360C2347
:10BB50008BF807608BF8063058466A7F2221FDF784
:10BB6000C7FEDAE70136F6B2B9F1000F04D00B23B5
:10BB700089F8076089F8063018F0100F484614BF9E
:10BB8000022112216A7FFDF7B3FEC6E732F0FCF90D
:10BB9000AEE7A246D3E7AA46D1E700BF384D002062
:10BBA000D82604085D8B00080348D0F8AC3113B1E7
:10BBB00000F5D27018477047BC0000200348D0F849
:10BBC000903113B100F5C47018477047BC000020D5
:10BBD0000348D0F8743113B100F5B67018477047B8
:10BBE000BC0000200348D0F8583113B100F5A8700C
:10BBF00018477047BC0000200348D0F83C3113B10F
:10BC000000F59A7018477047BC0000200348D0F830
:10BC1000203113B100F58C7018477047BC0000202C
:10BC20000348D0F804310BB1FC301847704700BF0F
:10BC3000BC0000200348D0F8E8300BB1E0301847D2
:10BC4000704700BFBC0000200348D0F8CC300BB1D7
:10BC5000C4301847704700BFBC0000200348D0F82C
:10BC6000B0300BB1A8301847704700BFBC000020AF
:10BC70000348D0F894300BB18C301847704700BFA0
:10BC8000BC0000200248836F0BB17030184770472A
:10BC9000BC0000200248C36D0BB1543018477047F8
:10BCA000BC0000200248036C0BB1383018477047C5
:10BCB000BC0000200248436A0BB11C301847704793
:10BCC000BC0000200248836803B11847704700BFDA
:10BCD000BC000020431C00F00E812DE9F04F4FEA1C
:10BCE000C00808EB00039B00DFF8E8A25AF803B095
:10BCF00087B00AEB0304BBF1000F00F0F9801433A6
:10BD00000AEB03010022DBF804704AF803204A60C2
:10BD10008A60CA600346A56801900133D4F80C908C
:10BD2000DBB2002D00F0E8801522EB71AA71B9F1A9
:10BD3000000F00F0FA80162289F8062089F80730F3
:10BD40009BF80E0032F020F9BB8823F440731B04EB
:10BD50001B0CBB802846FDF755FF4846FDF752FFF8
:10BD600011212846FDF748FC11214846FDF744FC07
:10BD70000826642403E03CB132F024F9013C284653
:10BD8000FDF7DEFF0028F6D02846FDF735FF32F03C
:10BD900019F92846FDF736FF32F014F9013EEED1CD
:10BDA0004846FDF729FF32F00DF92846FDF724FF3C
:10BDB00032F008F92846FDF725FF32F003F948462E
:10BDC000FDF720FF019B08EB03040AEB84042846DF
:10BDD000637C002B0CBF122132210422FDF788FD69
:10BDE000637C002B0CBF1221322148460422FDF750
:10BDF0007FFD704B9F4200F0B7806F4B9F4200F079
:10BE0000BD806E4B9F4200F0A580BB8801996C4AB3
:10BE10006C4C23F440731B041B0CBB803B88884490
:10BE20000AEB880A9BB243F001039AF810103B809A
:10BE3000BD8802A8002918BF14461AF065FC049AB0
:10BE40006148B2FBF4F325F03F05A0FB02122D047C
:10BE5000900C2D0C0543BD805C4C39884FF49672D4
:10BE600002FB00F284FB02409BB2D217002BC2EB14
:10BE7000A01221F0010108BF01230904013243F49B
:10BE80000043090C92B239803A84BB833B889BB251
:10BE900043F001033B803B8823F4816323F00203DA
:10BEA0001B041B0C43F480634FF480423B803A81B7
:10BEB0003B8823F080031B041B0C3B809BF8103055
:10BEC0008DF808300024012302A88DF80B308DF87E
:10BED00009408DF80A401AF075FC9BF80F308DF878
:10BEE000083002A88DF809408DF80A401AF090FC3D
:10BEF00007B0BDE8F08F7047B9F1000F48D01622A7
:10BF000089F8073089F806209BF80E0032F03CF8DB
:10BF1000BB8823F440731B041B0C2846BB80FDF731
:10BF200071FE4846FDF76EFE1EE79BF80E0032F0EC
:10BF30002BF8BB8823F440731B041B0CBB802846E2
:10BF4000FDF760FE4846FDF75DFE11212846FDF72E
:10BF500053FB0DE71E4A136A43F4000313624FF4C8
:10BF600000001AF01BFB50E7194A136A43F4001350
:10BF700013624FF400101AF011FB46E7144A136ADB
:10BF800043F4800313624FF480001AF007FB3CE790
:10BF90009BF80E0031F0F8FFBB8823F440731B04BC
:10BFA0001B0C4846BB80FDF72DFE4846FDF72AFED8
:10BFB000DEE600BF0054004000580040005C004036
:10BFC000009F2400804F120083DE1B43D34D62107C
:10BFD00000380240604D0020F8B54FEAC00E274FF0
:10BFE000069C0EEB000507EB85056E68002E42D01F
:10BFF0004900C9B2A9754FF0000C0121EA7585F816
:10C0000019C0A9762B76697585F814C0B3882C629F
:10C010009905EC6114D43388DA050CD44FF48054BC
:10C0200001E0013C1ED033889B05FAD433889BB2D3
:10C0300043F480733380B3889BB243F44073B3807E
:10C040000EEB000107EB81024FF4805401E0013C4C
:10C0500008D0537D002BFAD107EB81073C7D84F09B
:10C060000100F8BD064A138801339BB21380FFF725
:10C0700031FE2046F8BD3046F8BD00BF604D0020BF
:10C080002C35002070B590F904506C1C82B00AD099
:10C09000032D08DC16460A46417900962846FFF72C
:10C0A0009BFF02B070BD002002B070BD70B5037878
:10C0B000012B82B004D106236A46F721FFF7E2FF85
:10C0C0009DF801209DF804309DF800609DF8035014
:10C0D0009DF802409DF80500074912011B0142EA44
:10C0E000063243EA053342EA141243EA1013CA60E7
:10C0F0008B6002B070BD00BF7425002000B583B016
:10C10000002000920A466821FFF766FF03B05DF841
:10C1100004FB00BFF0B5C60033189B00254DEA585C
:10C120005468A28A83B092B20192019A2B4412F40D
:10C13000706F1CBF01221A75019B13F4E06F074654
:10C140000CD1A38A3E4423F4706305EB86051B04DF
:10C150001B0C0022A3826A7503B0F0BD238BA38859
:10C1600023F480631B041B0CA380019B9B05E8D474
:10C1700023889805E5D42388D9050ED52388DA05C8
:10C18000FCD423889BB243F40073238023889B054F
:10C19000FCD43846FFF79EFDD3E723889BB243F4D7
:10C1A00000732380A38823F440731B041B0CA3801B
:10C1B000C7E700BF604D0020F0B583B0441C8DF888
:10C1C000073001D0032802DD002003B0F0BDC70016
:10C1D000244E3B1806EB83035D68002DF4D0490024
:10C1E000C9B2997501240021DA755C7699761C76BE
:10C1F0005C751975A9880DF107028905DA611A6263
:10C2000014D42B88DA050CD44FF4805401E0013C9F
:10C210001ED02B889B05FAD42B889BB243F48073E5
:10C220002B80AB889BB243F44073AB80074406EB92
:10C2300087024FF4805401E0013C09D0537D002B6C
:10C24000FAD106EB87073C7D84F0010003B0F0BD16
:10C25000054A138801339BB21380FFF73BFD20464C
:10C26000B3E700BF604D00202C3500200378012B80
:10C2700000D07047417990F904003123F4229BE704
:10C28000134600200A46682196E700BF0220FCF70B
:10C2900041BD00BF02203DE70120FCF73BBD00BFD0
:10C2A000012037E70020FCF735BD00BF002031E753
:10C2B0001549164B16484A6810B4CC681549B2FBAC
:10C2C000F4F203FB02F30360D1F88820124B134C05
:10C2D00042F47002C1F888201A68002042F001027E
:10C2E0001A6098601A6822F0847222F480321A6010
:10C2F0005C601A684FF0006422F480221A60D860F3
:10C300008C605DF8044B70470000002040420F0035
:10C310000C7D002000ED00E00038024010300024C9
:10C32000044B4FF4F07002210A225860D9609A60E1
:10C33000FFF7BEBF0000002038B50B4C23688BB15F
:10C340005A68821A002A054604DA0CE05A68AA1ACA
:10C35000002A07DB9A68226018461A68904723680B
:10C36000002BF3D138BD38BD243000200B4B002208
:10C3700010B4027203F1D804012102E0072A09DC9B
:10C380009979890702D51979815401329C4203F1C8
:10C390001803F3D15DF8044B704700BF4047040811
:10C3A00013230370704700BF012310B431213024E0
:10C3B000322244704171C2700370037183705DF862
:10C3C000044B70472DE9F0410B78047BDB43DEB270
:10C3D00000F1100200F1380342F8044F9342FBD100
:10C3E000DFF89CC000F16001002243F8042F8B426B
:10C3F000FBD14FF0140E0521002546FA01F303F09E
:10C400000103002B1D4414BF4FF019084FF00A0818
:10C4100011F0010FEDB214BF2746002700220EEBEA
:10C4200002039BB200EB8303013242455F61F6D108
:10C43000013A92B2013201390EEB02034A1C9BB25F
:10C4400001D09E46D9E715F0010F14BF19250A2522
:10C4500000215A1892B200EB82020131A9425461C4
:10C46000F7D10B449BB21A1D00EB8202013300216D
:10C470009BB25160ACF800300361BDE8F08100BFB1
:10C4800088250020254B5B880B332DE9F04F8A4629
:10C4900001F1060B1FFA83F94FF001080021002774
:10C4A0001AF801EB3E464C460122A4F10B039BB265
:10C4B00007E001339BB2B0F80CC0C5F814C09C4231
:10C4C0000AD000EB8305002AF3D100EB830501338A
:10C4D0009BB29C426A61F4D1231D00EB83030136B9
:10C4E000092FF6B259600CD0092E14D008FA07F3C0
:10C4F00013EA0E0F14BF012200220C34A4B201373C
:10C50000D3E709F17809DA451FFA89F9C7D1034B56
:10C510005980BDE8F08F0022EFE700BF882500209A
:10C520002DE9F047DFF85C80B8F8043004338A4620
:10C530001FFA83FC01F109094FF0010E1AF8017B83
:10C5400064460026231F0EFA06F29BB23A40BAB1A7
:10C55000818900EB830501339BB29C426961F6D16E
:10C5600001360434082EA4B2ECD10CF1200CCA45DB
:10C570001FFA8CFCE2D10023A8F80430BDE8F08754
:10C580001146E6E78825002008B529F095F9FEF761
:10C59000B5FF00BF024A034B1278197827F074BC2C
:10C5A0007028002071280020038A2DE9F047858932
:10C5B000ADB21D4029D00F4606464FF000484FF05F
:10C5C0000009B5FA85F328FA03F2D24391B21B3B76
:10C5D00015403182042B16D8DFE803F031292119E8
:10C5E00003007B6A002B32D003F1FF3A1FFA8AFA6C
:10C5F000C7F824903C6A34B12368204651469847D6
:10C600006468002CF8D1002DDBD1BDE8F0873868D4
:10C61000716B036889B29847002DD2D1F5E778682D
:10C62000B16B036889B29847002DCAD1EDE7B868AD
:10C63000F16B036889B29847002DC2D1E5E7F8682D
:10C64000316C036889B29847002DBAD1DDE7F36AEF
:10C650001FFA83FACEE700BF2DE9F04F2DED028BD4
:10C66000A0F10A0389B00C46E72B00F21A87DFE835
:10C6700013F01C01180718071807180718071807E0
:10C6800018071807180718071807180718071807B2
:10C6900018071807180718071807180718071807A2
:10C6A00018078805180718071807780518071807C6
:10C6B0001807710518070E051807F5041807EA048E
:10C6C0001807E2041807BD041807A904180718077B
:10C6D0001807A3049C0418078F0418071807DD0126
:10C6E0001807B501180718071807A2011807180737
:10C6F0001807180783011807FC001807DE05410614
:10C7000018071807180718071807180718077503D8
:10C71000180747031807130318075B0218071502C9
:10C720001807180718071807F002AF02E902E4011A
:10C73000E800B6032C061406830418074C043004E2
:10C7400018071807180718072504180718070404FE
:10C75000180718071807F50392067D06D50618076F
:10C760001807180704066506180764011807180754
:10C7700018071807180718071807180718071807C1
:10C7800018071807180718071807F00218071807DE
:10C7900018071807180718071807180718071807A1
:10C7A0001807180718072D01180718071807180782
:10C7B0001807180718071807180718071807180781
:10C7C0001807180718071807180718071807180771
:10C7D0001807180718071807180718071807180761
:10C7E0001807180718071807180718071807180751
:10C7F0001807180718071807180718071807180741
:10C800001807180718071807180718071807180730
:10C810001807180718071807180718071807180720
:10C820001807180718071807180718071807180710
:10C830001807180718071807180718071807D20548
:10C84000A705A04E337853B19F4F002537F8021F3C
:10C850002046FEF78DF833780135AB42F6DC012037
:10C8600009B0BDEC028BBDE8F08F964E3378002BFB
:10C87000F5D0964F0025B846236817F81520591CA7
:10C8800021601A7098F8011001EB810101EB810120
:10C8900001F2EE2189B22046FEF76AF833780135BD
:10C8A000AB4208F10208E7DCD9E7894D284632F0AF
:10C8B00091FB0028D3DD2B460544226813F8011BA9
:10C8C000501C9D4220601170F7D1C8E70B68DFF85B
:10C8D00050C2591C9CF8002021601A709CF800304E
:10C8E000002BBCD07B4E7C4D7C487D4900232268C8
:10C8F00016F8017F02F1010EC4F800E017702268FB
:10C9000015F8017F02F1010EC4F800E017702268EB
:10C9100010F8017F02F1010EC4F800E017702268E0
:10C9200011F8017F02F1010EC4F800E017709CF8C5
:10C93000002001339A42DADC91E70B68694F591CF9
:10C940003A7821601A703B78002B88D00025EEB22F
:10C9500030461BF075F823684278591C2160304638
:10C960001A701BF06DF801892046FEF701F83B783C
:10C970000135AB42EBDC72E70B685B4D591C2A7941
:10C9800021601A7023686A79591C21601A702988FD
:10C990002046FDF7EDFF2368AA79591C21601A7023
:10C9A00069882046FDF7E4FF2368EA79591C216075
:10C9B00001201A7054E70B6800255A1C0A602046B3
:10C9C0001D702946FDF7BCFF29462046FDF7B8FF3C
:10C9D00020462946FDF7B4FF012041E70B68434A92
:10C9E000434D1178434A581C206019701168204645
:10C9F000FDF7A6FF2368404A591C127A21601A707D
:10CA000029882046FDF7B4FFA9882046FDF7B0FF2E
:10CA100029892046FDF7ACFF00212046FDF7A8FF3D
:10CA200020460021FDF7A4FF012019E7084608224F
:10CA30003149FDF755FF012012E7304D304E9FED93
:10CA4000318ADFF8E080DFED308A05F120070EE063
:10CA5000FCEEE77ACDED017ABDF8041020460435EE
:10CA6000FDF786FFBD4206F118063FF4F8AE717C73
:10CA70000029F3D0254BD5ED007A1B78012BE7D1A7
:10CA8000234B1B68DB0440F1CC85F5EE407AF1EED8
:10CA900010FA40F0008640F2DC51DFE70B681D4AD7
:10CAA0001D49D0781D4A5D1C25601870236849799E
:10CAB000581C206019702368D278591C216001200D
:10CAC0001A70CDE638A500203AA40020F4340020E6
:10CAD00020390020AB510020BB510020DB51002049
:10CAE000CB510020D93A0020E4AD0020F8680020A6
:10CAF000D84D0020ECB000207C5D0020F8660020BE
:10CB0000045800200000404200E08244E858002021
:10CB1000185C0020D068002050C10020E068002090
:10CB2000A9510020DB9B914100212046FDF720FF09
:10CB300000212046FDF71CFF00212046FDF718FFCD
:10CB40002368B94D00265A1C22601E7023682A688B
:10CB5000591C92F82C2021601A7023682A68591CED
:10CB600092F8362021601A7023682A68591C92F8BE
:10CB7000372021601A7023685A1C22601E702368B7
:10CB80005A1C22601E7023685A1C22601E702B687B
:10CB90002046598FFDF7ECFE2B682046198FFDF7D4
:10CBA000E7FE23682A68591C92F82E2021601A702B
:10CBB00023685A1C22601E702B682046598EFDF790
:10CBC000D7FE2B682046998EFDF7D2FE012047E65E
:10CBD000964B9B8AB3F5006F00F22C85B3F5806FFE
:10CBE00000F25685B3F5007F34BF01270227904D30
:10CBF00005F10C0655F8041B91FBF7F1204689B2AC
:10CC0000FDF7B6FEAE42F5D18A4D8B4F05F10C060D
:10CC1000B5EC010AD7ED087A80EE270A33F068FBFD
:10CC200081B22046FDF7A4FEAE42F1D1834D05F15D
:10CC30000C0655F8041B204689B2FDF799FEB54253
:10CC4000F7D10CE6084610227D49FDF749FE012088
:10CC500006E600258146DFF8FC81DFF8FCB105958A
:10CC600004950695079501214FF6FF7A05E00135F9
:10CC70000B2D00F0368418F9011F4F1C4AFA05F3FA
:10CC8000F5D0DE07F3D5BBF800302B41D807EED541
:10CC900006A8FEF7B3F9EAE76A4E0B687279624DAF
:10CCA000591C21601A702B682046198CFDF760FE14
:10CCB0002B682046D98BFDF75BFE71892046FDF776
:10CCC00057FEB1892046FDF753FE2B682046598C4C
:10CCD000FDF74EFE2B682046998CFDF749FEF18941
:10CCE0002046FDF745FE318A2046FDF741FE2A68C1
:10CCF000236892F82620591C216001201A70AFE5A4
:10CD0000504EF378002B00F098840B680822591CD1
:10CD100021601A7023680122991821601A70236813
:10CD2000494D591C2A7921601A702368AA78591C28
:10CD300021601A7029882046FDF71AFEE9892046ED
:10CD4000FDF716FE2368F279591C21601A702368DA
:10CD5000EA78591C216001201A7081E527F078F8E3
:10CD6000FF28064600F07D8408A9002501F8125D21
:10CD70000DF10D008DF80D5027F04AF808A800F8C5
:10CD8000115D27F039F808A800F8105D27F028F8A1
:10CD900008A820F8085D27F017F823685A1C2260BD
:10CDA0001E7023689DF80D20591C21601A7023689D
:10CDB0009DF80E20591C21601A7023689DF80F20E1
:10CDC000591C21601A7023689DF81020591C21609D
:10CDD0001A702046BDF81810FDF7CAFD3FE51B4B41
:10CDE0000A681B781A4D511C03F00203216013706E
:10CDF00023682A7D591C21601A7029682046FDF796
:10CE00009FFD69682046FDF79BFD29892046FDF7B7
:10CE1000AFFDE9892046FDF7ABFD2046298AFDF7E5
:10CE2000A7FD01201CE500BF38390020A03D0020EF
:10CE3000D83D00200C5C00203CC400202CAF00201A
:10CE4000E8660020F45B0020C4580020183E002053
:10CE50001C3E002030270408E8380020AE4D08466C
:10CE60002988FDF785FD69882046FDF781FD20466C
:10CE7000A988FDF77DFD0120F2E4A84D05F16006CB
:10CE8000A9882046FDF774FDE9882046FDF770FD6E
:10CE900029892046FDF76CFD2368AA7A591C216078
:10CEA0001A702368EA7A591C21601A7055F80C1B15
:10CEB0002046FDF745FDAE42E2D1D0E49849522329
:10CEC0002268501C2060137011F8013F002BF7D12D
:10CED000C5E4944800232268056803EB4301561C0F
:10CEE0006D5C26601570026825680A446E1C5278D5
:10CEF00026602A70026825680A4401339278691C0A
:10CF00000A2B21602A70E6D1A9E4874D0B682A68B4
:10CF1000591C127821601A702B6822689978531C6A
:10CF20002360002311702A6821681A440133527962
:10CF3000481C032B20600A70F5D123682A68591C0D
:10CF4000127A21601A7023682A68591CD2782160ED
:10CF50001A7023682A68591C127921601A702B688C
:10CF600020465989FDF704FD2A682368527A591C26
:10CF700021601A702A6811E06C4B08461968FDF7A9
:10CF8000DFFC6B4B20461988FDF7F2FC012067E4BB
:10CF90000B68684A581C9178206019702368527891
:10CFA000591C216001201A705AE40B68012299185B
:10CFB000216010461A7053E408460021FDF7C0FCBA
:10CFC00001204DE45C4D5D4E05F1200795F90210FE
:10CFD0005B4B93F906208A4203F1080300F0648258
:10CFE0009E42F6D10835BD42F0D138E4554B03F1ED
:10CFF0005A0522685979501C2060117022681978EE
:10D00000501C2060117022685978501C20601170EB
:10D0100022689978501C206011702268D978501CC1
:10D0200020601170226819790633501C9D422060DF
:10D030001170DED113E40B68434A591C527D216004
:10D0400001201A700CE4414D05F1800655F8041FCB
:10D050002046FDF775FCAE42F8D100E43C4D05F1E9
:10D060004006B5F880102046FDF782FC236895F84D
:10D070008220591C21601A70236895F8832004359A
:10D08000591CB54221601A70EBD1FFF7E8BB2E4D59
:10D090000B682A7A591C21601A70A98B2046FDF76B
:10D0A00067FC298B2046FDF763FC698B2046FDF762
:10D0B0005FFC2368EA7C591C21601A70A98C204609
:10D0C000FDF756FCE98C2046FDF752FC2368AA7F49
:10D0D000591C21601A70236895F82020591C216082
:10D0E0001A70698C2046FDF743FC2368EA7A591CC4
:10D0F00021601A70E9682046FDF722FC23682A7C2B
:10D10000591C21601A70236895F82120591C216050
:10D1100001201A70FFF7A4BBC8AD00205CAE002050
:10D120000027040838390020E0CD0020F43D00201D
:10D13000E83D0020EC680020187C0020785D00208D
:10D14000585D0020543600207C5D0020B837002058
:10D15000BC3700200B689C4A581C1178206019705D
:10D160001CE79A4D08462988FDF702FCA98820464D
:10D17000FDF7FEFB20462989FDF7FAFB0120FFF7AA
:10D180006FBB934D05F15006287830F0E3FE23681D
:10D19000027A591C21601A7023686A78591C216030
:10D1A0001A702368AA78591C21601A702368EA78DB
:10D1B0000435591CAE4221601A70E5D1FFF74FBB10
:10D1C000844B03F1700522681978501C206011709F
:10D1D00022685978501C2060117022689978501C80
:10D1E000206011702268D978501C2060117022686C
:10D1F0001979501C2060117022685979501C2060E8
:10D200001170226899790733501C9D42206011707B
:10D21000D9D1FFF724BB704D0846E989FDF7A8FB7B
:10D220002046A989FDF7A4FB0120FFF719BB0B6875
:10D230006A4D01269A190A601E701CF063F90028D5
:10D2400040F00882664B2268511C216010702268F1
:10D2500041F2B410511C185C216041F27811107039
:10D2600059582046890AFDF76BFBA96A20464908F0
:10D27000FDF766FB0120FFF7F3BA5A4D0846298AED
:10D28000FDF776FB698A2046FDF772FB2046A98AE6
:10D29000FDF76EFB0120FFF7E3BA534D08462988DE
:10D2A000FDF766FB69882046FDF762FBB5F904309F
:10D2B0004E4AD91782FB0323C1EBA301204689B252
:10D2C000FDF756FB0120FFF7CBBA494B08461988FA
:10D2D000FDF74EFB474B20461988FDF749FB464BAF
:10D2E00022681B78511C03F0010321600120137098
:10D2F000FFF7B6BA0B68414E01255A1C0A601D7033
:10D300000B68B278591921601A7021F059FE236810
:10D310003B4A3C495F1927601870B1F90010B2F917
:10D320000000FDF7AFFC23685A192260187031889D
:10D330002046FDF71DFB2846FFF792BA0A68324BDC
:10D34000501C19782060117022685978501C206098
:10D35000117022689978501C206011702268DB7867
:10D36000511C216001201370FFF77ABA0B68274A1D
:10D3700019491078264A5D1C256018702368897841
:10D38000581C2060197023689278591C2160012074
:10D390001A70FFF765BA0A681E4B1F491878551CAA
:10D3A0002560107022685878551C2560107022681E
:10D3B0009B78501C206013702046C988FDF7D8FA6E
:10D3C0000120FFF74DBA00BFF8680020D84D0020BB
:10D3D000FC68002054A70020D068002090A2002004
:10D3E000E08D0020C4580020F83D00206766666686
:10D3F00080BF00201E3900207C5000205CBF002030
:10D400004A6700204C67002090510020F45B002008
:10D41000E0680020C8680020C8AD0020DFF840E3C5
:10D420000027FEB2714600232268501C206016704F
:10D430002268501C20601370226811F8010F01331C
:10D44000551C062B25601070EED10137062F0EF10A
:10D45000060EE6D1B64900232268501C20601770E2
:10D460002268501C20601370226811F8010F0133EC
:10D47000551C0B2B25601070EED12368AD4A581C4B
:10D4800007212060197023680021581C2060197042
:10D49000236892F8F020591C216001201A70FFF7D0
:10D4A000DFB90020FFF7DCB923685A1C226019702D
:10D4B00029882046FDF75CFA2368EA78591C216028
:10D4C0001A7023682A79591C21601A702368AA7976
:10D4D000591C21601A7023686A79591C21601A70DE
:10D4E00080E5DFF880A200254FF008080135C5F17E
:10D4F000200208FA02F2A5F120032AFA05F61643E3
:10D5000028FA03F31E43252D06F001024FF0000315
:10D510000BD01343EAD0E8B231F072F90028E5D01D
:10D52000294606A8FDF76AFDE0E7834B1B78DA077A
:10D5300000F19E800025814E2F4602E00135252D09
:10D540000DD029463046FDF769FD0028F6D0294662
:10D5500006A8FDF763FD00285ED10137EEE7784BA2
:10D56000784DB3F850102046FDF702FA764B198833
:10D57000204689B2FDF7FCF9744B19684B0103F0A2
:10D580002002C1F340031343C1F3800243EA420384
:10D59000C1F3C00243EA8203C1F3401243EAC2036B
:10D5A00001F0100119432046FDF7E2F904A9042215
:10D5B0002046FDF795F923682978654A581C2060B4
:10D5C000197011886429A8BF64212046FDF7D0F99D
:10D5D000B9F1960F51D000212046FDF7C9F9216815
:10D5E000B7F1190348BFA7F11203A3F3C4034A1C00
:10D5F000226020461A460B7005A9FDF771F92368D1
:10D60000544A581C10212060197020461188FDF7DB
:10D6100097F90120FFF724B9394604A8FDF7EEFC7D
:10D620009BE7F4EEC87AF1EE10FA59DA4FF47A710A
:10D63000FFF714BA0827FFF7DABA0B68B178464A41
:10D64000581C2060197023681278591C21601A70C8
:10D65000FFF765BB95F82420404B002A38D13046AF
:10D66000F1E523685A1C226001201E70FFF7F8B80C
:10D67000069B43F0010306935CE723680322591CD1
:10D6800021601A7023686A78591C21601A70A6E715
:10D690000427FFF7ACBAF4EEC87AF1EE10FA3FF5C2
:10D6A000FAA9F4EEE87AFDEEE77AF1EE10FA17EE59
:10D6B000901A2DD86FF4F973303903FB01F140F261
:10D6C000E73391FBF3F101F2DB5189B2FFF7C6B901
:10D6D0005978022917D003290CBF04203046B2E53F
:10D6E000FDEEE77A40F2E73217EE903A303B02FB6C
:10D6F00003F388FB0312D917C1EB622101F2E93170
:10D7000089B2FFF7ABB9042A34BF022003209AE59F
:10D7100040F2F313A1F5836103FB01F140F2E7331B
:10D7200091FBF3F101F2DD5189B2FFF797B900BF28
:10D730009F380020BC370020593A0020F8C3002051
:10D74000080A0020FC7B00202C350020143E00201D
:10D7500030350020A0BF0020C4680020E08D0020EC
:10D760007B38002090E33FF41B4C08B501210220D8
:10D77000FCF7CCFA237803F00502052A27D003F042
:10D780000903092B08D000210120FCF7BFFA002172
:10D790000846FCF7BBFAFEE7104CA168E2680B688C
:10D7A000206923F001030B60138823F001031B049D
:10D7B0001B0C138018B1292200238271C37103222C
:10D7C0004A21FCF795F82069FCF716FADBE728F008
:10D7D00005F92378D3E700BF344D002088250020C9
:10D7E000022828BF022010B4084C094B207000EB1F
:10D7F0008002C0EBC20207495DF8044B013003EB25
:10D800004203C0B20B602DF079BB00BFFC7B00204F
:10D81000BEAF00203839002008B514F053F8FCF7EB
:10D8200043FEBDE8084014F035B800BF38B5484B9A
:10D830005A899989914224BF00225A81198ADA892A
:10D84000914224BF0022DA81DA78CAB1072A41491D
:10D850006AD091F85700404D012400210A282C700D
:10D860009C70D9715DD00C2807D0002A6CD0DFEDF8
:10D870003B7A072A0ED00A2862D0DFED397A09E018
:10D88000344A92F857000A2856D00C285BD1D9792F
:10D89000DFED347A344C9FED350AA278002918BFA9
:10D8A000F0EE407A062A04D8314901EB820191ED6D
:10D8B0000F0A217979B1013A032A0BD8F7EE007AE1
:10D8C00087EE800A32F014FD2388984228BF18465C
:10D8D000208038BD38BD9B781F4A07EE103A11787A
:10D8E000B8EEC77A67EE277A07EE101AB8EEC77A55
:10D8F00027EE277AB4EEC70AF1EE10FAEADD80EEE1
:10D90000277AFDEEC77A17EE903A102BA8BF1023A6
:10D91000012BB8BF0123DBB28B4238BF0B4613701B
:10D9200038BDDFED147AA4E791F857000A2803D038
:10D930000C28ACD0D9799AE7D979DFED0E7AA9E72E
:10D94000DFED0D7AA6E7D979DFED047AA2E700BF13
:10D95000F45B00203CC40020C46800206F1203392F
:10D960006F12833A0AD7A339C45800206F120338C4
:10D97000002704085304E9380F506E3A38B50C4CB0
:10D980000C4DAC4206D2616820461434FCF718FDF9
:10D99000AC42F8D3084A094B094C146000220949EB
:10D9A0001A705A7008480860BDE838401FF072B914
:10D9B000900100086806000838390020FC7B002030
:10D9C000BEAF0020E0CD002002A5002008B5FFF783
:10D9D000D5FF13F077FFFCF767FDBDE8084013F0B3
:10D9E00059BF00BFF0B50C2934D8DFE801F0893306
:10D9F00033335E333333343333330700048C968947
:10DA0000B2F802E01788734D24F480542404240CE7
:10DA10000484038C8488818B23F4005321F4E64131
:10DA20001B0409041B0C46EA0E06090C43EA0633E4
:10DA300041EA0721A8429BB2A4B289B200F09E80BD
:10DA400005F58065A84200F0998092688480818302
:10DA500002640384F0BD048C9589B2F802C0B2F868
:10DA600000E05C4F24F480742404240C0484038CB0
:10DA70008688818B23F400731B0421F073011B0C37
:10DA800045EA0C04090443EA0423090CB8429BB29A
:10DA9000B6B241EA0E015CD04F4CA04259D0926818
:10DAA00086808183C2630384F0BD048C9589B2F8BB
:10DAB00002C0B2F800E0474E24F010042404240C05
:10DAC0000484038C8788018B23F0200321F4E64132
:10DAD0001B0409041B0C45EA0C04090C43EA04135B
:10DAE00041EA0E21B0429BB2BFB289B25DD03A4C3E
:10DAF000A0425AD092688780018382630384F0BD7C
:10DB0000048C9789B2F802E01688324D24F00104A3
:10DB10002404240C0484038C8488018B23F00203E6
:10DB20001B0421F073011B0C47EA0E0709043B4359
:10DB3000090CA8429BB2A4B241EA060125D005F522
:10DB40008065A84221D09268848001834263038467
:10DB5000F0BDD589148A578A23F4006343EA05256A
:10DB60004FF6FF332B40958826F440563C4343EA5A
:10DB7000052346EA04169BB2B6B290E7158A24F450
:10DB8000804444EA8514A4B25FE7D689158A578A8F
:10DB900023F00803334324F4407496883D4323F074
:10DBA00004032C433343A4B2CDE7D489158A568AA3
:10DBB00023F0800343EA04134FF6BF741C4093889C
:10DBC00027F44067354344EA031347EA85079BB2CD
:10DBD000BFB28FE700000140000401402DE9F04F83
:10DBE0004FF48C72002183B08A488B4CDFF84C9242
:10DBF0008A4D8B4E8B4FDFF8488234F086FC8A4882
:10DC00008A49DFF840E2DFF840C20022135983421C
:10DC100000F0D580B3F1804F00F0E580AB4200F01A
:10DC2000E480B34200F0E380BB4200F0E280734541
:10DC300000F0E180634500F0E080434500F0DF80C4
:10DC4000DFF808A2534500F0DC800AF5806A5345EE
:10DC500000F0D9800AF5806A534500F0D680AAF515
:10DC6000983A534500F0D3800AF5806A534500F096
:10DC700084800AF5806A534508BF0D237ED0183290
:10DC8000F02AC3D1644C6A4E6A4F6B4D04F1F00820
:10DC900002E01834A0456DD0A379002BF9D0237988
:10DCA0004FEA131909F1FF39B9F1030F03F00F031C
:10DCB000EFD836F8190040FA03F2D207E9D54FF051
:10DCC000010A0AFA03F3013B184031F09DFE17F8F0
:10DCD0000930184415EBC002DBD055F83000DFF8EE
:10DCE00070E1217A00F13F4303F57E039B0A1EF8A1
:10DCF000033003F01F0E5B09032B0AFA0EFA60D003
:10DD0000042B67D0022B07D1DFF820E1DEF8443086
:10DD10004AEA0303CEF8443093880093B3FA83F3BE
:10DD2000C3F11F039BB2DA0800EB820203F0070382
:10DD3000D2F820E09B004FF00F0C0CFA03FC2EEA07
:10DD40000C0EC2F820E0D2F820E001FA03F343EA17
:10DD50000E03136269460023022218348DF8042052
:10DD60008DF805308DF806308DF8073018F0ECFA94
:10DD7000A04591D103B0BDE8F08F0C2309EBC3039C
:10DD80004FF0010A93F85C3003F01F0B5B09032B83
:10DD90000AFA0BFA09D0042B0CD0022B7FF46FAFD8
:10DDA0004B6C4AEA03034B6469E70B6C4AEA0303D2
:10DDB0000B6464E70B6B4AEA03030B635FE7002322
:10DDC000DCE7DFF868E0DEF840304AEA0303CEF82B
:10DDD0004030A1E7DFF854E0DEF830304AEA0303D0
:10DDE000CEF8303098E70123C8E70223C6E70323C3
:10DDF000C4E70423C2E70523C0E70623BEE70723E1
:10DE0000BCE70823BAE70923B8E70A23B6E70B23E0
:10DE1000B4E700BFD82C00204047040800040040AD
:10DE200000080040000C00400000014000380240A3
:10DE3000085A0408045A040824CC002000270408C7
:10DE40000004014000100040001400400040014068
:10DE50005C48040801490248FEF7A6BBC82D002013
:10DE60000040014001490248FEF79EBBA02D002062
:10DE70000004014001490248FEF796BBA02D002096
:10DE80000004014001490248FEF78EBB782D0020B6
:10DE9000000C004001490248FEF786BB502D0020CF
:10DEA0000008004001490248FEF77EBB282D0020F3
:10DEB0000004004002494FF08040FEF775BB00BFF0
:10DEC000002D002001490248FEF76EBBD82C00202F
:10DED0000000014001490248FEF766BBD82C002033
:10DEE00000000140F0B504684D4DA30AAB427AD062
:10DEF00009D94C4DAB426ED00F35AB425AD0103DD4
:10DF0000AB4274D0F0BD023DAB4268D056D8B3F5F9
:10DF1000801F70D14FF0480E01264779B0004FEABC
:10DF2000970C002968D063460227A5899F40831972
:10DF30000CEB43032F4303F1040C3B4DBFB245F8F8
:10DF4000231045F82C20A781EFF31181502282F392
:10DF50001288821905EBC2021369002B32D01362BA
:10DF60000433821905EBC202576917B11F60536968
:10DF70000433821905EBC202976917B11F609369D8
:10DF80000433821905EBC202D76917B11F60D36948
:10DF900004330027CAB21F6082F31188304405EBB6
:10DFA000C000036A8BB9A38923F001031B041B0C77
:10DFB000A381F0BD4FF4887E0626AEE74FF0980EA1
:10DFC0000326AAE705EB0E03CBE7A3899BB243F038
:10DFD0000103A381F0BD4FF0E80E05269DE74FF049
:10DFE000700E022699E74FF0C00E042695E74FF019
:10DFF000200E002691E7F0BD0223BF0803FA07F7C1
:10E00000A389094D9BB223EA070387190CEB470C40
:10E01000A3810CF1040345F82C1045F8232093E765
:10E020000300100041001000D82C002010B5036838
:10E0300083480139834282B089B200F0CB80A0F5D9
:10E040008060834200F0C68000F58040834200F08B
:10E05000B88000F58060834200F0B38000F58060F6
:10E06000834200F0AE80774C188824686408B4FBC3
:10E07000F2F4013CA4B282B2B3F1804F0AD07248EC
:10E08000834207D000F58060834203D000F58060B2
:10E09000834202D122F0700292B26C48834200F0B7
:10E0A000A28000F58060834200F0A78022F44072D5
:10E0B00000F56C4092B283421A80D9621C854FD021
:10E0C0005F4A93424CD001229A821A8892B242F05F
:10E0D00001021A80B3F1804F00F099805A4A9342AE
:10E0E00000F0978002F58062934200F0948002F580
:10E0F0008062934200F0918002F58062934200F0CA
:10E100008E8002F58062934200F08B8002F57042AF
:10E11000934200F0888002F57052934200F08580AF
:10E1200002F58062934200F0828002F580629342A1
:10E130007FD0A2F5983293427DD002F5806293425F
:10E140007BD002F58062934208BF0D2215D002A851
:10E150004FF0012340F8043D18F034FB02B010BD2D
:10E160000122002119869A821A88394892B242F017
:10E17000010283421A80ADD10A46364B03EBC2033B
:10E1800001A893F85D408DF80440012300228DF82A
:10E1900005308DF807308DF8062018F013FB1B2C86
:10E1A00008D02E2CDAD12C4B019301A818F00AFBD1
:10E1B00002B010BD294B019301A818F003FB02B077
:10E1C00010BD204C18882468B4FBF2F4013CA4B2C2
:10E1D00082B251E71B4C18882468B4FBF2F4013C6E
:10E1E000A4B282B256E701201A80D9621C859882B7
:10E1F0001A8892B202431A8070E701201A80D9620D
:10E200001C8598821A8892B202431A8062E7012222
:10E21000B3E70222B1E70322AFE70422ADE705220C
:10E22000ABE70622A9E70722A7E70822A5E709220C
:10E23000A3E70A22A1E70B229FE70C229DE700BF7C
:10E24000000401400C7D002000040040001000404C
:10E2500000000140002704082C0100011901000101
:10E260002C4B98423DD0B0F1804F3CD0A3F57C437D
:10E2700098423AD003F58063984238D003F5806322
:10E28000984236D003F58063984234D003F580631A
:10E29000984232D003F57043984230D003F5705362
:10E2A00098422ED003F5806398422CD003F580630A
:10E2B00098422AD0A3F59833984228D003F580637A
:10E2C000984207D003F58063984208BF0D2202D020
:10E2D000002070470C22104B03EBC20393F85C0044
:10E2E00070470022F7E70122F5E70222F3E7032255
:10E2F000F1E70422EFE70522EDE70622EBE707222C
:10E30000E9E70822E7E70922E5E70A22E3E70B222B
:10E31000E1E700BF00000140002704082DE9804824
:10E32000013085B0C3B203938A4D8B4F8B4C8C4E1A
:10E330000A230293DFF82C9222F076F94FF4FA7A4E
:10E340004FF0100C4FF47A70D9F80430C3F308037F
:10E35000002B40F0C180EFF31183002B40F0BC8014
:10E360002968A26800BF2B689942F9D1D7F800E06C
:10E3700000FB0EF39B1AB3FBFEF300FB01314FF0E1
:10E38000010E0191D9F80430C3F30803002B40F0CB
:10E390008780EFF31183002B40F082802B68A16807
:10E3A00000BF2A689342F9D1D7F800B000FB0BF206
:10E3B000521AB2FBFBF200FB0323019A9B1AB3F53E
:10E3C0007A7FDFD3BAF1010ABED1039B002B40F064
:10E3D000BD804FF47A7ADFF88C9150464FF0100CE4
:10E3E000D9F80430C3F30803002B40F09280EFF318
:10E3F0001183002B40F08D802968A26800BF2B6834
:10E400009942F9D1D7F800E000FB0EF39B1AB3FB59
:10E41000FEF300FB01314FF0010E0191D9F80430F9
:10E42000C3F3080303BBEFF31183EBB92B68A168B7
:10E4300000BF2A689342F9D1D7F800B000FB0BF275
:10E44000521AB2FBFBF200FB0323019A9B1AB3F5AD
:10E450007A7FE3D3BAF1010AC2D1029B013B029356
:10E460007FF468AFFDF738F8EFF311888CF312886A
:10E47000A1682368DB0344BFC6F800E0A1682B68ED
:10E4800032685FFA88F888F31188D7F800801A4458
:10E4900000FB08F35B1AB3FBF8F300FB0233D4E78D
:10E4A000EFF311888CF31288A1682368DB0344BF63
:10E4B000C6F800E0A1682B6832685FFA88F888F334
:10E4C0001188D7F800801A4400FB08F35B1AB3FBED
:10E4D000F8F300FB023370E7EFF311828CF312883C
:10E4E000D4F808E02368D90303D501233360D4F8B6
:10E4F00008E02B683168D2B282F311883A68194477
:10E5000000FB02F3A3EB0E03B3FBF2F300FB0131BC
:10E5100035E7EFF311828CF31288D4F808E0236812
:10E52000D90303D501233360D4F808E02B683168A0
:10E53000D2B282F311883A68194400FB02F3A3EBCC
:10E540000E03B3FBF2F300FB013164E718462FF032
:10E5500087FE3EE704C4002008C4002010E000E06D
:10E5600000C4002000ED00E02DE9F047AB4FAC4EB9
:10E5700013F0A8F9BE421ED2DFF83083DFF83093E3
:10E580004446258862197DB14A450DD2052D0BD927
:10E5900033886188C3F30B03994200F0ED80144681
:10E5A00025886219002DEFD1716830461436FBF7CB
:10E5B00007FFBE42E4D39B4A1378A3F11701022957
:10E5C0000FD9994911F83300002840F01A81D8007A
:10E5D0000144497829B1954911F833300BB9182312
:10E5E0001370934C6378022B84BF002363702378ED
:10E5F000022B84BF002323708E4B9A78042A00F0EC
:10E60000F78032B91A88B2F5F07F84BF4FF4F07208
:10E610001A80894D894A2B681A40002A00F0FA8036
:10E62000D80700F1E080590400F1D8801A0700F102
:10E63000D0809B0400F1C680814D2B685A8C998C48
:10E64000914224BF00225A84FFF7F0F81FF0E6FB46
:10E65000002800F0B3804020FBF7E8FE4FF4007084
:10E66000FBF7E4FE4FF00070FBF7E0FE4FF0806038
:10E67000FBF7DCFE6378022B06D8724A724903EB83
:10E68000430302EB83030B602378022B07D803EBD1
:10E6900083016E4AC3EBC10302EB43032B6030F0EE
:10E6A00027F9002130226A4833F02FFF286826F02E
:10E6B000B5FD684B2D6803F1500102E00433994227
:10E6C0007AD01A78002AF9D19C78D8788442F5D289
:10E6D0006149624B0A7028461D6025F00DFB604BB6
:10E6E000604A1E7960496148614B1160C825642207
:10E6F00012FB06525F4C406B31F8061C5A60002238
:10E7000021809A60DA601A615A619A61DA6183F84D
:10E71000202083F8212008B112F032FF564B9FEDE4
:10E72000575A1B88564A9FED576A557E564C574993
:10E730005748086006EE903AF8EEE66A938AC5EE0E
:10E74000265A07EE103AD38A127EC4ED005A07EE1D
:10E75000903AB8EEC77A4F4BF8EEE77A1D725A72CC
:10E7600027EE067A67EE867ABDE8F04783ED017AF8
:10E77000C3ED007A13F08EB863799B077FF40FAF77
:10E78000716894F804A03046FBF71AFE3388BAEBA0
:10E79000133F04D01436BE42FFF4F2AE0BE7738889
:10E7A0007068AA1FC3F30B039A4204F10601A8BFC5
:10E7B0001A4631F093FBEDE7012289E736482BF04A
:10E7C00085FB48E73548FBF731FE4020FBF72EFE7E
:10E7D00032E73348FBF72AFE2B682AE73148FBF77C
:10E7E00025FE2B6822E73048FBF720FE2B681AE74E
:10E7F0009A8AB2F57A7FBFF40CAF4FF47A729A829C
:10E8000007E7D8000C186468002C7FF4E1AE1724E9
:10E810001470DDE643F008032B6001E7680600088A
:10E8200090010008F8680020644804084852040871
:10E83000FC7B0020C4580020ECB0002009600002DE
:10E840003839002002A50020E0CD0020BEAF002016
:10E85000202A0020FC6800209C230020542A00204D
:10E86000E4AD0020D0C30020D6680020A03D0020E9
:10E87000F0380020E43300205C2C0020C0C9FB48A5
:10E880008825002017B7D138602C00201CA6002056
:10E890003661023DF8A50020187C002009400002E6
:10E8A0000160000209200002086000020240000826
:10E8B0000080000808B513F005F8FBF7F5FD12F02D
:10E8C000E9FFFFF751FE0120BDE808402CF016BB20
:10E8D0002DE9F04F013085B0C3B203930B4602918E
:10E8E0008B4C8C4E002B00F099808B4D8B4FDFF8BA
:10E8F000309221F099FE4FF4FA7A4FF0100C4FF459
:10E900007A70D9F80430C3F30803002B40F0DE809E
:10E91000EFF31183002B40F0D9802968A26800BF73
:10E920002B689942F9D1D7F800E000FB0EF39B1A4F
:10E93000B3FBFEF300FB01314FF0010E0191D9F85A
:10E940000430C3F30803002B40F08780EFF31183FA
:10E95000002B40F082802B68A16800BF2A68934298
:10E96000F9D1D7F800B000FB0BF2521AB2FBFBF260
:10E9700000FB0323019A9B1AB3F57A7FDFD3BAF128
:10E98000010ABED1039B002B40F0BD804FF47A7A80
:10E99000DFF88C9150464FF0100CD9F80430C3F3D7
:10E9A0000803002B75D1EFF31183002B71D1296877
:10E9B000A26800BF2B689942F9D1D7F800E000FBAC
:10E9C0000EF39B1AB3FBFEF300FB01314FF0010E77
:10E9D0000191D9F80430C3F3080313BBEFF311839B
:10E9E000FBB92B68A16800BF2A689342F9D1D7F818
:10E9F00000B000FB0BF2521AB2FBFBF200FB032348
:10EA0000019A9B1AB3F57A7FE3D3BAF1010AC4D114
:10EA1000029B013B0293002B7FF467AF05B0BDE87A
:10EA2000F08FEFF311888CF31288A1682368DB0361
:10EA300044BFC6F800E0A1682B6832685FFA88F826
:10EA400088F31188D7F800801A4400FB08F35B1A9A
:10EA5000B3FBF8F300FB0233D2E7EFF311888CF33A
:10EA60001288A1682368DB0344BFC6F800E0A168F0
:10EA70002B6832685FFA88F888F31188D7F800802D
:10EA80001A4400FB08F35B1AB3FBF8F300FB0233F4
:10EA900070E7EFF311828CF31288D4F808E0236852
:10EAA000D90303D501233360D4F808E02B6831681B
:10EAB000D2B282F311883A68194400FB02F3A3EB47
:10EAC0000E03B3FBF2F300FB01317FE7EFF311829A
:10EAD0008CF31288D4F808E02368D90303D5012306
:10EAE0003360D4F808E02B683168D2B282F3118821
:10EAF0003A68194400FB02F3A3EB0E03B3FBF2F3F5
:10EB000000FB013118E718462FF0AAFB3EE700BFD3
:10EB100010E000E000C4002004C4002008C400206D
:10EB200000ED00E0204B5B68C3F3080330B4BBB9D1
:10EB3000EFF31183A3B91D4B1D4C1868A16800BFEA
:10EB40001A689042F9D11B4B1C684FF47A7202FB91
:10EB500004F3591AB1FBF4F130BC02FB001070470A
:10EB6000EFF31182102383F3128811498C680B682C
:10EB700013F4803F104B02D0012018608C680B49C1
:10EB8000D2B20D68186882F311880A4B19684FF4E5
:10EB90007A72284402FB01F31B1B30BCB3FBF1F378
:10EBA00002FB0030704700BF00ED00E004C400200D
:10EBB00010E000E008C4002000C400202DE9F84F58
:10EBC0008046FFF7AFFF254E2549DFF8A0E0254A34
:10EBD000254D844610274FF47A740120DEF8043066
:10EBE000C3F30803D3B9EFF31183BBB90B68D2F8B1
:10EBF00008A000BFD1F800904B45F7D1D6F800B07F
:10EC000004FB0BF9A9EB0A09B9FBFBF904FB03931D
:10EC1000A3EB0C034345E1D3BDE8F88FEFF3118A72
:10EC200087F31288D2F808B01368DB0344BF28606A
:10EC3000D2F808B00B68D5F800905FFA8AFA8AF328
:10EC40001188D6F800A0994404FB0AF3A3EB0B0348
:10EC5000B3FBFAF304FB0933DAE700BF08C4002072
:10EC600004C4002010E000E000C4002000ED00E03B
:10EC70002DE9F04FDFF830C1474A4849484E494D29
:10EC80008046102718F1FF38C0F08480DCF804308B
:10EC9000C3F30803002B5CD1EFF31183002B58D191
:10ECA0000B68946800BF08688342F9D1D6F80090D9
:10ECB0004FF47A7000FB09FEAEEB040EBEFBF9FECA
:10ECC00000FB03EEDCF80430C3F308034FF47A745E
:10ECD0000120FBB9EFF31183E3B90B68D2F808A068
:10ECE00000BFD1F800904B45F7D1D6F800B004FB37
:10ECF0000BF9A9EB0A09B9FBFBF904FB0393A3EB9E
:10ED00000E03B3F57A7FBDD2DCF80430C3F30803F9
:10ED1000002BDFD0EFF3118A87F31288D2F808B006
:10ED20001368DB0344BF2860D2F808B00B68D5F83D
:10ED300000905FFA8AFA8AF31188D6F800A0994405
:10ED400004FB0AF3A3EB0B03B3FBFAF304FB093355
:10ED5000D5E7EFF3118487F31288D2F8089013688F
:10ED6000D80303D501232B60D2F808900B682868DC
:10ED7000E4B284F31188D6F800A04FF47A7400EB63
:10ED8000030E04FB0AF3A3EB0903B3FBFAF304FB42
:10ED90000E3E97E7BDE8F08F10E000E004C40020CD
:10EDA00008C4002000C4002000ED00E030B4EFF300
:10EDB0001183102282F312880649074C0A6807481B
:10EDC000013200250A602560DBB2026883F31188F6
:10EDD00030BC704704C4002000C4002010E000E0F4
:10EDE0000F4B1B88014643B90E4B0F4A1B78106826
:10EDF0000BB981F00101FAF781BF0C4B5A691AB1C6
:10EE000018B91A68106058747047094A1868118850
:10EE1000084A92FBF1F2012102605974704700BF69
:10EE2000BCCD0020BECD0020C0CD0020C4CD002030
:10EE3000DCCD002020A1070038B5254B9C68236B52
:10EE400073B1636D626BCAB1998A1A88C90592B2AF
:10EE500001D5D20700D438BD4FF6F7721A8038BDFD
:10EE6000636D99891A88890692B2EBD59206E9D525
:10EE7000E26ACAB1988880B29047E2E799891A8815
:10EE80000D0692B2E0D51006DED5A26A616A8A420A
:10EE900019D0A1692569885C98800132B2FBF5F12F
:10EEA00005FB1122A262CFE79B88E2696169DBB2B0
:10EEB0008B54E269E068636D0132B2FBF0F100FB54
:10EEC0001122E261BEE7DA6822F08002DA60BBE775
:10EED000384D00202DE9F04F2DED028B95B0804686
:10EEE00029F050FA8E4B1D7825B115B0BDEC028B80
:10EEF000BDE8F08F8B4B1B685905F6D58A4BDFF8C0
:10EF000080B21B686BB1894ADBF800101368CB1A1A
:10EF10007C2B06D98648116003780133037019F001
:10EF200025F9844B1B78002B6DD0834C834AD4F891
:10EF30001031A8EB0303934201F2278394F8189150
:10EF4000B9F1000F32D17E4F3868FAF75BFAC0B2E0
:10EF500001280FD902287B4E42F013803378002B12
:10EF600042F00881D4F81C31A8EB0303B3F57A6FA3
:10EF700082F0CE82D4F82031002B44D094F818319E
:10EF8000BBB9714B1B689B7801211E3B00228B4251
:10EF900084F8181184F82C2142F26C82386802211E
:10EFA000043019F095F894F8243110E0D4F82031A9
:10EFB0004BB3D4F8283140F6B732A8EB03039342A1
:10EFC00021D994F82431002B01F0D9865C4F013B04
:10EFD000DBB284F82431002B01F00A84D4F82061DC
:10EFE00094F82C2116F8011B94F82D313868C4F8D8
:10EFF00020610A44013384F82C2184F82D31FAF77A
:10F0000005FAC4F82881514BDBF800601B7843B146
:10F010004F4F386828B14F4B1B78013B012B41F211
:10F02000F6834D4B1B786BB14C4F3B6853B1DBF80B
:10F030000030414C03931A46D4F84431D31A632B61
:10F0400001F29381464F3B78022B01F078863D4ECA
:10F0500096F87430032B01F0B683424B1B7873B1E2
:10F06000414D2B685BB1344CFFF75CFDD4F8503157
:10F07000039044F61F62C31A934200F231813B4B66
:10F080001B78002B7ED13A4B1B7843B12A4CD4F825
:10F09000A03203F5C333A033984581F03782354B56
:10F0A0001B78002B3FF421AF234E334C334D06F237
:10F0B000C1272068FAF7A6F900283FF416AF2068A8
:10F0C000FAF798F92B7880465A1E33B120682A70D7
:10F0D000FAF798F90028F2D107E703223946781E9B
:10F0E00033F0F9F996F8C03296F8C12286F8C38257
:10F0F00083F47F4383F0FF039B1A1FFA88F89BB2C7
:10F10000B8EB132FD5D196F8C222DBB29A42D0D1F8
:10F11000781E18F00FFD2B7818442870C9E700BF3F
:10F1200080530020185C0020803B0020F03D002030
:10F13000EC3D002032C00020AC2500203F0D030034
:10F14000983D0020200000209C3D002034C000207D
:10F15000883B00203CC0002044C00020903D00209F
:10F1600028C200204CC0002050C00020BCC000209D
:10F17000CDC0002056C000205CC0002060C0002030
:10F1800004C40020484C2278A2B1484B9B7A53B16A
:10F19000FFF7C8FC464B1B68C31AA3F57A73B3F597
:10F1A000FA6F07D82278434B43491868FAF7F6F804
:10F1B00000232370414CD4F8983203F5C333A033B5
:10F1C0009845FFF460AF3E4DC4F898822B78002B31
:10F1D00041F010873B4D2B78002B41F06B8694F863
:10F1E0009C2239498D5CEA0702F10780AF0701F1E3
:10F1F000C787680701F188872A0748D5334B344E03
:10F200000D9314AA1146A3F13D0241F8202D0020D0
:10F21000A3F140020D4603F8400C05910223112191
:10F220005170937028463168FBF764FB284671687B
:10F23000FBF760FBF389274903EBC3039B0005330E
:10F2400081FB0321DB17C3EBA101284689B2FBF741
:10F2500069FB338A03EB8303590089B22846FBF725
:10F2600061FB1D4B059D1B789B0743BF318901F551
:10F270007A7189B24FF47A712846FBF753FB0C9BE5
:10F28000327D591C0C9128461A7029F00BF8134A4C
:10F2900094F89C321178013393FBF1F201FB1233A5
:10F2A00084F89C32EFE600BF24C000207C5D002083
:10F2B0005C300020C0C00020E4BF0020AC2500204E
:10F2C000C4C00020C5C00020C8C00020E4BF00208A
:10F2D0001C3E002067666666183E0020CCC00020F9
:10F2E00094F85631002B41F0CB85D34B1A6802F0CD
:10F2F0000803002B48F603414AF60B404BF60F4338
:10F3000049F6074604BF03460E4612F0040F4FF0BD
:10F31000190118BF1E46970684F8561103D546F406
:10F32000804646F02006C54B5F79C6F30909002FD9
:10F3300042F013819B79002B42F01E821F4664200D
:10F340004FF0FF3A4FF0000E0C960D96ADF83E7060
:10F35000ADF83CE0CDF842E0CDF846E0CDF84AE02B
:10F36000CDF83890ADF840A08DF84E000CAE0FCE21
:10F37000B34F84F805E00FC796E80F0007C727F8DA
:10F38000023B39464FF0010E1B0CFE261F20C822FF
:10F3900001F81E39A670A27184F807E0E07094F8B5
:10F3A0006601207180F0F10383EA0313DAB21309D6
:10F3B00083F0E70343EA022383EAC2031BB283EA32
:10F3C0000312D2B2C3F3072383EA121343EA0223E0
:10F3D00083EAC2031BB283F0C80282EA0212D2B2ED
:10F3E000C3F3072383EA121343EA022383EAC20327
:10F3F0001BB283EA0E0686EA0616F6B2C3F30722AC
:10F4000082EA161242EA062200EB0E0382EAC606E0
:10F4100007EB0E0084F86631268011F8013B73403B
:10F4200083EA0313DBB21A0982EA162242EA0322B4
:10F4300082EAC3031BB29EB281422680EDD183F0E3
:10F440007C0383EA0313DBB24FEA131E8EEA162E07
:10F450008EEA032E8EEAC30E0FFA8EFE1FFA8EFC82
:10F46000784FA4F800C05FFA8EFE4FEA1C2C84F897
:10F4700028C084F827E007F5C77904F1220A386824
:10F480007968BA68FB684E460FC610375745B146D3
:10F49000F5D1386830606C4E3B7989F8043006F15C
:10F4A000270784F8B5E184F8B6C116F8011F28686B
:10F4B000F9F7ACFFB742F8D194F85731002B41F07F
:10F4C000E4846249DBF8002009780A2084F85701B7
:10F4D000002901F000865E4E01293088079042F233
:10F4E000518170880690022902F04F80B088059003
:10F4F000032902F05E81F0880490042902F054810F
:10F500000529308902F04C810629B6F80A9002F0EC
:10F5100044810729B6F80CC000D0F38994F866112D
:10F520000C920F4687F0300282EA0212D2B216091C
:10F530004849089786F07A0646EA02260988277124
:10F5400086EAC202444EC1EB012186FB017A079E86
:10F550004FF0000E66F30F0E069E12B266F31F4EBA
:10F560008A44059ECDF834E0C917C1EB6A2A00270A
:10F5700082EA0211C9B266F30F07C2F3072200261E
:10F5800082EA111260F30F06002007926CF30F005D
:10F59000049A8DF845A063F31F40079B109062F317
:10F5A0001F4769F31F464FF000090E970F968DF81D
:10F5B000449043EA01220DF1300E82EAC106BEE812
:10F5C0000F0036B286F0C80C8CEA0C1C1C4F84F875
:10F5D00005905FFA8CFCC6F307260FC786EA1C1657
:10F5E00046EA0C239EE8030083EACC031BB283F0B7
:10F5F000230247F8040B82EA0212D2B2C3F30723B4
:10F60000089E83EA1213384643EA022383EAC202C1
:10F6100006F1010E20F814194FF0230C1621FE26D6
:10F62000C82384F866E102372280E17084F807C0BD
:10F63000A670A371114611E0143E0020003E002088
:10F64000B4250020AE2500203B27002038A500204F
:10F650003CA400207CBF00200308208010F8013B60
:10F660004B4083EA0313DBB21A0982EA112242EA11
:10F67000032282EAC3031BB299B2B8422180EDD1C2
:10F6800083F0F40383EA0313DBB24FEA131E8EEA1E
:10F69000112E8EEA032E8EEAC30E0FFA8EFE1FFA8B
:10F6A0008EF7C84E27804FEA172C5FFA8EFE84F83B
:10F6B0001EE084F81FC07168B2683068F36806F510
:10F6C000C7770FC730697169B26904F28F1607C72F
:10F6D00004F2AD1784F8ADC184F8ACE116F8011F4F
:10F6E0002868F9F793FEB742F8D194F85A31002B05
:10F6F00041F0DB83B44B06931B681922980684F80B
:10F700005A2140F1EA82B14BB14E1B78990741F181
:10F710002187337D042B8CBF03270227FFF702FAD2
:10F72000338A32890C9003EB83035B00ADF84A30D7
:10F730004FF47A7033688DF84C700E93F18996F817
:10F7400014E073688DF84DE000FB02F24FF0000CFE
:10F750000CAF4FF0FF30CDF834C010920F93ADF8DE
:10F7600048101190BE46BEE80F000597994F0FC78D
:10F770009EE80F0007C73A46182122F81C39E171AC
:10F7800094F8661184F805C081F0780383EA0313C6
:10F79000D8B2030983F0F60343EA002383EAC003E7
:10F7A0001BB283EA0310C0B2C3F3072383EA10132A
:10F7B00043EA002383EAC0031BB283F0C80080EA57
:10F7C000001E5FFA8EFEC3F3072080EA1E1040EA97
:10F7D0000E2080EACE0000B280F0180383EA031303
:10F7E000DBB2C0F3072080EA131040EA032080EA6E
:10F7F000C30301F1010EFE204FF01E0C4FF0C809AB
:10F80000A0700237217184F866E1238084F803C078
:10F8100084F80690184612F8011B414081EA011154
:10F82000C9B20B0983EA102343EA012383EAC10129
:10F8300009B288B2BA422080EDD181F0180181EA84
:10F840000111C9B20A0982EA102383EA012383EA7B
:10F85000C1031BB29AB25B490491DBB24FEA122C8E
:10F860002280079384F827C084F826300F4601F5DC
:10F87000C77A04F1220938687968BA68FB68D64605
:10F88000AEE80F0010374F45F246F4D13868CEF895
:10F890000000DFF84C919DF81C3084F8B43109F178
:10F8A000260784F8B5C1CA461AF8011F2868F9F777
:10F8B000ADFD5745F8D1FFF735F9069B71681B6818
:10F8C0003289069113F0140F4FF47A71D6F800E0E4
:10F8D00001FB02F141F00B860E4694F866A10C90F4
:10F8E0008AF06A003C4B3D4FB3F90420CDF834E078
:10F8F00080EA0010C0B2030983F0D50343EA002375
:10F9000083EAC0031BB283EA0310C0B2C3F3072328
:10F9100083EA101343EA002383EAC0031BB287FB88
:10F920000207D2174FF0000CC2EBA7020698DDF8D1
:10F9300014E0109683F0C8070E900F91ADF84A209E
:10F94000ADF844C0ADF846C0ADF848C087EA071727
:10F95000FFB2C3F30726BEE80F0086EA171646EA91
:10F96000072686EAC7071B4E84F804A03FB20FC6DD
:10F9700087F021039EE8070083EA0313DBB2C7F395
:10F98000072787EA13170AF1010E47EA032786E8DB
:10F99000070087EAC30384F866E14FF0210A4FF0BD
:10F9A000FE0E1C27C8220C3684F805C084F807A078
:10F9B00084F802E0A6F11C01E7701846A2712380CA
:10F9C00010E000BFAE250020143E0020183E0020AD
:10F9D0001C3E0020B4250020F83D002067666666C6
:10F9E0003B27002011F8012B424082EA0212D2B2DA
:10F9F000130983EA102343EA022383EAC20212B204
:10FA000090B2B1422080EDD182F0680282EA021207
:10FA1000D2B24FEA121A8AEA102383EA022A8AEA49
:10FA2000C20A0FFA8AFA1FFA8AF3D74E23804FEAE6
:10FA3000132C5FFA8AFA04F1220384F825C084F8B3
:10FA400024A006F5C77E0693F36830687168B26833
:10FA500077460FC7069B10369E42BE46F4D13388C8
:10FA6000CA4E3B804F4684F8B2A184F8B3C117F860
:10FA7000011F2868F9F7CAFCBE42F8D194F866E184
:10FA8000C34AC44E84F804E08EF0EB0383EA031308
:10FA9000D9B20B0983F0C50343EA012383EAC1030A
:10FAA0001BB283EA0310C0B2C3F3072181EA10112D
:10FAB00041EA002181EAC0010CCA09B281F0C807FD
:10FAC00087EA0717FFB24FF0000C0C92C1F3072131
:10FAD000059A0D93CDF838C081EA171343EA07233E
:10FAE00007CA83EAC7031BB283F0310786E8070021
:10FAF00087EA0717FFB2C3F3072383EA171343EA22
:10FB0000072383EAC703277A607AA17AE27A267B01
:10FB100084F805C01BB25F4087EA0717FFB2C3F342
:10FB2000072383EA171343EA072383EAC7031BB2B9
:10FB3000584080EA0010C0B2C3F3072383EA1013D1
:10FB400043EA002383EAC0031BB2594081EA011053
:10FB5000C0B2C3F3072181EA101141EA002181EA12
:10FB6000C00109B24A4082EA0212D2B2C1F30723AD
:10FB700083EA121343EA022383EAC2031BB25E4004
:10FB800086EA0616F6B2C3F3072383EA161343EA9E
:10FB90000623607BA17BE27B277C94F811C083EA7B
:10FBA000C6031BB2584080EA0010C0B2C3F307235B
:10FBB00083EA101343EA002383EAC0031BB25940CF
:10FBC00081EA0111C9B2C3F3072383EA111343EA9F
:10FBD000012383EAC1031BB25A4082EA0212D2B265
:10FBE000C3F3072383EA121343EA022383EAC2031F
:10FBF0001BB25F4087EA0717FFB2C3F3072383EA0C
:10FC0000171343EA072383EAC7031BB28CEA030CEA
:10FC10008CEA0C1C5FFA8CFCC3F3072383EA1C13E9
:10FC200043EA0C2383EACC03A17CE27C5A4F1BB24B
:10FC3000594081EA0111C9B2C3F3072383EA1113C2
:10FC400043EA012383EAC1031BB25A4082EA02124B
:10FC5000D2B2C3F3072383EA121343EA022383EAEF
:10FC6000C2031BB283F0270686EA0612D2B2C3F3A0
:10FC7000072686EA121646EA022686EAC20636B247
:10FC80000EF10103B2B231204FF0FE0C0C2184F8CA
:10FC90006631C8234FEA122E5FFA86FA2280E0719D
:10FCA00084F802C0E170A371049E84F814A084F863
:10FCB00015E07168B268F3683068B6F810C00FC715
:10FCC00027F803CB84F8A3E184F8A2A119F8011F57
:10FCD0002868F9F79BFB4F45F8D194F85E71002F27
:10FCE00041F0DE802D4B94F866E1B3F90010B3F9D2
:10FCF0000220B3F904309FED2A6A677107EE103ACB
:10FD0000DBF800300C938EF06A0383EA031306EEEF
:10FD1000901AD9B20B0983F0D50343EA012383EA91
:10FD2000C1031BB283EA03115242C9B207EE902A03
:10FD3000C3F3072383EA111343EA0123F8EEE77ABA
:10FD4000F8EEE66AB8EEC77A83EAC1031BB267EE43
:10FD5000867A66EE866A27EE067A002083F0C80C63
:10FD6000CDED0E7ACDED0D6A8DED0F7A10901190DC
:10FD700012908CEA0C160DF13009F6B2C3F3072C81
:10FD8000B9E80F000EE000BFAE2500205F2700207D
:10FD9000C0500020B42500203C270020F83D002062
:10FDA00088C3E43A8CEA161C4CEA062C8CEAC60C92
:10FDB000D04E0FFA8CFC0FC68CF01E0799E8070096
:10FDC00087EA0717FFB2CCF3072383EA171343EA46
:10FDD000072386E8070083EAC707C8214FF0050913
:10FDE0004FF01E0CFE231C200EF10102A17184F8BD
:10FDF0005E9184F807C0A370E070A6F1100184F84A
:10FE000004E00C36278084F8662111F8013B7B4022
:10FE100083EA0313DBB21A0982EA172242EA0322B9
:10FE200082EAC3031BB29FB2B1422780EDD183F0B7
:10FE3000270383EA0313DBB24FEA131E8EEA172E61
:10FE40008EEA032E8EEAC30E0FFA8EFE1FFA8EFC88
:10FE5000A94FA4F800C05FFA8EFE4FEA1C2C84F86C
:10FE600025C084F824E007F5C77904F1220A386830
:10FE70007968BA68FB684E460FC610375745B146D9
:10FE8000F5D19E4E3B88A9F8003006F1240784F88E
:10FE9000B2E184F8B3C116F8011F2868F9F7B6FA81
:10FEA000B742F8D194F85F91B9F1000F40F0F287B2
:10FEB000934B1B68052284F85F219A0641F1158156
:10FEC000904ADFED917AD18907EE101AB8EEC77A21
:10FED00013F0140F27EE277A01F071838B4BDFEDBF
:10FEE0008A6AD3ED007AF8EEE77A67EEA67A94F89C
:10FEF00066C1874B874AB3F90410B2F90620864ED3
:10FF000086488DED0D7A8CF0220383EA0313DFB26D
:10FF10003B0983F0590343EA072383EAC703B2F599
:10FF2000FA6F1BB2A8BF4FF4FA6283EA0317FFB25D
:10FF3000B2F57A7FC3F3072383EA1713B8BF4FF4F0
:10FF40007A724FF0640E43EA0723A2F57A720EFB31
:10FF500002F283EAC70786FB02E680FB01E03FB2BC
:10FF6000C917D217C2EBA612C1EBA0034FF0000ACB
:10FF70000CA987F0C806CDED0E7AADF84220ADF899
:10FF80004030CDF830A0CDF83CA08E4686EA06166B
:10FF9000F6B20591C7F30727BEE80F0087EA1617E8
:10FFA00047EA062787EAC606524FDEF800E084F8E3
:10FFB00004C00FC736B286F04A0383EA0313DBB2EC
:10FFC000C6F3072181EA13113A4641EA03210CF1F5
:10FFD000010C81EAC303142042F810E9FE264FF019
:10FFE0004A0E002184F866C14FF0C80CE0702380EF
:10FFF000043784F807E0A670617184F806C01846DB
:020000040801F1
:1000000012F8011B414081EA0111C9B20B0983EAD0
:10001000102343EA012383EAC10109B288B2BA423C
:100020002080EDD181F0140181EA0111C9B24FEABB
:10003000111E8EEA102E8EEA012E8EEAC10E2E4B74
:100040000FFA8EFE1FFA8EF61F464FEA162C5FFA45
:100050008EFE84F81CE084F81DC0386859689A68E0
:10006000DB68B7F818A0049726803E4607F5C777E7
:100070000FC73069716903C704F28F16A7F800A093
:10008000374684F8ABC184F8AAE104F2AB1A17F83A
:10009000011F2868F9F7BAF9BA45F8D1204B214A6F
:1000A0001B781278013B12F00100DBB214BFC021B3
:1000B0004021172B03D81C4A134493F830901B4B54
:1000C0001A8897071ABF002341F01001012312F488
:1000D000027F18BF022312F0100F18BF062312F080
:1000E000200F18BF1023002841F008824FF0030CA6
:1000F0001EE000BFB4250020AE2500203B270020D5
:10010000143E00201C3E00200AD7233CF43D002072
:10011000F83D00203CA40020D34D6210676666665F
:10012000F8680020593A0020C8270408E838002061
:1001300094F866E10C938EF0460383EA0313DAB277
:10014000130983F0920343EA022383EAC2031BB23A
:1001500083EA0310C0B2C3F3072282EA101242EA14
:10016000002282EAC00212B282F0C80787EA0717AB
:10017000FFB2C2F3072282EA171200238DF837C0BC
:10018000032042EA072C059A8DF834908DF835301B
:100190008DF836108DF8380007CA8CEAC70C0FFAB4
:1001A0008CFCD04FE3718CEA0C1903C75FFA89F914
:1001B000CCF3072C8CEA191C4CEA092181EAC90905
:1001C00094F808C03A700FFA89F98CEA090C8CEAA5
:1001D0000C1C5FFA8CFCC9F3072282EA1C1242EA6B
:1001E0000C22607AA17A94F80B90637182EACC02B7
:1001F00012B2504080EA001C5FFA8CFCC2F3072068
:1002000080EA1C1040EA0C2080EACC0000B2414099
:1002100081EA0111C9B2C0F3072282EA111242EA4F
:10022000012282EAC10212B289EA020989EA0919A5
:100230005FFA89F9C2F3072282EA191242EA092217
:1002400094F80CC0607BA17B84F804E082EAC902C8
:1002500012B28CEA020C8CEA0C1C5FFA8CFCC2F322
:10026000072282EA1C1242EA0C2282EACC0212B273
:10027000504080EA0010C0B2C2F3072282EA101296
:1002800042EA002282EAC00212B2514081EA011120
:10029000C9B2C2F3072282EA111242EA012282EABB
:1002A000C102E17B94F8109013B281EA030282EA62
:1002B0000212D2B2C3F3072383EA121343EA0223E2
:1002C00083EAC2031BB289EA030282EA0212D2B2B3
:1002D000C3F3072383EA121343EA022383EAC20328
:1002E0001BB283F0320282EA0212D2B2C3F30723B6
:1002F00083EA121343EA022383EAC2031BB29AB2CF
:100300004FF0FE0C5FFA83FB0920C8210EF1010EAD
:1003100084F802C04FEA122CE070A17184F866E103
:10032000228084F812C084F811B0049B18685968C0
:100330009A68B3F80CA007F5C07EAEE8070007F591
:10034000C8778EF80290AEF800A084F8A0C184F8B7
:100350009FB116F8011F2868F9F758F8B742F8D18D
:10036000039BC4F85031FEF78ABEDFF898A15E4EB9
:10037000DFF89491412017F057FEBAF9023086FB5E
:100380000320DB17C3EBA00080B217F031FEBAF9EF
:10039000003086FB0320DB17C3EBA00080B217F010
:1003A00027FEBAF9043086FB0320DB17C3EBA0005D
:1003B00080B217F01DFE99F800103868F9F726F89A
:1003C00094F848A11AF0010600F0F784474B069311
:1003D0001B689A0673D5464B464E1B789B0741F126
:1003E0005180337D042B8CBF4FF0030A4FF0020A7B
:1003F000472017F019FE306817F0C6FD706817F037
:10040000C3FD3D4AF3893868A2FB0323C3F34713B6
:1004100019460493F8F7FAFF069B99F800101A683A
:10042000049B12F0140F83EA010389F8003040F0B6
:1004300067863389642000FB03F017F0A5FD367D45
:1004400038684AEA8606F6B23146F8F7DFFF99F8CF
:10045000003038685E40314689F80060F8F7D6FF12
:1004600094F848A1BAF1000F29D1244E4F2017F07B
:10047000DBFD306817F088FD706817F085FD504689
:1004800017F082FD01213868F8F7C0FF184A99F883
:1004900000301678386806F00106314683F0010313
:1004A00089F80030F8F7B2FF99F8003038685E40FC
:1004B000314689F80060F8F7A9FF94F848A1039B3A
:1004C0000F4AC4F844310AF10103DBB2A2FB031264
:1004D000D20802EB8202A3EB420384F84831FEF714
:1004E000B1BD00BFB425002067666666143E0020DB
:1004F000183E00201C3E00201F85EB51C0500020FC
:10050000CDCCCCCCF83D0020943D002094F8A43212
:10051000C24AC4F8A08202EB8302926C42B314ADCB
:1005200004F2AB23BE4E45F8203D002104F2BD236A
:1005300031800D9380211523A52784F8AA322846FF
:1005400084F8A91284F8A872904728463188FAF7EF
:100550000FFA0C9DB34804F52A716D1A152DA8BF2A
:1005600015252A462FF0BAFCAF4A94F8A43215702C
:10057000AE4A013382FB0312A2EBE37202EB4202AA
:100580009B1A84F8A432FEF78ABDA94AA94BD4F875
:100590001411DBF800001B88D77AA74A401A4FF4E1
:1005A0007A71DEB201FB07F11B0A96771675884255
:1005B0004FF00006D37753759670167180F0D18492
:1005C0009E4E9F4BD6F800C01B689E4E9E48DFF89B
:1005D000989201688068DFF894E286FB0376DB1767
:1005E000C3EB661303F5FA739BB293761B0AD376BB
:1005F00089FB0173C917C1EBA30189FB007911774E
:10060000C0170912C0EBA90051778E4982F820006B
:100610000CF5EA43001281FB0C71303382F82100A3
:100620004FEAEC701B12C0EB6110884E9EF800E0A0
:1006300082F823307830864B82F824000CF13001A8
:10064000307D03901EF0020F82F82210987600F0A1
:100650008584D6F800E07F4AD6F804A07E48DFF80B
:1006600010C282FB0E194FEAEE7182FB0A72C1EBD7
:10067000A9514FEAEA79C9EBA25200FB01E900FB5C
:1006800002A009EB490900EB40004FEA490940008C
:10069000049207468CFB0920801405908CFB072CE4
:1006A000F089049A3689079702EB820206F5FA76FA
:1006B00000EBC00002EB8202B6B204960892059EDF
:1006C0008200099201EB81014FEAE972B01A01EB55
:1006D0008101624E06910246039906FB1292069E24
:1006E00040B2052900EB86004FEAE7714FEAAC4CB7
:1006F0005A4E0590ACEB0100014606FB1070089EB7
:10070000504FDFF870C14FEADA7A49B201EB860147
:100710004FEADE7E87FB006983F80EA087FB026A42
:10072000099F83F809E0DFF850E13E468EFB066E34
:10073000BCF8006003969DF810605E75049EBDF8DD
:1007400014C083F80AC04FEA162689B204964FEA0D
:10075000E2724FEAE777424ED973C2EB6A12C7EBF7
:10076000AE174FEA1C2A4FEA112E4FEAE0700399A8
:10077000368883F80BA0C0EB691083F810E04FEACD
:1007800022291A739DF810209A754FEA202CC7F37E
:10079000072A4FEA112134BF4FF0320E4FF0330ECB
:1007A0009DF80C2083F80D90587483F812C0DF7107
:1007B00083F808A0DA74197583F81BE01E77C4F873
:1007C0001081FEF7BBBBDFF8B490D9F80000F8F752
:1007D00009FE00283EF441ACD9F800000121F8F7E9
:1007E000FDFD0222002386F874203B70FEF735BC25
:1007F00094F82C1194F82D3138684A1C013384F890
:100800002C2184F82D31F8F701FEFEF7FABB154CC8
:10081000DFF86C904FF0000A3FE000BFC8270408E3
:10082000A2BF0020F02E0020052F00205655555560
:10083000703B00209C3B002064C00020E83D00206D
:10084000F43D00201F85EB51903B00201C3E002012
:1008500090C000206BCA5F6B806967FF40420F0049
:100860001E390020AC25002067666666183E002011
:1008700083DE1B4380BF0020D34D6210A8340020CC
:10088000200000201B2B00F06F820D2B00F04B810D
:100890004FF0010389F801303868F8F7B3FD0028FC
:1008A00039D03868F8F7A6FD83B27E2BDBF800203C
:1008B0002AD099F801100029EED194F82E21002AAF
:1008C000E0D07D2B00F0368294F83CE1BEF1000FC1
:1008D00004D080F02003DBB284F83C11511CC9B273
:1008E0002244092984F82E1182F8303100F0168252
:1008F0000829D1D8B4F83A21134403EB132303F0A9
:10090000FF03A4F83A31C7E784F82EA184F82FA199
:1009100089F801A0C0E794F83D3133B194F8313142
:1009200084F83D01302B00F0C18594F82F21C54B90
:10093000C549DFF850A3DFF850E391464A46002A44
:100940003EF46FABDBF80020921B012A24D894F808
:100950003E21002A40F01E8294F83FC133F81C006B
:10096000F8B94FF0010284F83F210A689706E5D5EF
:100970009AF800209007E1D5B44EB549F2894FF4BA
:10098000F36303FB02F381FB0321DB17C3EB61116C
:100990004FF4036017F082FB002384F82F31FEF739
:1009A00040BB0CF1010C5FFA8CFCB0F5E06F84F8F1
:1009B0003FC100F098801BD8B0F5047F00F0238180
:1009C00035D8B0F5887F00F0CD80B0F5007F00F01D
:1009D000B380B0F5807FB1D10A685207AED59D4B88
:1009E000196817F05BFB002384F82F31FEF719BB61
:1009F000B0F5026F00F05A816AD8B0F5E46F00F0EC
:100A00008180B0F5006F00F0D680B0F5E26F95D12F
:100A1000914BDA6B998A642303FB02F393FBF1F1A8
:100A200017F03CFB002384F82F31FEF7FABAB0F53B
:100A3000826F00F05181B0F5C06F00F02781B0F5F2
:100A4000806F7FF47BAF94F840310133DBB2032B2E
:100A500000F2AD8142F2107184F8403101FB03F1E4
:100A60007E4B1B88002B40F0A08101317C4B1B7812
:100A7000DB077C4B1B8848BF0431DF0748BF0A31C6
:100A8000980748BF14311A0648BF2831DF0548BF10
:100A90002831580748BF64311A0748BFC8319F053D
:100AA00048BF01F5C871980648BF01F57A71DA06AA
:100AB00048BF01F5FA615F0648BF01F57A614FF45E
:100AC000806017F0EBFA002384F82F31FEF7A9BA03
:100AD000B0F5046F1AD0B0F5116F52D0B0F5036FB6
:100AE0007FF42CAF41E75C4B91469A6B998A642363
:100AF00003FB02F393FBF1F117F0D0FA84F82F9186
:100B0000FEF78FBA544B91461A6CEFE7564BB3F988
:100B1000041001EB81019146490017F0BFFA84F8F7
:100B20002F91FEF77EBA4FF0010184F82E1184F860
:100B30003031A4F83A21AFE69EF80620002A3FF4AF
:100B4000FDAE4A4B4A491B6881FB0321DB17C3EB0F
:100B5000A1014FF4007017F0A1FA002384F82F319F
:100B6000FEF75FBA0A6852077FF5E8AE414B4FF4D3
:100B70008870196817F092FA002384F82F31FEF775
:100B800050BA9EF80520002A3FF4D8AE3A4A1078B1
:100B900000283FF4D3AE394B1B8803EB8303590085
:100BA00091FBF0F14FF4116017F078FA002384F80C
:100BB0002F31FEF736BA0A6897067FF5BFAE9AF86E
:100BC000002090077FF5BAAE1CF0010F1F4E2049A0
:100BD00000F05C84726882EAE273A3EBE27303EBD9
:100BE0005303A1FB0331C908002AACBF41F0004107
:100BF00041F040414FF4006017F050FA002384F8B0
:100C00002F31FEF70EBA9EF80520002A3FF496AE6B
:100C1000194A107800283FF491AE194B5B7B002BEA
:100C200000F09484154B1B8893FBF0F000EB8000E0
:100C300041004FF4047017F031FA002384F82F318B
:100C4000FEF7EFB9C8270408143E00201C3E002020
:100C50001F85EB51F43D0020A03D0020A0BF0020E7
:100C6000593A0020E8380020F83D0020903B002051
:100C700067666666E83D0020D33B00209C3B002071
:100C8000703B0020183E0020003E00209EF8062009
:100C9000002A3FF453AEC34B4FF4C060996817F07D
:100CA000FDF9002384F82F31FEF7BBB90F68BF06AA
:100CB0007FF544AE9AF800C01CF0020F3FF43EAE40
:100CC000B94E33896421914601FB03F117F0E6F92F
:100CD00084F82F91FEF7A5B90A68900640F1F180DB
:100CE000B24BB14E1878317D00F00203002B0CBFDF
:100CF00000234FF47A7340F6B83208BF4FF4FA621B
:100D000010F0010F18BF134619444FF4826017F01A
:100D1000C5F9002384F82F31FEF783B9B4F83A21DE
:100D2000C2F1FF0293427FF4B3AD4FF0010384F8A8
:100D30003D31ADE54FF0010384F83C31ACE5FDF702
:100D4000F1FE9B4B1B68C01A40F6B833984200F284
:100D50001E81DFF89CA29AF804303A2B00F0BA8288
:100D600000233B70FEF779B93868F8F74BFB002891
:100D70007FF48EAD4FF0010384F82F318CE5C4F879
:100D8000203184F818318B4F17F0D6F994F82431BC
:100D9000FEF71DB98849062016F052FF002384F89B
:100DA0003E0184F82F31FEF73CB902315EE60123A3
:100DB00084F8403142F2107152E6804B1B88D8050E
:100DC00013D4D90600F17A839A0600F1F18358060C
:100DD00000F1F383190700F1F983DA0700F11484B5
:100DE00013F0020F0CBF04260C26754B754A1B78B6
:100DF000D27803F001030AB143F0020353200493B5
:100E000017F012F9704A128802EB820202EB82029A
:100E1000900080B217F0ECF8002017F0E9F86B4A68
:100E20006B4912883868C2EBC212520081FB023152
:100E300011444FEAE27ACAEB612A5FFA8AFA514614
:100E4000F8F7E4FA99F80020049B38681E438AEA10
:100E5000020A002189F800A0F8F7D8FA314638686C
:100E6000F8F7D4FA99F8003038687340DBB21946C5
:100E700089F80030F8F7CAFA94F848A1FFF7F2BAF7
:100E8000013B84F85631FEF717BB013B84F857311C
:100E9000FEF72BBC09F1FF3984F85F91FFF760BAC8
:100EA000013F84F85E71FEF7FDBF013B84F85A31C3
:100EB000FEF713BF47493A2016F0C2FE2870FEF72E
:100EC000E2B8454A1268120600F1FA82434A127BE0
:100ED000002A3FF433AD94F84111032900F28A83CC
:100EE000DFE801F0322819023D4B1B6859799A79E5
:100EF000DB7901F1407101EB022101EB0341002399
:100F000084F841314FF4826017F0C8F8002384F868
:100F10002F31FEF786B8334B1A68137A50799278DE
:100F20001B0403EB002313444A1C84F8412103EB08
:100F30000161E7E72B4B1A68D379107952781B04CB
:100F400003EB00231344EFE7264B1A689379D0781C
:100F500012781B0403EB00231344E5E72D22DA7615
:100F60002DE4214BDBF800101B78C4F81411013B71
:100F7000012B3FF625AB1021022391701371FFF76F
:100F80001FBB17F0C9F801233370FDF7F3BF174AF1
:100F9000B2F84A3100210133A2F84A313970FEF724
:100FA0005CB800BF903B00201C3E0020183E002093
:100FB00030C20020983D002095800208E8380020CB
:100FC000593A0020F03800209C3B00207CBF0020D4
:100FD0000308208005830308185C0020703B002074
:100FE000E0CD00203839002094BF0020AC2500203F
:100FF00018C20020A64EA74B00930024A6F13F0183
:10100000A54BA64A0A9106F8404CA5490B960CA898
:10101000F9F786FD0A9E731C0A9334700A9B2922F5
:10102000591C0A911A700A9BEA22591C0A911A70DB
:101030000A9BC822591C0A910CA81A702DF0CAFFED
:10104000471C0CA93A460A982EF048FF0A9AD31971
:1010500001330A93D4550A9B5A1C0A921C700A9BAE
:101060005A1C0A921C700A9B5A1C0A921C700A9BFA
:101070005A1C0A921C700A9B5A1C0A921C700A9BEA
:101080005A1C0A921C700A9B5A1C0A921C700A9BDA
:101090005A1C0A921C700A9B5A1C0A921C700A9BCA
:1010A0005A1C0A921C700A9B5A1C0A921C700A9BBA
:1010B000FF22591C0A911A700A9B0122991814A840
:1010C0000A911A7050F8283D9B1B337027F0EAF8FC
:1010D0002C70FDF7D8BF8C468946084604910591CF
:1010E000069107910B46FEF719BA9FED6E7A13F041
:1010F000140F08BFF0EE477A7EF4F0AEFEF7F7BEAD
:10110000694B1868FFF799B9684A614B12680D93EB
:10111000A3F14007002103F8401C2123D100BB703C
:1011200040F13A8262490326624B1B885A0500F15E
:101130002982D80700F13E8203F002035E4A002BA9
:101140001CBF03261146DFF88891324648462EF030
:10115000C5FE06EB090314A80133A9F1020140F80A
:10116000203D00225B1A06F809207B7027F09AF8D0
:10117000FEF742B8C4F81C8186F80090FDF7FABE6D
:10118000434A4E4B0D9214AEA2F13D0046F8200D9D
:1011900019884B4FA2F1400300204FF00A0E02F8CD
:1011A000400C082283F801E030469A70F9F7BAFB48
:1011B0003B684449DA1781FB0313C2EBA30399B2DE
:1011C0003046F9F7AFFB18F0A5FFBF680C9B3A0C4F
:1011D000591C0C911A700C9B3A0A591C0C911A70EC
:1011E0000C9B5A1C0C921F700C9B5A1C0C92187072
:1011F000304627F057F8FDF7FCBF334F9FED338A99
:10120000B7F9022022480D9007EE902AF8EEE77A0F
:1012100014AE67EE887AA0F13D01FDEEE77A46F85C
:10122000201D00F8403C0823CDED037A00F83F3C38
:101230001E23BDF80C1000F83E3C3046F9F772FB57
:10124000B7F9003007EE903AF8EEE77A304667EEED
:10125000887AFDEEE77ACDED037ABDF80C10F9F748
:1012600061FBB7F9043007EE903AF8EEE77A3046C2
:1012700067EE887AFDEEE77ACDED037ABDF80C10C3
:10128000F9F750FB304627F00DF8FDF7AFBF00BF70
:10129000E4BF0020027C0020545A04085C5A040871
:1012A000685A040800000000F43D002098BF0020A8
:1012B000405A0408E8380020505A04089C3B00209B
:1012C000903B002067666666F83D002058A08B4181
:1012D000A7BF00209AF80240C4B1013CE4B2013437
:1012E00054445146002211F8013B534083EA031352
:1012F000DBB2120ADE0042EA03228C4286EA1313B2
:1013000082EA0302EFD1002A7FF42AADC04AC14E1F
:10131000C14B1288C149C24CF261DFF838931A6898
:1013200009689B68F262B4F84A21F066F364D9F860
:101330000000F163F265F6F71FFF039000287DF4CB
:1013400087AE0221D9F80000F8F748F894F84C313C
:101350009AF803200492642B4FF0040286F874205C
:1013600040F07C8194F84D31072B04BF9DF80C3080
:1013700084F84D3194F84D31079306EB031ADAF8EF
:101380000410039108462DF025FEDAF808100691A6
:101390005FFA80FA08462DF01DFEC0B205900AEBF8
:1013A0000002079B9F48039903900832C27123F003
:1013B0000F0286468272059803F00F0300EBCA0005
:1013C0008EF80D3052468EF80E000EF10F002EF002
:1013D00085FD954B059A06990AF1090018442EF0EF
:1013E0007DFD0398C37903F1010ACBB1013B5FFA9C
:1013F00083FC0CF1080CDFF860E284440023073022
:1014000010F8011B59408B00CA0883EA410302F01F
:1014100018024B404EFA02F253408445DBB2EFD142
:10142000814A04980AF8023020F0A4FE94F84D3165
:101430000022013384F84D3184F84C21039BDDF800
:101440000CA09B785BB11AF80510D9F80000F7F7EB
:10145000DDFF01359AF80230EDB2AB42F3D894F8D3
:101460004C310322013384F84C3186F874203A70F1
:10147000FFF7ABB902213868F7F7B0FF94F82431D1
:10148000FDF7A5BD4FF0010AFEF7B2BF326882EA50
:10149000E273A3EBE27303EB5303A1FB0331C9082F
:1014A000002AB8BF41F08041FFF7A4BB5F49881F05
:1014B00016F06AFC84F83E01FFF737BA342694E44C
:1014C00010230026042218460CA98DF830308DF820
:1014D00031208DF832608DF833608DF834608DF8EE
:1014E000356016F0BBFD84F82F61FDF79ABD4B4BBC
:1014F0001E6806EB86067600FEF7EFB94C4AD278F6
:10150000002A0CBF4FF0040C4FF0050CFEF710BE84
:10151000012338683370F7F76DFF06463868F7F730
:1015200069FF72067DF426AD8A2851D08E287DF49D
:1015300021AD94F81831002B7DF438AD3D4BC4F843
:1015400020312D2384F82431FDF71BBD304B188842
:10155000FFF76CBB0127FEF7E1B82D499A790B889C
:1015600003EB830303EB83039F00BFB2002A00F069
:101570001181294B1B680FFA83FA18F0CBFD40B29A
:10158000FDF7E0BE03262C49DDE59C46994618464A
:1015900004930593FDF7C2BF284B294A1B682949CC
:1015A00003F48003002B16BF114604260326BBE577
:1015B00024261AE424490426C5E5102615E41389D7
:1015C00007EE903AF8EE677AFEF791BC20260CE41D
:1015D0001E4B1B689B067DF5CDAC94F81831002B93
:1015E0007DF4E4AC1A4BC4F820312D2384F8243167
:1015F000FDF7C7BC4B1CDBB2042B84F841314FEA2A
:1016000001613FF47CAC7DE40826FFF7EEBB00BF30
:101610009C3B002020000020903B0020F43D002057
:10162000AC25002004A000200AA00020E426002011
:10163000F038002064C00020445A0408185C0020E0
:10164000405A0408385A0408485A0408143E002036
:1016500090C00020A83400200007090E96F875A05D
:10166000574905951AF00F0F04BF0AF1010A5FFAF6
:101670008AFABAF1070F28BF4FF0010A4FEA0A1C95
:1016800006EB0C03187C4F4B03930A18002392F8C7
:1016900024104C4A93725FFA8CF31A464A4B9646D2
:1016A00006EB0C024EEA000001291870D26803F123
:1016B00001000CD90239C9B28D1C1D44034603F840
:1016C000012BAB424FEA1222F9D101310844B44454
:1016D00022F060030AF1010A9CF811205FFA8AFAED
:1016E0001343BAF1080F037000F1010340D04FEA31
:1016F0000A1C06EB0C01344A087C314901449A1A51
:1017000091F8241055180EF1100E132D5FFA8EFE6D
:10171000C6DD059D0398DFF8BCE0D2B2931DDBB2B5
:1017200043F04001C17103F1010CCBB10532D3B2DA
:101730000833C31805930EF10100002310F8011BB4
:1017400059408B0083EA4103CA084B401F4902F00D
:10175000180241FA02F25340059A8242DBB2EDD1FF
:1017600004980CF80E3086F875A020F003FD65E6AD
:10177000154A059D9A1ACDE7154B6420B3F900A0D0
:10178000FDF7E0BD9C4699461846049305930693E1
:10179000FDF7C4BE4FF0FF33EDE69C46FDF7BEBE3D
:1017A0009C469946FDF7BABE9C4699461846FDF7F9
:1017B000B5BE9C46994618460493FDF7AFBE00BFE0
:1017C000C827040804A0002011A000200007090E6B
:1017D000903B00200AA000202DE9F047B0F9085006
:1017E0000D81EDB2442D92B00C46174600F06B828D
:1017F000064642D9812D00F0A98200F29580542D31
:1018000000F0C88040F2F7816E2D00F02A82802D12
:1018100040F01181944B93F8009009F1020919F0FE
:10182000FF0900F09480914B914F924EDFF878A21F
:10183000994403F101080A2516E0322D01F01884BD
:10184000A5F13C00C0B2132841F21C840023226899
:10185000511C216015702268C84502F10101216008
:10186000137074D018F8015B0A2DE6D1BAF8003075
:10187000FF2BA8BFFF23DBB2E9E7052D00F01182A3
:101880001ED8022D7ED040F2A381032D00F0DD8111
:10189000042D40F0D0802A4677492046F9F720F8F9
:1018A00000212046F9F764F822680221531C012523
:1018B000236028462B461170638112B0BDE8F08783
:1018C000242D5DD040F23A81282D00F00482382D7D
:1018D00040F0B1800A68694B0125511C21601570E8
:1018E0002268052150192060117022680A215019C0
:1018F0002060117022680021501920601170226848
:101900001978501920601170226859785019206098
:10191000117022689978531923602B46117028465C
:10192000638112B0BDE8F087A02D17D040F2258169
:10193000B82D00F00982FE2D7DD1514D05F108062C
:1019400035F8021B2046F9F713F8AE42F8D101250D
:101950002B462846638112B0BDE8F087494B084604
:101960001968F8F7EDFF484B20461968F8F7E8FFCB
:10197000464B196820460125F8F7E2FF2B46E8E7B9
:10198000434BF6E70422434920460125F8F7A8FF18
:101990002B46C4E70B68404A404F581C1121206079
:1019A000197023681278591C21601A70236897F8FF
:1019B0005B20591C21601A70236897F85A20591C23
:1019C00021601A70B7F856102046F8F7D1FF0021B1
:1019D0002046F8F7CDFFB7F858102046F8F7C8FFB3
:1019E000BD1E07F1480635F8021F2046F8F7C0FF74
:1019F000AE42F8D122682A4B0C21501C20605D18A1
:101A00001170226813F8011F501C9D422060117054
:101A1000F7D123680222591C21601A70B7F85C10B4
:101A20002046F8F7A5FF0125B7F85E102046F8F725
:101A30009FFF2B4673E721462846FAF70DFE002844
:101A400085D1742D00F0F480772D2FD13368726822
:101A50009A421BBF5A1C326001461978114A20462F
:101A60002CF024FA73E700BFD93A00201C280408A0
:101A7000676666662C3F0020027C0020A9AF00202C
:101A8000FC3A0020107AFF1F147AFF1F187AFF1FFC
:101A9000ECB00020D05A04080C7C0020F4BE0020DA
:101AA0003DBF0020ADD10308543F0020F52D01F0CB
:101AB0001C83762D00F0DE8137687168A5F1210363
:101AC000CA1B3846362B00F21583DFE813F090026C
:101AD0001303130313031303130313031303E50285
:101AE0001303130313031303130313031303130346
:101AF00013031303130313031303130313035A02F0
:101B00001303130313031303130313031303130325
:101B10001303130313031303130313031303130315
:101B20001303130313031303130313031303130305
:101B30001303AF0213036A021303FA01202D7FF48B
:101B40007AAF0B68B64D591C6A7821601A70236809
:101B50002A78591C21601A702368AA78591C2160C0
:101B60001A7029892046F8F703FF23686A79591CFF
:101B700021601A702268A97998E6822D7FF45BAF04
:101B80000B68A84AA84D1178A54A581C2060197006
:101B900011892046F8F7ECFEA44B22681B88FF2B26
:101BA00002F10101A8BFFF2321601370A96881F32E
:101BB000100189B22046F8F7DBFE296801F30F0116
:101BC00089B22046F8F7D4FE994B226819786DE661
:101BD000012D7FF430AF0B680022591C21601A7070
:101BE00023685A1C22601D7022682421531C236024
:101BF0002B46117093E6522D7FF41DAF0A688D4B72
:101C0000501C0321206003F10C06117006200121F5
:101C10002268551C256011702268B34202F101014F
:101C20002160107000F0DA809979D8790633EFE7F7
:101C3000336872689A421BBF5A1C32600146197899
:101C40007D4A20462CF032F981E60B685A1C0A6066
:101C50001D700B680222591C21601A702268002135
:101C600024E6724B0A681B886F4DFF2BA8BFFF2329
:101C7000511C21601370A96881F3100189B22046BC
:101C8000F8F776FE6D4B20461988F8F771FE296843
:101C900001F30F0189B220460125F8F769FE2B46B2
:101CA0003DE60B2266492046F8F71AFE08226549F0
:101CB0002046F8F715FE0125072263492046F8F76C
:101CC0000FFE2B462BE6002A3FF441AE5F4B13601C
:101CD00001252B4623E60B68DFF894815C4E591CE6
:101CE000022221601A70236806275A1C22601F7086
:101CF00023680A22591C21601A70236801255A1989
:101D000022601D70B8F800102046F8F731FEB8F8D0
:101D100002102046F8F72CFE23685A1922601F7023
:101D200023685022591921601A702368002259191A
:101D300021601A7031882046F8F71AFE7188204613
:101D4000F8F716FE2B46EAE5424B12E6424B1E78A8
:101D5000033616F0FF063FF4FAAD404B404F1E44E9
:101D600003F101094FF00A0820E0B8F1500F01F02B
:101D70008681B8F1320F01F09B81A8F13C00C0B21E
:101D8000132841F299810025294623685A1C2260B4
:101D9000204683F80080F8F7EBFD29462046F8F747
:101DA000E7FDB1453FF4D3AD19F8018BB8F10A0F47
:101DB000DBD12C4B9D68196805EB85054FF6FF7349
:101DC0006D009D42A8BF1D469942A8BF194625EA4D
:101DD000E57521EAE171ADB289B2D6E7224B2168FF
:101DE0001A78481C20600A70002A3FF4B0AD013A0E
:101DF000D2B21E4902EB420201EB420292F82120CC
:101E0000002A3FF4A4AD0132D5180133226813F83B
:101E1000011F501CAB4220601170F7D197E500BF45
:101E2000003E0020D33B0020903B00209C3B002044
:101E300094BF00203C28040855DD03087CBF002027
:101E4000D85A0408E45A0408F05A040889C500085E
:101E5000143F002048360020D93A00202C280408DE
:101E6000243F0020E03E0020846A00201C28040853
:101E7000C068002033685A1C32601B78002B01F0C8
:101E8000B181102B07BF8F4A92E8220005462946F0
:101E90002268501C206013702046F8F751FD294637
:101EA0002046F8F74DFD884B20461968F8F748FDA5
:101EB00020460021F8F75CFD00212046F8F758FD88
:101EC000CCE67B1C336017F8378B0DF1070201332A
:101ED000336013F8011C02F8011F9F42F7D17B4ABF
:101EE0001378002BFCD1DFF8049299F80050002DF4
:101EF000FDD1DFF8FCA10126DAF8000089F80060C6
:101F0000F7F77AFE724B28461E702CF00DF9284622
:101F10002CF00AF909202CF007F940462CF004F9BE
:101F200002AF3D460DF13E08EE1BF6B20A202CF042
:101F3000FBF830462CF0F8F815F8016B0B202CF06C
:101F4000F3F830462CF0F0F80020F7F779FAA845BE
:101F5000EAD108202CF0E8F8A0202CF0E5F8A02029
:101F60002CF0E2F800202CF0DFF810F02006F6D17B
:101F7000DAF800000125F7F745FE89F800602B46E6
:101F8000CDE47B1C33603B780A2B01F07081304636
:101F9000F8F7A0FC3046F8F79DFC3046F8F79AFCBD
:101FA000D5E47B1C336097F80080B8F1FF0F01F097
:101FB0009B81B8F1FE0F01F047813046F8F77EFCB7
:101FC00096E80C009B1A002B07DD531C3360137836
:101FD0001BB9B8F10B0F41F27C81B8F1240F00F26C
:101FE00019833C4B012523F818002B4697E43B4608
:101FF0007A1C3260384D13F8022B6A7033607B789C
:102000002B70FB1C3360BB78AB703046F8F756FC86
:1020100033682881591C1A46316012F8021B697115
:1020200032605B78AB7101252B4678E47B1C336012
:102030003878032800F2EE82431E284D2849DBB28F
:1020400003EB430305EB4303087093F8215000288A
:102050003FF47DAC531EDBB2AB4240F0DB8200228A
:10206000C1F80620C1F802208A725BB1581C33689F
:1020700008444A1C0133336013F8011C02F8011FA5
:102080009042F7D1174B1B78002B3FF460AC012531
:102090001EF030FF2B4642E47B1C33603B780A2B5A
:1020A00001F0A580502B40F032823046F8F706FC54
:1020B0000D4F38803046F8F701FC012578802B461B
:1020C0002DE400BF582A0020502C0020554E00203F
:1020D0008A530020F4BE0020003E00201C28040883
:1020E000846A0020044E0020143F00208153002009
:1020F000F07B00200B3DEF2D00F28C8201A353F802
:1021000025F000BF3B3001081526010815260108FF
:1021100015260108152601081526010815260108AF
:10212000152601081526010815260108152601089F
:10213000152601081526010815260108152601088F
:10214000152601081526010815260108152601087F
:10215000152601081526010815260108152601086F
:1021600015260108EB2F010815260108D12F0108BB
:1021700015260108AF2F01081526010815260108AC
:10218000152601082B2E010815260108D12D01085E
:10219000152601089F2D010815260108792D010833
:1021A00015260108432F010815260108EF2E010806
:1021B00015260108A12E010815260108152601087B
:1021C00015260108152601084F19010815260108D2
:1021D000852E01081526010815260108552F01082E
:1021E00015260108C5240108152601081526010831
:1021F00015260108152601081526010815260108CF
:1022000015260108152601086F2F0108152601085B
:102210002B2D01081526010815260108EB2C0108B5
:10222000152601081526010815260108152601089E
:10223000152601081526010815260108AB2B0108F3
:1022400015260108772C0108152601083D2B0108E9
:1022500015260108712A010815260108492A0108D6
:102260002B2A010815260108152601081526010844
:10227000152601081526010815260108152601084E
:10228000152601081526010815260108152601083E
:10229000152601081526010815260108152601082E
:1022A000152601081526010815260108152601081E
:1022B000152601081526010815260108152601080E
:1022C00015260108152601081526010815260108FE
:1022D00015260108152601081526010815260108EE
:1022E00015260108152601081526010815260108DE
:1022F00015260108152601081526010815260108CE
:1023000015260108152601081526010815260108BD
:1023100015260108152601081526010815260108AD
:10232000152601081526010815260108152601089D
:10233000152601081526010815260108152601088D
:10234000152601081526010815260108152601087D
:10235000152601081526010815260108152601086D
:10236000152601081526010815260108152601085D
:10237000152601081526010815260108152601084D
:10238000152601081526010815260108152601083D
:10239000152601081526010815260108152601082D
:1023A000152601081526010815260108152601081D
:1023B00015260108012A010815260108EB29010844
:1023C00015260108152601081526010815260108FD
:1023D00015260108152601081526010815260108ED
:1023E00015260108152601081526010815260108DD
:1023F0001526010815260108912901083F29010821
:1024000007290108152601086B2801085128010831
:102410003528010815260108C1270108C926010829
:10242000A1260108152501084726010815260108DF
:1024300093270108152601081526010871270108B0
:10244000432701082F2701081F260108F725010847
:10245000D5250108A925010815260108152601081A
:10246000152601081526010815260108152601085C
:10247000152601081526010815260108152601084C
:10248000152601081526010815260108152601083C
:10249000152601088F2501081526010815260108B3
:1024A00037250108152601081526010815260108FB
:1024B000152601081526010815260108152601080C
:1024C0001F2501087B1C3360C44B3A78DFF8588322
:1024D0001A700023C8F800303046F8F7D7F9326890
:1024E000D8F80030BE49BF4D0343501CC8F8003037
:1024F000306013780B723046F8F7E0F92860304608
:10250000F8F7DCF968603046F8F7D8F9A86030468B
:10251000F8F7D4F93046F8F7D1F9FFF718BAB24B0B
:102520001B78DB0776D40125FBF776F9FCF71CF85E
:102530002B46FFF7F4B97B1C33603B780F2B69D82F
:10254000BA1C3260C3EBC303A84A7978D154F91C92
:1025500031601344BA785A703A1D3260FA789A7032
:102560007A1D32603A79DA70BA1D32607A791A715E
:10257000FA1D3260BA795A7107F108023260FA79AD
:102580009A71012522F0D2FB2B46FFF7C8B93046DD
:10259000F8F794F9964FF8813046F8F78FF901254E
:1025A000B8812B46FFF7BBB93A467B1C3360914B91
:1025B00012F8021B197032607A785A70FA1C326075
:1025C000BA789A703A1D3260FA78DA7001252B4693
:1025D000FFF7A5B93046F8F771F9874F38823046D2
:1025E000F8F76CF978823046F8F768F90125B88277
:1025F0002B46FFF794B93B467A1C326013F8020B66
:102600003360FB1C79783360BA7813F01BFB002829
:102610007FF49DA94FF0FF352B46FFF780B93B466D
:102620007A1C3260754A13F8021B11703360704ACD
:102630007B789370FB1C3360714BBA789A700125DC
:102640002B46FFF76CB90D2AE4D17B1C33603D7833
:10265000072DDFD8DFF8D48130460C27F8F72EF9A4
:1026600007FB05F708EB0705A8803046F8F726F9C1
:10267000E8803046F8F722F9336828811A46591C59
:10268000316012F8021BA97232605B78EB7230463F
:10269000F8F7FCF8012548F807002B46FFF73FB98B
:1026A0007B1C33603878060600F191864E4B1B7810
:1026B000DD073FF54CA9032828BF00200125FBF7C3
:1026C0008FF82B46FFF72BB97B1C3360304697F809
:1026D0000090F8F7DBF880463046F8F7D7F8054663
:1026E0003046F8F7D3F807463046F8F7E7F83046B3
:1026F000F8F7E4F83046F8F7EDF8B9F1000F00F01C
:102700007D86B9F1100F7FF422A93E4BC3F80080FB
:102710005D600FB13C4B1F603C493D4B0222081FDE
:1027200001251A7021F086FA2B46FFF7F8B8394BCD
:10273000394918684E2201252DF0D0FB2B46FFF7B2
:10274000EEB83A467B1C3360344B12F8021B19700A
:1027500032607A785A70FA1C3260BA789A703046D1
:10276000F8F7ACF82E4B0125D8802B46FFF7D7B8E9
:102770003046F8F7A3F82A4F38803046F8F79EF82D
:1027800078803046F8F79AF80125B8802B46FFF795
:10279000C6B8DFF89C8098F80030002B3FF4D7A82B
:1027A000204F00253046F8F789F823F003F898F811
:1027B0000030A7EC010A01359D42F3DBFFF7C7B8F3
:1027C000094B1B78D8073FF5C2A80125FBF7FEF897
:1027D000FBF7CAFE2B46FFF7A2B800BFF86800203F
:1027E0007C5D0020D84D0020593A002054A70020DD
:1027F000D068002090510020C4580020F45B0020D5
:10280000E0680020582A0020502C00205C2A00207C
:102810007E50002038390020884F0408C868002006
:10282000C8AD002020AD0020ECB000205CAE002040
:10283000D93A0020B34B1B78DA073FF588A8B24A93
:102840001378012543F0040313702B46FFF767B894
:10285000AC4B1B78D9073FF57AA8AC4B4FF4C87244
:1028600001251A802B46FFF75AB8092A7FF7D2AE06
:10287000DFF8C4823B467A1CD8F80050326013F867
:10288000022B2A7033607B78AB70FB1C3360BB7803
:10289000642BA8BF64233A1D6B713260FB78642BF4
:1028A000A8BF64237A1DAB7132603B79EB71BB1D0D
:1028B00033607B79642BA8BF6423FA1D2B723260CE
:1028C000BB79EB7007F108033360FB792B7130465D
:1028D000F7F7F4FF726833686881D11A00290CDDBC
:1028E000591CD8F800003160521A002A1978417238
:1028F00003DD9A1C32605B78437001252BF0F8FFF2
:102900002B46FFF70CB8824B1868FB1C0246213798
:10291000991E316013F8031C1170591E316013F8B1
:10292000021C5170336013F8011C917003339F42F5
:1029300002F10302ECD122F0E7FDFFF708B87B1C9F
:1029400033603B78704A002B00F06D85137843F0BC
:102950000203B91C13706F4D31607B782B753046C4
:10296000F7F794FF28603046F7F790FF686030462D
:10297000F7F7A4FF28813046F7F7A0FF664AE88101
:102980001378012543F0020313702B46FEF7C7BFEF
:10299000C2F34705122D3FF63DAEB5B112AB0DF1B6
:1029A000060903EB4507C846423F3046F7F786FF66
:1029B00028F8020F4745F8D1584B39F8022F23F871
:1029C000022FC845F9D1112D09D8554A6B00023B99
:1029D00013440021223223F8021F9A42FBD1514AAC
:1029E00001231D461370FEF79ABF4F4F0023304658
:1029F0003B60F7F74BFF012538602B46FEF78FBF92
:102A00003B467A1C326013F8025B3360FB1C78781B
:102A10003360B978002D00F04B85012D7EF497AF1F
:102A20000BF09CFB2B46FEF77ABF364B1B7813F05E
:102A300001017FF4EFAD7B1C3360387801250BF08A
:102A4000D1FA2B46FEF76BBF3B467A1C3260374A01
:102A500013F8021BD1703360354A7B785371FB1C2D
:102A60003360344BBA78DA7001252B46FEF757BF36
:102A70003046F7F723FF3046F7F720FF3046F7F7E9
:102A80001DFF3046F7F726FF3368214D1946581CC5
:102A90002A68306011F8020B82F82C0031605978F6
:102AA00082F83610D91C31609B7882F83730304676
:102AB000F7F710FF3046F7F70DFF3046F7F70AFF3C
:102AC00030462F68F7F7FAFE78873046D5F8008051
:102AD000F7F7F4FE37687368A8F83800DA1B012AA4
:102AE0000ADD7A1C2B6832603A7883F82E20304653
:102AF000F7F7F0FE37687368DB1B032B00F3728473
:102B0000286818E7593A0020183E002000CE00201F
:102B1000383900201C3E00207C5000206AC1002073
:102B20006CC1002068C1002048360020D068002019
:102B300050C10020E0680020E0CD00207B1C336005
:102B4000C44DDFF838833B7888F8053030462F686D
:102B5000F7F7B4FE38843046D5F80090F7F7AEFEAC
:102B600073683768A9F81E00DA1B072A00F3868409
:102B7000DA1B032A00F37484DB1B002B05DD7A1CAF
:102B80002B6832603A7883F82620FAF74FFE1AF065
:102B90009BFDB14B1B68002B00F0D68328680125F4
:102BA00022F058F92B46FEF7BABE3046F7F786FEFC
:102BB000054621F04DF9FF283EF4C9AE3F2D00F245
:102BC00037840DF14808002308F8403DEF084146DE
:102BD0000DF107008DF80730013721F019F99DF844
:102BE0000730FFB205F00705BB4205F1010503D12F
:102BF0009DF80830AB4203D02946384621F014F93D
:102C000033687268D21A012A7EF7A1AE5A1C12A844
:102C1000326000221D7800F8412D21F0EDF89DF87A
:102C20000730AB420AD08D4B1B683BB19A79AA4260
:102C300004D31B681B690BB12846984733685A1C9C
:102C40003260404600221D788DF8082021F0C8F837
:102C50009DF80830AB423EF47AAE804B1B68002BE7
:102C60003EF475AE1B685B69002B3EF470AE2846DF
:102C70009847FEF76CBE3B467A1C3260DFF8FC8159
:102C800013F8022B88F802203360754A7B781370A2
:102C9000FB1C3360734DBB782B713B1D3360FB789D
:102CA000092BA8BF09233046AB70F7F707FE37683A
:102CB00073682880DA1B012A05DD3046F7F7FEFD30
:102CC00037687368E881BB4240F04983FAF7AEFD8C
:102CD000336872689A423EF43AAE5A1C32601B78EE
:102CE000EB7001252B46FEF71ABE5F4B1B78012BBC
:102CF0003EF62DAE7B1C3A463360DFF8848112F835
:102D0000023B88F802303260FB1C78783360CB1AC3
:102D1000012BB97840F30C833046F7F7CFFD01253E
:102D2000A8F800002B46FEF7FABD7B1C336097F82D
:102D30000080B8F1110F3FF66DACBB1C33604B4DFA
:102D40007B7805F818303046F7F7B8FD40F6CA032F
:102D50009842A8BF184640F2EE23984205EB48017E
:102D6000B8BF18460125A0F2EE222B46192092FB8F
:102D7000F0F24A70FEF7D3BD7B1C33603D781F2D07
:102D80003FF648AC052A7FF445AC3046F7F77EFDA8
:102D9000374B43F8250019F07DFFFEF7D8BD344DC1
:102DA00005F140073046F7F789FD3368A5F8800044
:102DB000591C1A46316012F8021B85F882103260E5
:102DC0005B7885F883300435BD42EBD1FEF7BFBD9B
:102DD0007B1C284D33603B782B723046F7F76EFD35
:102DE000A8833046F7F76AFD28833046F7F766FD7B
:102DF000336868835A1C32601B78EB7473689A1AC4
:102E0000032A00F3C5823768DA1B052A00F3B08273
:102E1000DB1B002B7EF79BAD7B1C33603B7885F87A
:102E2000213001252B46FEF77ABD7B1C3360124A08
:102E300038781070C91A00297EF789ADBB1C336041
:102E40007B78003318BF0123012553702B46FEF712
:102E500066BD00BF38390020F468002034390020F6
:102E6000C4680020C4580020D7B00020F4340020EB
:102E7000BC3700207C5D0020F8680020F45B002057
:102E80005CBF00203B467A1C3260C54A13F8021B27
:102E9000917033607B78537001252B46FEF73FBD60
:102EA0000723B2FBF3F3C3EBC301521A7FF4B2ABB7
:102EB000DBB203F1FF395FFA89F9002B3EF447AD2D
:102EC000DFF8E0A209F101099046431C336090F954
:102ED0000020B44B002593F90210914203F108033E
:102EE00000F0D6810135042DF5D1FFF793BB7B1C93
:102EF00033603B780E2B3FF68DABBA1C326078788E
:102F000003283FF687ABA849062202FB03F28B1881
:102F1000FD1C58713560B87888543A1D3260FA78D3
:102F20005A707A1D32603A799A70BA1D32607A7995
:102F3000DA70FA1D3260BA791A7101252B46FEF754
:102F4000EEBC7B1C3360994B3A785A7501252B46B1
:102F5000FEF7E5BC964B03F10802791C3160397825
:102F600003F8011F9A423EF4F2AC3768F5E73B469E
:102F70007A1C904D326013F8022B2A7133607B78F3
:102F80006B713046F7F79AFC336828805A1C326020
:102F90001B78AB713046F7F791FC336868805A1C98
:102FA00032601B78EB7101252B46FEF7B8BC30462A
:102FB000F7F784FC804F38603046F7F77FFC786085
:102FC0003046F7F77BFC0125B8602B46FEF7A7BC1F
:102FD0007A4F00233B603046F7F758FC3B680125E9
:102FE00003433B602B46FEF79ABC7B1C33603D7865
:102FF000132D3FF60FABBB1C336078782AF090FF9F
:1030000000283FF407AB6E4B027803F82520FA1C2A
:10301000326003EB8503BA785A703A1D3260FA7851
:103020009A707A1D326067493A79DA70086801252A
:103030002BF0ECFB2B46FEF772BC634B102A4FF0D3
:10304000000128BF1022196059609960D960197475
:10305000002A3EF47CAC3168013B0A440131316006
:1030600011F8010C03F8010F8A42F7D1FEF76FBC8B
:103070003388FF2BA8BFFF23DBB2FEF7E8BB534B1F
:10308000FEF798BE14F0DCFC00283EF4DFAB0378BA
:103090000A2B28D8B0F9023087FB0312DB17C3EBE9
:1030A000A2039BB2FF2BA8BFFF23DBB2FEF7CFBB6F
:1030B00097E82200FEF780BE14F0C2FC00283EF420
:1030C00062AE03780A2B3EF65EAEB0F90430B0F97A
:1030D000061003EB830383F3500521EAE171ADB2DF
:1030E00089B2FEF752BE0023DFE7336872689A4266
:1030F00040F08380364BFF221A704FF00009354DA7
:103100000AF080FA49462022334885F800902FF0D3
:10311000FCF98DF808909DF80830072B00F2068125
:10312000DFF8BC802C4E4A469DF8083003EB430381
:1031300008EBC3035B7CE3B19DF8083003EB43036A
:1031400008EBC30320215B699BB19DF8083003EBBA
:10315000430308EBC303586946F82200F6F794FCD2
:103160002B7856F82300F6F74DFD2A780132D2B2BB
:103170002A709DF808300133DBB28DF808309DF8D5
:103180000830072BD0D92368591C21601A70002FF2
:103190003EF4DDAB114B3B6001252B46FEF7BFBB78
:1031A000EC680020187C0020543600207C5D002054
:1031B0007B5D0020E4AD0020D84D0020ECB0002065
:1031C000FC6800203839002020390020183F0020FA
:1031D00070280020A3C2002064C20020D5970308F5
:1031E00004580020B54A92E82200FEF751BE30464E
:1031F000F7F764FBB24FFEF75CBF5A1C194632600A
:10320000B04811F8022B027031605B784370042AD9
:1032100003D9FF2A7EF422AD6FE7AB4909789942C2
:1032200005D8022A7EF41AADFF2B7EF417AD236871
:1032300001255A1922601D70002F3EF488ABA34B64
:103240003B602B46FEF76BBBBB1C33607D78022DC9
:103250003FF6E0A93046F7F731FB9D4B03EB450302
:103260004FF0FF35A3F85C002B46FEF758BBBB1CA4
:103270003360984B7A781A70FA1C3260BA785A70B8
:103280003A1D3260FA789A7001252B46FEF747BB4B
:103290000AEBC5073046BA70F7F710FB33682AF817
:1032A00035001A46591C316012F8021BF970326061
:1032B0005A783A71DA1C32609A78BA71181D306007
:1032C00008F10108DB787B71C1457FF4FEADFEF7A4
:1032D0003EBB7F4B0030984418BF0120012588F881
:1032E0004A002B46FEF71BBBBB1C33607A4B7A7837
:1032F0001A70FB1C3360DFF8D881BB7888F85B302C
:103300003B1D3360FB7888F85A303046F7F7D6FA21
:10331000A8F856003046F7F7D1FA3046F7F7CEFA5C
:103320000125A8F858002B46FEF7F9BA4A462AE7C5
:103330006A4B1A88012512FB00F22B4692FBF1F230
:10334000A8F80020FEF7EBBA65486649664A674B65
:10335000036001250B6013602B46FEF7E0BA7B1C6F
:1033600033603B78003318BF012388F80730ADE4A1
:103370007B1C33603B78EB723046F7F787FA336893
:10338000E8605A1C32601B782B74376873683FE51D
:103390003046F7F793FAA8843046F7F78FFA376884
:1033A0007368E884DA1B032A7FF72EAD3B467A1C4C
:1033B000326013F8022BAA7733607B7885F82030CF
:1033C0003046F7F77BFA3768736868841CE500F0CD
:1033D0007F00032828BF002001250AF0DBFE2B46D2
:1033E000FEF79DBA30462F68F7F768FA78863046C0
:1033F0002E68F7F763FAB086FFF782BB2F4B1020D9
:10340000C3F800805D6027F091FD394A137843F0DE
:1034100001031370002F3EF49AAA364B01251F605A
:103420002B46FEF77CBA137803F0FD03FFF791BA41
:103430000DF10808404620F0C7FCBDF80830AB424B
:103440003FF4DEAB2C4B1B68002B3FF4D9AB1B6861
:103450009B69002B3FF4D4AB28469847FFF7D0BBBD
:103460003046F7F72BFAA8F80E003046F7F726FAA1
:1034700037687368A8F81000FFF77EBB3046F7F78F
:103480001DFAA8F80A003046F7F718FAA8F80C0059
:1034900030462F68F7F712FA78843046D5F8009056
:1034A000F7F70CFA37687368A9F82400FFF760BBD8
:1034B000012521F097FE2B46FEF731BAC0500020BF
:1034C000C068002070280020D93A002095C5000867
:1034D000F4BE0020A9AF00200C7C00204A67002029
:1034E00044A8002098A8002098AC00202987000854
:1034F000183E0020502C0020343900202DE9F047E0
:10350000C44B1C6862072DED028B03D4BDEC028B0B
:10351000BDE8F087C04D2B78002BF7D06E6846F2DF
:10352000A713861B9E42F1D9DFF850936860B9F863
:103530000070DFF84C83002F40F0A68198F8062039
:10354000AB689FEDB60ADFEDB60ADFF8F492013AF8
:10355000B3FBF2F307EE903AF8EE677AB7EE008A23
:1035600027EE800A2DF034F8DFEDAE7A38EE400A0F
:1035700020EE270A2CF0BCFEB8F80830DFEDAA6A6E
:1035800007EE103AEB68C01AB8EEC77A07EE900A59
:10359000A7EE668AB8EEE70AD9ED097AF8EEE77A7F
:1035A00020EE080A67EEA67AA7EE270A2CF0A0FE06
:1035B0009E4BC9F8240002461860A30740F1AA8177
:1035C000DFF8C0E29A4CDEED007A9FED9A5A21684E
:1035D000F8EE677A27EE855A002900F0BB81964BFA
:1035E00007EE101AD3ED026AB8EEC77AF8EEE66A73
:1035F00086EE878A914991ED004AB8F80C10D5ED16
:10360000054ADFED895A95ED066A67EE847A06EE83
:10361000901A67EE887A8A49B6EE004AF8EEE66AB2
:10362000F0EE643AE7EE843A66EEA56A91ED097A27
:103630007E49F7EE005A75EEE65AB8EEC77AA3EE69
:10364000856A77EEA47A27EE257AC5ED057AF0EE45
:10365000477AE6EE267ABDEEE77AC5ED067A81ED89
:10366000007A78490978122900F05B8100211960FD
:10367000596099602160CEF80010002F7FF446AFAA
:10368000E869EA61121A07EE102ADFED6F6A6F4BE4
:1036900007EE906AB8EEC77AF8EE677A27EE267AD8
:1036A00040F2DC52C7EE276A0A21FDEEE67A17EEF9
:1036B000900A9042A8BF10469842B8BF1846F7F744
:1036C000D1FAB8F80A309FED586AD5ED056A07EED1
:1036D000103AB8EEC77AF7EE007AE7EE467A05EED2
:1036E000900AF8EEE55A66EE866A67EEA57AE7EE8E
:1036F000267AB0EE670AC5ED057A2CF0F9FD0521B2
:103700000646F7F7AFFA524A5249B2F9004008604C
:1037100084EAE473A3EBE473B3F5487F74DAB2F997
:10372000022082EAE273A3EBE273B3F5487F6BDA1F
:10373000494B1B78002B40F01181484B3B4A1B68DA
:10374000126847489B1AB3F5FA7FA8BF4FF4FA7383
:103750009842B8BF18460A21F7F784FA414B1C6813
:10376000637A00FB03F00028B8BF7F30C211B2F5C6
:10377000967F3D4BA8BF4FF496729A42B8BF1A4647
:103780003A48E37E076895ED087ADFED396A911BC8
:1037900001FB03F3227F344E002B01FB0272B8BF02
:1037A0001F335B11B2F5C81F3249A8BF4FF4C812CE
:1037B000B3F5967FA8BF4FF496738A42B8BF0A4606
:1037C000617F026007EE901A37EE087AF8EEE77A2A
:1037D00027EE267AB34267EE877AB8BF3346002ACF
:1037E000B8BF02F5FF52FDEEE77AB8BF1F3203EB18
:1037F000623317EE902A962A6FF09501A8BF9622A1
:103800008A42ACBF9F1A5F1A1B4A85ED088A17606F
:103810007CE600BF143E0020742800200894253761
:10382000B1DC423ED048874A6F12833AF43D002013
:1038300030A60020BD37863520A60020E0AD002050
:10384000BC660020F83A00200024744924FAFFFFE7
:10385000F83D0020E83D0020582C0020502C00208E
:103860000CFEFFFF38390020D4FEFFFF482C00205B
:103870000000003B0000E7FF402C0020FECD0020B0
:1038800050C100202CA60020374998F806A00A68ED
:10389000AB689FED360ADFED360A002A0AF1FF3ADF
:1038A000B3FBFAF39246B8BF02F1070AA2EBEA02B1
:1038B00003EB020ABAF1000F5346B8BF0AF107033F
:1038C000DB1007EE903AF8EEE77AC1F800A027EE99
:1038D000800A2CF07DFEF7EE007A77EEC07A9FED3D
:1038E000257A2B6967EE877A9A4518BF07F1FF336F
:1038F000FDEEE77A14BF9FB200274FF00003C5ED3D
:10390000037A18BFC5F810A0A9F800706B61AB610D
:10391000002252E69FED188ADFF870E0174C184B32
:103920009FE695ED057AD5ED067ADFF864C020684C
:10393000996891FBF0F1BDEEC77AFDEEE77A17EEDC
:10394000100A17EE909AACF80200ACF80010ACF830
:1039500004908BE69FED088A094B4BE6094A0A4B17
:1039600012681C680CE700BF9800002008942537F7
:10397000B1DC423ED048874A0000000030A600205B
:1039800020A60020542C0020383900202CA600202E
:10399000FC3A00202DE9F843304B1B685B0701D44B
:1039A000BDE8F8832E4C2F4D94F82490B9F1010F07
:1039B00048D1EB69284698472B69284698472B6AD7
:1039C00004F12C0004F128019847274B276B9B79C1
:1039D000A668E06A07F101089845636B08BF84F8A0
:1039E000009003F1010208BF4FF00008032A1FD026
:1039F0001E49626394F8382041F82300FAB904EBB9
:103A0000870704EB8803F863DA6BAB89C4F830806E
:103A1000B61A30440022A06084F82420002BBFD0C6
:103A2000134A0A2B1268B8BF0A231361BDE8F88352
:103A30000E4B01229860002384F8382063631AF04B
:103A40005FFDDCE76B6928469847AB6928469847D5
:103A50000122EB8984F82420E0E700BF143E002017
:103A600074280020BC66002050C10020B05D0020FA
:103A700064C100202DE9F04F724B734A1C7893B05B
:103A800000F59C412031814606911160002C00F028
:103A900027856E4A1268904240F227826C4A6D492F
:103AA0001768DFF8E8B10492013C1C706A4C03917E
:103AB00007F48057002F40F02582039B5B7D002B8D
:103AC00040F09B84049B1B681D0400F17B87634BC3
:103AD0009945A37800F27383002B40F07383604B09
:103AE0000693049B1F6817F4805940F0FA83039BE8
:103AF000BBF906605B8B9E42B4BF00260126594B82
:103B00001B6813F0805300F00782069A127812F0B7
:103B1000010200F0088203985349408C91ED037A2A
:103B200007EE900AF8EEE77AB4EEE77AF1EE10FAD3
:103B300081F20F80002E40F0FD814C4D95F89C11D4
:103B4000002940F0F7814A484A49056895F82D5008
:103B500000200860486088604749002D40F0EB81F4
:103B60000D70002A40F0EC81444B1A78002A50D1A5
:103B70000399BBF900E04F8B898BBBF90200BE456E
:103B8000CCBF8025002545F040038E45A8BF2B46BD
:103B90009B0843F08005B842C8BF2B4643F0400560
:103BA0008842A8BF1D46BBF904E0BBF90600AD087A
:103BB00045F08003BE45C8BF1D4645F040038E4515
:103BC000A8BF2B469B0843F0800E284DB842C8BFC3
:103BD000734643F0400E95F89E718842B8BF734615
:103BE0009F4201F02F81A5F8A02185F8A221244948
:103BF00085F89E310F78002F01F0A0805F2B01F037
:103C000007816F2B00F0FD87069B1B78D90740F1D9
:103C1000BF87049B1B4A1B68059203F00403002B1B
:103C200040F04A850DF14008174D0023C8F80430D4
:103C300005F15009109340F6330A192740F28336F4
:103C400029E000BF58340020083000205434002000
:103C5000185C00207C5D0020F0380020404B4C00B8
:103C6000593A002098BF0020D43B0020742800203F
:103C700038390020A4660020DC2B0020F5C200208B
:103C80009C230020143E0020FC6800203CA400205F
:103C900004354D4520D0AA78EB789A4217FB026094
:103CA000F6D26978043117FB03623BF911305345B2
:103CB000A8BF5346B3F5617FB8BF4FF46173984214
:103CC000E6DA9A42E4DB29782429E1D84046043533
:103CD000F7F794F94D45DED1B04B98E803001F7813
:103CE000AF4B83E80300002F00F03C840121AC4877
:103CF000F7F794F9002840F09A81E378002B40F020
:103D00009681A84C23881DB225F00105AEB2B342BE
:103D1000268000F0B686A44D02270E204FF014092D
:103D20004FF0FF082F7085F8019085F8028026F08B
:103D3000CDFF39469A482688F7F770F9002841F0F8
:103D4000348026F002039BB2B34223800AD0964B04
:103D50001421FF2202250E201D7059709A7026F042
:103D6000B5FF2688914BDFF884A21978DAF80400B1
:103D70000393B50708BF81F00201C1F34001F5F7D5
:103D8000BDFF24218648F7F749F930B9069A137820
:103D9000590744BF23F004031370059B1B6813F0FD
:103DA0000A0F1DD005217E48F7F738F9002800F0EA
:103DB0009D8625886F0740F19E8779480621F7F791
:103DC0002DF9002800F07F866E0640F18C870721D0
:103DD0007348F7F723F9002840F03083059B1B68F0
:103DE000980600F13B8326886D480C21F7F716F9F9
:103DF000002800F0388146F48073B342238009D054
:103E0000694B02251421FF220E201D7059709A70F3
:103E100026F05CFF664B1B78082B00F030810E2BE0
:103E200000F02D81049B1B685E0544D5614B1B7916
:103E3000002B00F0E18014215948F7F7EFF8002833
:103E400040F0DF8024F09EFA012026F08DFE90B332
:103E5000DFF89C8100254FF0CC0902E0DDB2022D95
:103E600029D809FB05F76B1C58F80760002EF5D11F
:103E7000C378514A90F9020052F823300196032288
:103E800000920121324626F05BF8034605EB45001F
:103E900000EB0010049353B1314608EB8000CC22B4
:103EA0002EF033FB049B48F807300135EDB21DF0CE
:103EB000F9FB0028D3D1069B1B78DD0740F1F28087
:103EC0003E493F4A01230B701370039BDAF8000050
:103ED000197801F00101F5F711FF059B1B685A07DE
:103EE00000F1508113B0BDE8F08F364B364A1F68A1
:103EF000049307F480570392DFF8F8B0334C002F97
:103F00003FF4DBAD00212648F7F788F800287FF45E
:103F1000D4AD09F011FDD0E578023FF5F6AD069A73
:103F2000127802F001022A4D002185F89C11002E22
:103F30003FF409AE274901200870002A3FF414AE6F
:103F4000F9067FF511AE244A1278D2063FF50CAE81
:103F5000B9F1000F7FF408AE002B7FF405AE7B02B1
:103F60003FF502AE1D4B1B78002B01F009841C4B62
:103F70009B78002E41F041843BB11A4A1A4B1268DB
:103F80001B689B1A002BC1F273841020104D26F081
:103F90009DFE012385F89D31E6E500BF805300209A
:103FA00098BF0020E838002070370020ACCD0020FA
:103FB000F8680020703B0020105704085A3A00208F
:103FC000642C0020185C00207C5D0020F03800206C
:103FD00074280020DC2B0020183E00209C230020A9
:103FE000EC68002004C40020F02D0020B0CD00209B
:103FF0002CA000203CA40020069B1B78D8077FF54E
:1040000021AF3C201AF064FD00283FF454AF17F0B4
:1040100077F93C201AF0C6FC00283FF44CAF17F0AB
:104020006FF93C201AF0BEFC0028F0D143E7059B55
:104030001B689A077FF565AEBF4C2688F3073FF5EE
:1040400080AE46F001039E4223803FF47AAEBB4B24
:104050001421FF2202250E201D7059709A7026F03F
:1040600035FE26886DE626F480739BB2B34223802A
:104070007FF4C6AEB24B1B78082B7FF4D0AE2288FB
:1040800022F040039BB29A4223803FF4CBAEAB4B6D
:1040900002251421FF220E201D7059709A7026F0FF
:1040A00015FEBFE6A74B93F80090B9F1000F5FD162
:1040B000DFF8E482A44F18F8030C3E794146A8F1DA
:1040C00003052AF073FB002800F0F283002E40F075
:1040D000448405F1080168792AF068FB002841F062
:1040E000D1819A49A87A2AF061FB002800F0F38375
:1040F000022E41F0CB819649E87B2AF057FB00283D
:1041000041F0C8819349287D2AF050FB002800F037
:10411000F383042E41F0C2818F49687E2AF046FB6A
:10412000002841F0BF818D49A87F2AF03FFB00287D
:1041300000F0F383062E41F0A181894995F8230010
:104140002AF034FB002840F04787864995F828007C
:104150002AF02CFB002800F0F383082E40F026877D
:10416000814995F82D002AF021FB002840F0F383C7
:104170007E4B01221A702AF09CFD059B1B685A0792
:104180007FF5B0AE03202AF03BFB002800F05586F7
:10419000238813F008047FF4A5AE082026F0DEFE85
:1041A0007348744D7449754A754BBBF806600068D6
:1041B0002E80086014601C6013B0BDE8F08F0BB94E
:1041C0000123A3706F4B06931B201F7894F8216086
:1041D0002AF016FB012E07F00109824600F0148632
:1041E00007F00203059394F82030DFF8B081664DA4
:1041F000052B69D8DFE813F05B004F000600DC00F8
:10420000FF008D00012E04BF052384F82030B9F192
:10421000000F00F05281039B5C4FB3F91810B8F8FF
:104220000030002261F30F0263F31F42002361F3A9
:104230000F0361F31F43CBF8042039686269CBF8A0
:1042400000308A42C0F06C84012E41F0E6820322E5
:1042500094F820300592CBE72AF0FEFA012807D126
:104260004A4FB8F802303A68642101FB0323236106
:10427000BAF1000F04D098F80630002B40F090807F
:10428000012E21D0414F22693B689A42C0F020861E
:10429000012384F82030012E3BD098F80730012B01
:1042A00000F0148121F0B2FF94F82030A0E7B9F1BA
:1042B000000FD1D14FF48060BAF1000F00F0FF83FE
:1042C00026F04CFE00232361059B002B3FF409AC34
:1042D000059826F0FBFC049B1F6817F480593FF4F7
:1042E00006AC1D212A48F6F799FE00287FF4FFABA3
:1042F000284A039BD2881B8BBBF90660991A8E4211
:1043000040F3F08513449E42B4BF00260126FFF718
:10431000F6BB1E4F3A68B8F80230642101FB032354
:104320004FF480600022236184F82020E27026F0A0
:10433000FDFD94F820305BE7E8380020703700205E
:10434000F86800205A3A00209800002048370020E2
:104350004D37002052370020573700205C370020AF
:1043600061370020663700206B370020642C002066
:10437000F43D0020442C0020502C0020482C00202C
:10438000402C0020593A0020A0BF002004C4002087
:1043900098BF0020C8AD00203E370020E4AD0020CB
:1043A00021F034FF03224FF47A7384F82020E36174
:1043B000A74F2B8843F002032B8009F0BDFA3A681F
:1043C000E36913440422A36184F82020012E40F005
:1043D0008C853B68A2699A42BFF476AF9D4B1878F2
:1043E00020B92AF00DFA00287FF46EAF2B8823F055
:1043F00002032B808EE7964FE8E7039A013BD27DBC
:104400003BF91330002A40F08683A3F57A73B3F5A5
:104410007A7FA8BF4FF47A7323EAE37307EE903AEA
:104420009FED8D7AF8EEE77A67EE877A8B4AFCEE9D
:10443000E77A17EE903A1380FFF749BB884B894A19
:10444000B3F90430884982FB0302DB17C3EBA202F5
:10445000059B0A801B6898067FF5C5AC834B1B78CB
:10446000990704D5824F3B7D042B00F244852688B2
:1044700016F0300F3FF4B8AC102026F057FD202086
:1044800026F054FD7B4B268800221A707A4A7B481E
:104490007B4F7C4D002111607B4A396000232960ED
:1044A00041608161036083604361C3611360516057
:1044B000936053619161D36196E4654F3B6847F225
:1044C00030520323E26184F8203072E721F09EFE2F
:1044D000032240F6B83384F82020E3615C4F68E79C
:1044E0006A4F3B78002B00F08087694BDFF8B4817E
:1044F000DFF8B4B1DFF8B4A1039345465E460490FB
:1045000099460EE019F804109847032C28DC88B966
:104510003B782AF8020F01349C4205F1040580F231
:10452000EF80072CE1B23046DBF80430EADD984733
:1045300000B2EDE738F824206B88801A4FF47A71C6
:104540009B1A01FB00F040F6CA0290FBF3F008440E
:10455000904240F2EE23A8BF10469842B8BF1846DA
:1045600000B2D5E7DFF848A1DFF84881494D0AF1EC
:104570005A064FF0010951461AF8010C2AF016F9B3
:10458000F8B19AF804009AF802309AF803E000EBC8
:10459000400105EB8101013BD1F8B02103EB43035E
:1045A000434493420DD095F8DC2181F8ACE109FA3F
:1045B00000F022EA0000C1F8B031C1F8B47185F80A
:1045C000DC010AF1060A5645D5D13349204A334B5E
:1045D000334D09681B78D2F8009008910793A5F530
:1045E000D67A00266B685BB31F784FB3AA68A9EB35
:1045F0000202002A0ADB9AF8DC210121B14022EAFA
:10460000010209F5FA718AF8DC21A960079ABAB1AA
:104610002A7859780432D2B2002940F0A082039956
:104620003BF91220098B01F1C800824240F3228439
:104630009AF8DC119A7841FA06F3D80740F1B18470
:104640000136042E05F10C05CCD1FFF74FBB00BF9E
:1046500004C400209C230020AAF1823F7CBF0020DC
:10466000F83D002067666666382C0020183E002062
:104670001C3E00207E500020705100202051002060
:10468000B02B0020C02C002048510020AC3400206A
:104690007C5D002074280020E0CD0020B938002087
:1046A000202A0020C034002038A500206E290020D8
:1046B0005536002050280408A94D95F8A63153B16D
:1046C000069B1B78DE0706D5039BBBF906205B8B98
:1046D0009A4200F33C841121A248F6F79FFC00287F
:1046E00000F0258295F8AA312BB995F8A43113B9B9
:1046F0003223A5F8A831012385F8AA31FFF792BA31
:10470000DDF81090984A04921146984A0968A2FB75
:10471000092A42F201020A404FEA9A1A059200F071
:104720000282934D9348944C944A95F800E00078A7
:1047300084F800E01070BEF1000F04D08F4A92F8A8
:1047400000E08EF0010E864D0F2085F82001002B31
:1047500000F001838A4B039E0B931B78B6F826C0AA
:104760000A931C463B78B78C039E864A368B0E967E
:104770002646A2FB0442520802EB4202B21AD2B20F
:10478000CDF820C001F48051079295F82181DFF81F
:1047900010B2DFF82CC209900AF5967276460F9196
:1047A00005F592740020CDF830900D959646002EB8
:1047B00000F03C82744A32F910201FFA82F9B945A0
:1047C0004FEA400103D3089DA94540F273825CF88B
:1047D0002020924580F033823BF90120059D002D79
:1047E00040F04782013098422BF8012004F1060482
:1047F000DDDB09980D9D654ADDF8309085F8218153
:104800000F280CBF0121002185F82001117000F054
:10481000A9825F4C5F4E604F35883868A168626836
:10482000E06045F00405401A9042524F3580534DE8
:104830004FF0010188BF00223970297088BF84F8C9
:104840002120002B00F0A082049A03991768534E90
:10485000B1F824C0B1F818E0514817F48057354634
:1048600040F0B48239460EE06A7802EB820202EB35
:10487000820202F2EE2292B201318B4220F8022B28
:1048800005F102050ED016F81120002A00F015825D
:10489000022AE9D00131028820F8022B8B4205F16F
:1048A0000205F0D10B9A137801331370FFF702B9A8
:1048B00008F10501687929F079FF00283FF411AC6F
:1048C000012E40F0DF8505F10D01A87A29F06EFF79
:1048D000002840F0DB853349E87B29F067FF00289A
:1048E0003FF410AC032E40F0D5852F49287D29F0E8
:1048F0005DFF002840F0D2852C49687E29F056FFE4
:1049000000283FF410AC052E40F0CC852849A87F44
:1049100029F04CFF002840F0B185264995F8230086
:1049200029F044FF00283FF410AC072E40F05483D8
:10493000214995F8280029F039FF002840F03683F6
:104940001E4995F82D0029F031FF00283FF410ACE6
:10495000092E3FF40DAC4FF009094B4629E300BF87
:104960007428002098BF0020185C0020D34D6210EE
:10497000E42F0020A8000020B9380020A900002062
:1049800059340020ABAAAAAA7029002036A500201D
:10499000F0380020A0BF002004C40020F434002020
:1049A0003CA400204D37002052370020573700200C
:1049B0005C37002061370020663700206B3700200D
:1049C0005C340020D04DD5F88431A9EB0303002BD3
:1049D000FFF67DA8CD4A95F88831517C069AC5F836
:1049E00084210133CA4A039E32F81120B17D03F0BD
:1049F0000F0385F888312B4492B292FBF1F283F8D1
:104A00008C2195F88C1195F88D2195F88E3195F8BB
:104A100098010A4495F88F11134495F89021194490
:104A200095F891310A4495F89211134495F8932121
:104A3000194495F894310A4495F89511134495F862
:104A40009621194495F897310A44134495F8991121
:104A500095F89B21184495F89A3101440B441A4467
:104A600042F30B12642AF17DA8BF642213B209B18C
:104A7000C2F1640307EE903A9FEDA67AF8EEE77A6A
:104A8000D2E40221A448F6F7C9FA00283FF459A954
:104A90002580B7073FF566A946F00203B34223809D
:104AA0003FF460A99D4B02201421FF2218700E20B4
:104AB00059709A7026F00AF92688FFF753B926F044
:104AC00035FAFFF7FFBB25F040039BB2AB422380D2
:104AD0003FF47DA9914B02251421FF220E201D7069
:104AE00059709A7026F0F2F8FFF771B9238823F015
:104AF0000405ADB2AB4225803FF45FA9874B022588
:104B00001421FF220E201D7059709A7026F0DEF8D5
:104B10002588FFF752B9C3F53B6308331BB274E431
:104B200003230593CBE47E4A92F800E003E695F870
:104B3000A431002B3FF476A8069B1B7813F00103E9
:104B40007FF470A8012285F8A43185F8A521FFF72C
:104B500069B86D4D012185F89C11FFF7EBB901296A
:104B600000F0E5839AF8DC210123B34001361343BA
:104B7000042E8AF8DC3105F10C057FF433ADFFF724
:104B8000B5B8069B674A1B781060DF0700F1ED811E
:104B900095F8A21100297FF43CA8B5F9A031322B79
:104BA0007FF737A895F89E210120572A85F8A201A2
:104BB00000F07C84049B1B6813F0040302D05A2A83
:104BC00000F0CB855D2A00F0C9845B2A00F00985DE
:104BD0005E2A00F05085562A00F0B085972A00F032
:104BE0006B85A72A40F081844F49049B0A781B6893
:104BF00042F004020A704D4A059203F00403FFF7E5
:104C00000EB8B2F5FA7FFFF604A895F8A221002AA3
:104C10007EF4FFAF069B1B780121D80785F8A2110F
:104C200000F1A78407F0EAFFFEF7F3BF002F3FD0A3
:104C30005CF8202092454FEA4001FFF4CDAD3C4A9C
:104C40003B4D525C05EB0109002A00F0A280022ACC
:104C500046D199F8012002EB820202EB820202F2B5
:104C6000EE2292B2032832DD059D12B2002D3FF4F0
:104C7000B9AD079D24F81520B8F1000F03D10A9DA6
:104C8000022D7FF6AFAD2288B4F80290B4F804800C
:104C90004A449044274A0FFA88F882FB0852264D6E
:104CA000A2EBE87225F8018012B24FF0010899E5F5
:104CB0003A4641004CF820E090E5CAB2022A04D9F5
:104CC000032A7FF4E7AD6246D6E57246D4E50125B6
:104CD00005FA00F9099D25EA090512B209957DE555
:104CE0003BF80120BEE745F04003AB4223807FF450
:104CF000F1AEFFF76CB845F004039D4223807FF4CA
:104D0000FDAEFFF75AB800BF742800203C6A0020AF
:104D1000586A002014AE234198BF0020703700204D
:104D2000B9380020F42D0020183E0020143E002049
:104D3000F434002056555555E02900203946BF4827
:104D4000F6F76CF900283FF41CAF85F8A37107F063
:104D500055FFFEF759BFBA49BA4A0B91DFF808B3BD
:104D6000012111701B21B5480593F6F757F9059BF2
:104D700000287FF44EADB44CB44FE2683B68A360AA
:104D80009B1AC82B00F25383049B1F6807F48057BB
:104D900088E5C2B2022A40F2C882032AA0D10E9A44
:104DA0000F9D002D08BF3A465CE726F001039BB239
:104DB000B34223803FF46DAE0E202F7085F8019032
:104DC00085F8028025F082FF268862E600210FE048
:104DD0006A7802EB820202EB820202F2EE2292B2C7
:104DE0000131994220F8022B05F102053FF45AAD3A
:104DF00016F811201AB1022AEAD00288F0E7CAB2E6
:104E0000032AFAD87246EBE700230593FFF7EBB9C4
:104E1000B2F5FA7FFEF6FDAE95F8A231002B7EF4D6
:104E2000F8AE069B1B7801210B4085F8A21100F01B
:104E3000E08208F081FDFEF7ECBE082026F076F84F
:104E4000FFF750B8824A83491068B5F9A021C769B5
:104E500081FB07018911FF17781A00F5FF407F30A9
:104E600082423EF7C4AEC91B0A4412B2A5F8A02183
:104E7000FEF7BDBEC8398A425CDA9AF8DC119A782E
:104E800041FA06F3D9073FF5DBAB52420120099204
:104E900026F034F87B1E099A162B00F23B81DFE8DE
:104EA00013F0DC01F201C3011B0208022F0296017C
:104EB00081016A0153013C0139011B0229012F02C2
:104EC000960181011301FD00E700AB01B5009F00D1
:104ED00021F09CF9032240F6B83384F82020E361E6
:104EE000FFF767BA0126FEF70ABE3A68E369134482
:104EF000A361FFF7E9B90A2029F082FC26888046E1
:104F0000002800F05182F20640F13D83524D95F8A1
:104F1000EC81B8F1000F7EF467AF0D2025F0D6FECE
:104F2000012385F8EC312688B8F1000F7FF4AEAA92
:104F3000FEF75ABF9AF8DC310122B24023EA02039D
:104F400009F5FA728AF8DC31AA60FFF779BB002113
:104F50003A48F6F763F800287FF4BDAB322385F8B2
:104F6000A601A5F8A831FFF7B6BB3C4B1B78002B78
:104F70003EF44FAEE378002B7EF44BAE95F8A331B0
:104F80000133DBB2032B85F8A3317EF642AE344BFE
:104F90005B7813B9002E7EF43CAE08F0CDFCFEF732
:104FA00033BE002A0CBF0120022070E74FF0080931
:104FB0004B4603EB83031D4487F80490A978687877
:104FC0001EF032FF069B274A1B7801211170D9077A
:104FD0007FF5D1A8FEF779BF4FF007094B46E8E708
:104FE000DAF8E001DFF8848090F8361098F80230A3
:104FF00011446429A8BF642121EAE17180F83610C8
:10500000002B40F0658420F07FFAABE5DAF8E00190
:10501000DFF8588090F8371098F802301144FE29D4
:10502000A8BFFE2121EAE17180F83710002BEAD0F9
:10503000162029F043FCDAF8E001E4E798BF0020ED
:105040005934002036A50020F038002004C4002088
:1050500064C10020D34D621074280020B9380020AC
:10506000EC680020642C00203CA400205CBF0020E1
:10507000DAF8E001DFF8C08681781144C829A8BFBA
:10508000C82121EAE171817098F80230002BBAD072
:10509000142029F013FCDAF8E001B4E7DAF8E001B3
:1050A000DFF8948641781144C829A8BFC82121EAB5
:1050B000E171417098F80230002BA4D0132029F040
:1050C000FDFBDAF8E0019EE7DAF8E001DFF8688638
:1050D00001781144C829A8BFC82121EAE1710170F3
:1050E00098F80230002B8ED0122029F0E7FBDAF876
:1050F000E00188E7DFF84086089898F802304179A7
:1051000011446429A8BF642121EAE1714171002B97
:1051100040F09383DAF8E00175E7DAF8E001DFF8B0
:105120001886017A98F802301144C829A8BFC8210E
:1051300021EAE1710172002B3FF465AF0B2029F0E9
:10514000BDFBDAF8E0015EE7DAF8E001DFF8E885B8
:10515000C17998F802301144C829A8BFC82121EAB2
:10516000E171C171002B3FF44EAF0A2029F0A6FB7C
:10517000DAF8E00147E7DAF8E001DFF8BC85817989
:1051800098F802301144C829A8BFC82121EAE1716A
:105190008171002B3FF437AF092029F08FFBDAF83B
:1051A000E00130E7DAF8E001DFF88C85417998F822
:1051B00002301144C829A8BFC82121EAE171417118
:1051C000002B40F04183112F7FF456AF1BE7DAF834
:1051D000E001DFF86485017998F802301144C829AC
:1051E000A8BFC82121EAE1710171002B40F074834E
:1051F000102F7FF457AF06E70898DFF83C85417819
:105200001144B1F5967FA8BF4FF4967121EAE17180
:10521000417098F80230002B3FF47CAF152029F044
:105220004DFBDAF8E001EEE60899DFF80C850F791E
:105230001744642FA8BF642727EAE7770F7129F086
:1052400057FB98F80230002B3FF464AF0320394637
:1052500029F034FBDAF8E001D5E60898DFF8D884C5
:1052600001781144FA29A8BFFA2121EAE1710170FD
:1052700098F80230002B3FF44DAF012029F01EFBBF
:10528000DAF8E001BFE60898DFF8AC8481781144D1
:105290006429A8BF642121EAE171817098F8023085
:1052A000002B3FF437AF022029F008FBDAF8E001C9
:1052B000A9E60898DFF88084C17998F80230114493
:1052C00081F30801C171002B3FF424AF052029F0C0
:1052D000F5FADAF8E00196E6089BDFF85C84997944
:1052E00098F8020011446429A8BF642121EAE17101
:1052F0009971002840F0B0820D2F7FF4FDAE09E7D0
:10530000DAF8E001DFF83084C17898F8023011440F
:10531000C829A8BFC82121EAE171C170002B40F063
:1053200084820F2F7FF4D4AE6DE60E9A9AE43BF997
:1053300012209978B2F5617F4FF4966393FBF1F3F5
:105340004ADB40F633019142A8BF11460C2FA1F56C
:10535000617191FBF3F100F08481182F7FF402ACAE
:10536000C9B2C8290B46A8BFC823DAF8E001C27D3C
:10537000DFB297423FF4F6AB9A1ADFF8BC83C775E9
:1053800048BF0732D71098F802300137FFB23BB957
:10539000002F3FF4E7AB384625F0B0FDFFF7E2BB46
:1053A000182029F08BFAF3E7F30600F150810B2067
:1053B00029F026FA002840F01881B70600F1538141
:1053C000C34D95F8EC31002B3FF4A7ADB8F1000FB9
:1053D0007FF45CA8FEF708BD0C2F00F0EA80182FC0
:1053E0007FF4C0AB00210B46BFE7BA4A0392FFF738
:1053F00089B9B949096811F4003140F040810B4680
:10540000B648C65C0F2E03F10C031ED001311529DE
:10541000F7D1049BB2491B680591FA3AA5F8A0217F
:10542000002203F0040385F8A221FEF7F8BBAD4A81
:10543000049B1F68138823F004031380012307F4DF
:10544000805784F82130FFF72DBAA74ED6F800E038
:105450004B00BEF1000F07D05F1800EB87079EF8E6
:1054600001E07F787745D4D20B44A04FA04900EBF0
:105470008300002330603B800B60CAE74FF00609D1
:105480004B4696E54FF001094B4692E54FF0020975
:105490004B468EE54FF003094B468AE54FF0040971
:1054A0004B4686E54FF005094B4682E5914B924904
:1054B0001A684FF47A73B3FBF2F3C3EB431203EBB6
:1054C0008203049A1268DB001206A1F8B43000F1DE
:1054D000E680834B05931B685F0700F1D780049B30
:1054E0001B6803F00403FEF79ABB0021BB2A10914E
:1054F00000F08081B72A00F07981BE2A00F0748123
:10550000BD2A00F04D81792A00F0DB817A2A00F073
:10551000D1819E2A00F0C8819D2A00F0BE81AE2A6A
:1055200000F00182AD2A00F0F781EF2A00F0EE8151
:10553000FD2A00F0E581FB2A00F0DC81FE2A00F064
:10554000D381F72A00F08E817B2A7EF462AB4FF480
:10555000FA61022008F046FDFEF75BBB674B0022B4
:105560000120674D67492A700B6025F0C7FCFEF7E4
:1055700050BB049B64491B680A60594A059203F0BA
:105580000403FEF74CBB102025F0E8FC202025F09A
:10559000CDFC5E494E4D081F1EF04CFB5C4B0222B9
:1055A0001A7095F8EC31002B00F03B812688FEF74D
:1055B0006DBF00273946524B09915B78BB423FF4DF
:1055C000D1AADFF87481384608F0E4FD98F802307B
:1055D00009991BB1C9B20C2029F070F90137FFB24B
:1055E000D6E64C4B01220220BBE74B4A4B4B52897B
:1055F00093ED007A07EE902AF8EEE77AB0EEC77ADC
:10560000B4EEE77AF1EE10FA7FF5D7AE93ED017ABA
:10561000B0EEC77AF4EEC77AF1EE10FA7FF7CDAEAE
:10562000B3063FF5CDAE202025F098FC284D97E835
:105630000C0005F5F47105F5F270C5F8E421C5F824
:10564000E8311EF0F7FA324B01221A70A9E7102058
:1056500025F06CFC2E4B268883F800804FF0010863
:10566000A5E6CFB2A7E7202025F060FC284B184D17
:1056700000221A7095E72A4B0222032071E729497C
:105680000978032900F0C4801946B9E6049B264A2C
:105690001B680A21118003F00403FEF7C0BA234BF4
:1056A0001B789B077FF515AF214B1B7D042B7FF6E5
:1056B00010AF1EF049FA0CE7049B1E4A1B684FF41A
:1056C000C8711180064A059203F00403FEF7A7BAD9
:1056D000742800207C5D0020483600206C3E0408C1
:1056E000143E0020A0BF0020882B0020262C002084
:1056F000282C0020085C00203CC40020BEAF002005
:10570000FC7B002038390020F42D0020C4500020FC
:105710007E5000200CB0002014510020D43B00200B
:105720005AB0002094BF0020FECD0020183E00207B
:105730001C3E002000CE00205CBF00200CF0C2F810
:10574000F4F7B2FE0CF0A6F8F8F70EFF012025F0F2
:10575000D5FB95F89E21FFF741BA95F8A421002AC0
:1057600040F0938095F8A63183F0010385F8A631C7
:10577000002B40F085800C2025F0A8FAFEF749BAEE
:10578000002E3EF402AC6B4D95F89D31002B3EF49B
:10579000EBA925F07FFA002385F89D31FEF7E4B9E7
:1057A0004FF6FE73644A654896890590D089334464
:1057B00001449381D1810CF085F8F4F775FE0CF06B
:1057C00069F8F8F7D1FE012025F098FB049BB5F8A5
:1057D000A0211B68FA3A0021A5F8A02103F00403D8
:1057E00085F8A211FEF71BBA0223DBE70B464FF642
:1057F000FE71D7E70B460221D4E7002BC3D05049F6
:10580000504A09684FF47A7000FB03131360BAE73B
:1058100025F040FAB5F9A021FBE503230593FEF737
:1058200057BD4FF00108FFF778BB0F20099229F010
:1058300045F8DAF8E001099A73E50E2029F03EF800
:10584000DAF8E001FFF7DFBB1120099229F036F802
:10585000DAF8E001099AB6E40D20099229F02EF851
:10586000099A49E50021042008F0BCFBFEF7D1B9F4
:10587000304D08F061F8002385F89D31FEF774B9CA
:105880000B2025F023FAFEF7C4B92C4A85F8A411A1
:1058900085F8A5010592FEF7C2B90021FF202AF084
:1058A000C1FA95F89E213AE601202AF0BBFA95F854
:1058B0009E2131E6244A137A43F001031372FEF766
:1058C000A8B9214A137A23F001031372FEF7A1B994
:1058D000172028F0F3FF1DE41020099228F0EEFFB6
:1058E000DAF8E001099A83E40021032008F07AFB4A
:1058F000FEF78FB90021022008F074FBFEF789B98A
:105900000021012008F06EFBFEF783B90021084654
:1059100008F068FBFEF77DB9FF2100202AF082FA2B
:1059200095F89E2101E6012100202AF07BFA95F8E6
:105930009E21F7E574280020D0680020143E002046
:1059400004C40020F02D0020D05700202DE9F04F96
:105950002DED0A8B484B1B7893B0012B039001F07F
:105960002480464C94F80021002A41F02C80072B1B
:1059700001F033804FF0000ADFF810B1DBF804309B
:1059800058469847002800F0D680BBF8B470002233
:105990008BF85520002F41F03982DBF84C30BBF9F1
:1059A0004060BBF93C70DBF82410BBF93E50DBF8DB
:1059B0002820A6EB030E8EEAEE70791AA0EBEE70AB
:1059C000AA1ACBF830102E49CBF83420B0F5804F0E
:1059D000DBF82C200191D8BF33460D46A3EB020320
:1059E0009BF856102748D8BFCBF84C60CBF838301E
:1059F0000BF048FD2B68990040F13787DBED0D5A1D
:105A0000DBED0C7A204A94ED416AD4ED426A94EDC4
:105A1000437AD4F810311268B8EEE58ADBED0E5AFD
:105A2000F8EEE77AF8EEE58A013377EE867A38EE1B
:105A3000268A78EE878A9342C4ED417A84ED428AC1
:105A4000C4ED438AC4F8103101F029870A4B1F784E
:105A5000142F02F05E850023D4F818510293062D0E
:105A600000F2F686DFE815F0C913671205128C12F2
:105A70006006F712C61300BFF83A0020642A00201F
:105A8000185C00206CC40020AC3000203CC4002016
:105A9000D24D0294DFF8B083DFF8B093019C05F299
:105AA000DC670026CE4BDBED087A1B78172B01F064
:105AB000D38095ED007AB8EEC78A082B28EE278AA6
:105AC00007D1B0EE480A01932AF012FC019B29F895
:105AD0001600226892000BD5002E04F0AB81B0EEC8
:105AE000480ADBF8783707F170009847B0EE408A33
:105AF000B0EE480ADBF89836A7F170009847DBF85B
:105B0000083738469847B64B1B78032BB0EE408ACF
:105B100001F0AF80D5F85C06DBF8B830B0EE480A8B
:105B200098470136032E07F12407A8EC010A05F176
:105B30000405B7D1029CAA4B1D78072D01F02682DF
:105B400094F828310493002B40F0BD86A54B5B7977
:105B5000002B40F0C2850123A14A84F82831127835
:105B6000072A01F08786002306939F4B94ED4C9AF9
:105B700093ED007A9D4BDFF8D882D3F800A09C4BC0
:105B80000293F7EE007A37EEC9BA08F11C032BEE48
:105B900007BA0025B4EEE7BAF1EE10FA0593D4ED9A
:105BA0004BBA944BDFF8ACB2DFED938A9FED93AA2A
:105BB000DFED93AADFED939ADFF89C92924F019369
:105BC00088BFB0EE67BA2E46904B98ED008A2B4402
:105BD000D3ED007AF5EE407AF1EE10FA17D08C4B47
:105BE0002B44D3ED006A38EE667AB0EEC76AF4EE65
:105BF000C67AF1EE10FA08D5B5EEC07AF1EE10FAD9
:105C0000CCBF37EEA68A36EEE78A83ED008A814B59
:105C10001A8893073FD0022E3DD07F4B9AF82E1062
:105C200033F9163007EE103A059B07EE901A2B4415
:105C3000F8EEE76AB8EEC77AD3ED007A4B42A6EEEB
:105C4000A77A700007EE903AF8EEE77AB4EEE77ABA
:105C5000F1EE10FA0AD407EE901AF8EE677AF4EE35
:105C6000C77AF1EE10FA88BFF0EE477A6B4B6C49B9
:105C70000344085EB3F90C30C01A07EE100AB8EE00
:105C8000C77AD007E7EE687A40F12586654B93ED39
:105C9000008A27EE888A029B94F868212B44D3ED72
:105CA00001CA38EE6CCA002A3DD05F4BD4F86C2193
:105CB00003991B688A1A9A4235DD9AF84830022BFC
:105CC00001F0B086022E04F07E80584B1B689907C5
:105CD00040F1A987514B5249DFF848E131F916C02C
:105CE0009EED008ADFF874E1C7ED00AA03EB4600E1
:105CF00028EE288AB0F90C00A0EB0C0007EE900A01
:105D0000F8EEE77ADEF8000027EE888A904238EE57
:105D10006CCAC1F26C81F7EE007AB4EEE79AF1EE4C
:105D200010FA01F13B81424B2B4493ED000A019B99
:105D30002BEE800A022E20EE0C0AA3EC010A01933E
:105D400003F0FF873B4B9BED007AD3ED007A3A4B93
:105D5000D7ED006A93ED006A384B67EE277A2B4443
:105D600027EE8B7AD3ED007A67EE277AF0EE665A4B
:105D7000ECEE275AB1EE467AF4EEC75AF1EE10FA7D
:105D800008D4F4EEC65AF1EE10FA8CBFB0EE467AA3
:105D9000B0EE657A94ED4C6AF7EE007AB4EEE76AFD
:105DA000F1EE10FAACBF0123002343B1F0EEE66A36
:105DB000F0EEC77AF4EEE67AF1EE10FA01D587ED4F
:105DC000007A022E03F0B6871D4A1E4B52F82600B9
:105DD0001B68B0EE6C0A984742E000BF6CC400201C
:105DE000F83A0020F45B0020ECAC002038390020A9
:105DF000085C002098660020CDCCCC3DAE47813FAA
:105E0000000000000000C842A4660020E0AC0020B2
:105E1000A42B0020E8380020B02B0020D068002000
:105E2000F83D0020C8AC0020F4AC0020143E002057
:105E30009CAC0020A000002010AD0020A8AC0020E9
:105E400048A8002044A800200C5C0020FC3A002058
:105E5000982B002040A80020B0660020F0AC002065
:105E6000CC4ACD4B52F826001B6898479AF8373039
:105E700023B1CA4B1B88002B00F0B485B0EE6A8AB0
:105E8000C74B9BED007A38EE400A2B4493ED008A15
:105E900083ED000A9AF8483030EE480AC0EE077ADF
:105EA0002BB3C04B1B78DB0721D5B7EE007AB4EEDD
:105EB000C79AF1EE10FA04DB94F86831002B00F079
:105EC0005087D4F86C31039AD31AB74A12689A42B1
:105ED0000DDDB64B93ED007AB0EECCCAB4EEC7CA76
:105EE000F1EE10FA41F19F80002384F86831B04B45
:105EF00094F878212B4493ED007A2BEE877A67EEA5
:105F0000277AC9ED007A32B9019BC7ED00AA43EDAB
:105F100001AAC9ED00AA0136032E08F1040809F10F
:105F2000040907F1040705F104057FF44DAEA14B08
:105F30001B78072B01F02482012B01F0A0840023A1
:105F4000029394F88031002B40F098859A4B9B4A3D
:105F50001B68126813F4805C92F82C2040F08F8646
:105F60009749984891ED006A408B974984ED646A9F
:105F700091ED007A954984ED657A07EE900AF8EE86
:105F8000E76AD1ED037A924984ED626A37EE467A88
:105F900077EEE67AD1ED006A84ED617A012184F82A
:105FA0009811C7EEA65A8B488B4990ED005A8B4842
:105FB0009FED8B6A90ED004A8A48DFED8B6AD0ED49
:105FC000004A91ED007A35EE045AF7EE007AF4EECD
:105FD000E75A35EE245AF1EE10FA88BFF0EE675A10
:105FE00025EE065AF4EEE65AB1EE476AF1EE10FAE3
:105FF000B4EEC65AB8BFF0EE665AF1EE10FAC4ED30
:10600000675A01F11F80B4EEC75AF1EE10FA88BF4B
:10601000B0EE475A6F49DFED726AD1ED017A6F49F0
:1060200091ED014A6F4977EE847AD1ED014A77EE1E
:10603000A47A67EEA67AB4EEE76AF1EE10FA08DC0D
:10604000B4EEE77AF1EE10FA8CBFB0EE676AB0EE0C
:10605000476A6049DFED626AD1ED027A5F49D1EDAE
:10606000024A624977EEA47A91ED007A67EEA67A49
:10607000B1EE473AF4EEC37AF1EE10FA08D4F4EE3A
:10608000C77AF1EE10FA8CBFB0EE473AB0EE673A3D
:106090005749497809B9B1EE433A002A41F0928252
:1060A000F7EE003ADFF850B19BF80020002A02F02A
:1060B0000F825049DFED4C7AD1ED024AD1ED016AF1
:1060C00091ED037A66EE244AE5EE264AE3EE074AAE
:1060D00063EEA44AF4EEE74AF1EE10FAB4BFB0EE74
:1060E000674AB0EE644A98BFF0EE647A012ACDEDBB
:1060F0000A4A02F01D8291ED067AD1ED052AD1ED12
:10610000076A26EE077AA5EE227AA3EE267A23EE18
:10611000877AB4EEE77AF1EE10FAB4EEC47A8CBF67
:10612000F0EE676AF0EE476AF1EE10FA88BFF0EE23
:10613000676AB4BFF0EE447AF0EE477A022A8DED3A
:106140000B7A00F0138191ED0A7AD1ED092A91EDD5
:106150000B4A26EE077AA5EE227AA3EE047A23EE06
:10616000877AB4EEE67AF1EE10FAB4EEE77A8CBFF5
:10617000B0EE664AB0EE474AF1EE10FA98BFF0EE84
:10618000446AA8BFF0EE477A032A8DED0C7A00F03E
:10619000ED8033E09CA8002098A80020E83800207B
:1061A000D42B0020593A0020F4AC002000AD002090
:1061B000B4AC0020F83A0020185C002038390020E8
:1061C000506700207C5D0020B4680020D43B002094
:1061D000D0AD00209866002014AD0020A4660020F9
:1061E0006F12833AB06600200000000018AD002056
:1061F000F868002040AD0020D93A002091ED0E7AD9
:10620000D1ED0D2A91ED0F4A26EE077AA5EE227AFE
:10621000A3EE047A23EE877AB4EEE67AF1EE10FA72
:10622000B4EEE77A8CBFB0EE664AB0EE474AF1EEC4
:1062300010FA98BFF0EE446AA8BFF0EE477A042A3D
:106240008DED0D7A00F0928091ED124AD1ED112A78
:1062500091ED137A26EE044AA5EE224AA3EE074AF0
:1062600023EE844AB4EEE64AF1EE10FAB4EEE74AC1
:106270008CBFB0EE667AB0EE447AF1EE10FA98BFB9
:10628000F0EE476AA8BFF0EE447A052A8DED0E4A7B
:106290006CD091ED164AD1ED152A91ED177A26EEC4
:1062A000044AA5EE224AA3EE074A23EE844AB4EE3E
:1062B000E64AF1EE10FAB4EEE74A8CBFB0EE667A29
:1062C000B0EE447AF1EE10FA98BFF0EE476AA8BF3C
:1062D000F0EE447A062A8DED0F4A47D091ED1A4A26
:1062E000D1ED192A91ED1B7A26EE044AA5EE224A39
:1062F000A3EE074A23EE844AB4EEE64AF1EE10FA22
:10630000B4EEE74A8CBFB0EE667AB0EE447AF1EEB6
:1063100010FA98BFF0EE476AA8BFF0EE447A072A59
:106320008DED104A22D091ED1E7AD1ED1D2A91ED0E
:106330001F4A26EE077AA5EE227AA4EE037A27EE0C
:10634000237AB4EEE67AF1EE10FAB4EEE77A8CBF77
:10635000B0EE666AB0EE476AF1EE10FA8DED117A92
:1063600098BFF0EE466AA8BFF0EE477A77EEE67A7D
:10637000F7EE006AF4EEE67AF1EE10FAC4ED4C7A2C
:1063800043F3648386EEA77A022ADDED0B7A67EE8B
:10639000244A67EE877ACDED0A4ACDED0B7A2DD0EF
:1063A000DDED0C7A67EE877A032ACDED0C7A25D0E5
:1063B000DDED0D7A67EE877A042ACDED0D7A1DD0DA
:1063C000DDED0E7A67EE877A052ACDED0E7A15D0CF
:1063D000DDED0F7A67EE877A062ACDED0F7A0DD0C4
:1063E000DDED107A67EE877A072ACDED107A05D0B9
:1063F000DDED117A27EE877A8DED117ABA490968B9
:1064000011F0805800F09D87F6EE005AC4ED675AEF
:10641000002A02F0548094F99801D4ED654AB34DF6
:10642000B34994ED646AB34EB34FDFF8F8E2B5F8C0
:106430001AA0C978B6F9069097ED005A9EF800E0C8
:10644000D4ED616AD4ED627A07EE100AFDEEE44AFB
:10645000AA4814EE905A0078FDEEC64A03F01006E2
:1064600003F4800300F00107B8EEC77A14EE900A37
:106470000193002941F0E680A149002E40F09B875E
:1064800091ED006A9DED0A5A9E4B25EE866AA5EEB7
:10649000076AB0EE675AA6EE265ABDEEC56A16EE3A
:1064A00010EA16EE106AAE45A8BF2E467045C8BF6A
:1064B000064606EE106AB8EEC66A012A83ED006A47
:1064C00000F0DC8091ED046A9DED0B5A25EE866AA2
:1064D000A5EE076AB0EE675AA6EE265ABDEEC56A6B
:1064E00016EE10EA16EE106AAE45A8BF2E467045AD
:1064F000C8BF064606EE106AB8EEC66A022A83EDE9
:10650000016A00F0BB8091ED086A9DED0C5A25EE02
:10651000866AA5EE076AB0EE675AA6EE265ABDEE69
:10652000C56A16EE10EA16EE106AAE45A8BF2E46F2
:106530007045C8BF064606EE106AB8EEC66A032A62
:1065400083ED026A00F09A8091ED0C6A9DED0D5A80
:1065500025EE866AA5EE076AB0EE675AA6EE265AC1
:10656000BDEEC56A16EE10EA16EE106AAE45A8BF7B
:106570002E467045C8BF064606EE106AB8EEC66ADB
:10658000042A83ED036A79D091ED106A9DED0E5ACD
:1065900025EE866AA5EE076AB0EE675AA6EE265A81
:1065A000BDEEC56A16EE10EA16EE106AAE45A8BF3B
:1065B0002E467045C8BF064606EE106AB8EEC66A9B
:1065C000052A83ED046A59D091ED146A9DED0F5AA6
:1065D00025EE866AA5EE076AB0EE675AA6EE265A41
:1065E000BDEEC56A16EE10EA16EE106AAE45A8BFFB
:1065F0002E467045C8BF064606EE106AB8EEC66A5B
:10660000062A83ED056A39D091ED186A9DED105A7E
:1066100025EE866AA5EE076AB0EE675AA6EE265A00
:10662000BDEEC56A16EE10EA16EE106AAE45A8BFBA
:106630002E467045C8BF064606EE106AB8EEC66A1A
:10664000072A83ED066A19D091ED1C6A9DED115A57
:1066500065EE865AE7EE055AE6EEA57AFDEEE77A94
:1066600017EE901A8D42A8BF0D468842C8BF054656
:1066700007EE905AF8EEE77AC3ED077A2FB922B108
:10668000920021491F4829F029FC204B1B68002B50
:1066900040F0F0841E4B1B7893B19BF8000060B172
:1066A000184E1C4F0025E8B23B68B6EC010A98472B
:1066B0009BF8000001358542F5DB174B1B689847B6
:1066C000164B1B78072B00F06E86012384F80031EF
:1066D00013B0BDEC0A8BBDE8F08F114B1B78013B6A
:1066E000DBB2FFF739BA00BF98BF00207C5D002005
:1066F000F03800203CA400201CAD0020593A0020B6
:1067000040AD0020F866002020AD002038A8002011
:10671000F05B0020DC580020E4580020F83A00200C
:10672000C4680020E8580020BC4B1A78D4F81CE15B
:10673000BB4E9FEDBC7A4FEACE00331883ED007A52
:10674000002A7BD0B849B0EE476AF0EE476A0023D2
:10675000F1EC017A013367EEA77A05EE903AB4EED8
:10676000E77AF1EE10FAF8EEE55AB8BFB0EE677AC4
:106770009A4276EEA76AA7EEA56AE9D1F5EEC06A5D
:106780003318F1EE10FA83ED007A57DDC6EE265A83
:10679000A64BA74A1288B7EE000AD3ED007A75EE31
:1067A000C05A65EEA77AFDEEE77A17EE903A812B94
:1067B00041F3DB879342A8BF134607EE903AF8EE09
:1067C000E77A9C4B00EB0E0103EB810393ED057A16
:1067D000D3ED003A93ED066A93ED014AD3ED046AD6
:1067E000D3ED034A93ED025AA3EEA77AA4EE276AEB
:1067F00066EEC76AA7EE646ABDEEC77AE5EE276A61
:1068000017EE101A812983ED056AC3ED066A41F37C
:10681000A9878A42A8BF0A4607EE902AF8EEE77ACF
:10682000FCEEE77ACDED047ABDF810303218938093
:10683000BEF1000F02D1132F03F0FC80152F41F0A1
:106840006D8330447C4E838826F81E30D4F818516E
:106850007A4B013583FB05235A19EB17C3EBA203CF
:10686000C3EBC303ED1AC4F81851754B1B78002B0A
:106870007FF40EA9734EDFF8008206F24C7506F520
:10688000F767F6EC017A9BED080ADBF87837F8EE4B
:10689000E77A284627EE800A9847A5F1E000DBF862
:1068A00098369847A5F17000DBF808379847D6F876
:1068B0005806DBF8B83098472435AF42A8EC010AF7
:1068C000DFD1FFF738B9013B84F8283113B0BDECB4
:1068D0000A8BBDE8F08F94ED577AB1F90000D4ED42
:1068E000586AB1F902E0584AF4EEC76A80EAE073E8
:1068F0008EEAEE71A3EBE073F1EE10FAA1EBEE710C
:10690000B4BFB0EE476AB0EE666A8B42B8BF0B46C2
:1069100007EE103A1378B8EEC77A27EE287A002BE4
:1069200040F0F081494BD3ED005AF4EECA5AF1EE33
:1069300010FA40F19A87B7EE005A75EE654ADFED1E
:10694000446A9FED445A444B36EEC77A24EE855A8A
:10695000D3ED006AE7EE055A65EEA65AF5EEC05A89
:10696000F1EE10FA40F2E984C9EEA56AB7EE007ABA
:10697000F0EE475AE6EE665AF0EE656AF4EEC76A44
:10698000F1EE10FA88BFF0EE476AF5EEC06AF1EE5C
:1069900010FAB8BFF0EE6A6A304B93ED007A67EEFA
:1069A000877AA7EEA68AFFF776B92D4B1E4C196899
:1069B0002C4A214E94F80031C969128831807280C6
:1069C000002B3EF4D7AF03F0AFFA002384F8003178
:1069D000254B1B78072B7EF4CDAFF8F7A3F8824642
:1069E000FEF7CABF214B224A2B4493ED007AD2ED29
:1069F000007A204B67EE277AF7EE006AF4EEE67A2B
:106A0000F1EE10FA93ED007A88BFF0EE667A67EE49
:106A1000877A27EE888AFFF733BA00BFB2300020AA
:106A2000D032002000000000642A0020B430002092
:106A3000B0300020E8320020FC3A00209324499234
:106A4000A53000206CC40020D4AC0020DCAC0020B9
:106A500000003443610BB63BD0AC0020CCAC00202E
:106A600064C1002030350020F83A0020C02B0020FF
:106A7000C4AC0020C0AC00200C5C0020CE4BDFF882
:106A800088B31B789BF80020DD077FF5F8AD002A5E
:106A90003FF4FBADD4ED583A94ED574AC74BD4EDD3
:106AA000627A93ED005A94ED617AD4ED555A94EDE3
:106AB000546AC349C34BF4EEC43AF3EE046AF1EEF0
:106AC00010FA77EEA64A00F1E58791ED026A26EE0C
:106AD000656AB0EE674AA6EE074AB4EEE44A34EEC1
:106AE000666AF1EE10FA48BFB0EE456A012A83EDFE
:106AF000006A3FF4CAAD91ED066A26EE656AB0EE13
:106B0000674AA6EE074AB4EEE44A34EE666AF1EE4E
:106B100010FA48BFB0EE456A022A83ED016A3FF4DD
:106B2000B4AD91ED0A6A26EE656AB0EE674AA6EE4C
:106B3000074AB4EEE44A34EE666AF1EE10FA48BF52
:106B4000B0EE456A032A83ED026A3FF49EAD91EDF3
:106B50000E6A26EE656AB0EE674AA6EE074AB4EE04
:106B6000E44A34EE666AF1EE10FA48BFB0EE456AC8
:106B7000042A83ED036A3FF488AD91ED126A26EE94
:106B8000656AB0EE674AA6EE074AB4EEE44A34EE10
:106B9000666AF1EE10FA48BFB0EE456A052A83ED49
:106BA000046A3FF472AD91ED166A26EE656AB0EEA6
:106BB000674AA6EE074AB4EEE44A74EE666AF1EE5E
:106BC00010FA48BFF0EE456A062AC3ED056A3FF4A5
:106BD0005CADD1ED1A6A66EEE56AB0EE674AA6EEE4
:106BE000874AB3EE046AB4EEE44A74EE466AF1EE04
:106BF00010FA48BFF0EE456A072AC3ED066A3FF473
:106C000044ADD1ED1E6A66EEE55AE5EE877AF4EE04
:106C1000E74A77EEC67AF1EE10FAC8BFF0EE457A91
:106C2000C3ED077A31E5684BC7ED00AA1B689342B4
:106C3000BFF671A8654B1A88002384F86831002AD2
:106C400041F03384624A634B1178186881F0010186
:106C5000F3F754F8FFF767B895ED007A0BEB4602AF
:106C6000B8EEC78A928F29F8162028EE278AFEF7F9
:106C700030BF29F03DFB29F81600FEF74BBF4E4907
:106C80000978C80703D45449098BA4F88C115349D7
:106C90005348098890ED037A07EE901AF8EEE77AE8
:106CA000B4EEE77AF1EE10FA40F2CD864D48008856
:106CB00007EE900AF8EEE77AB4EEE77AF1EE10FA12
:106CC000C0F2798648484949D0ED006A91ED006AE2
:106CD0004748C4ED646ABCEEC75A76EE665A15EEB4
:106CE000101AC4ED626AC4ED615A84ED656AA4F8B5
:106CF0008C110121D0ED006A84F8981177EE677A43
:106D0000FFF74FB93B4B93ED005AB5EEC05AF1EE89
:106D100010FA40F31283384BD3ED006AF5EEC06AE7
:106D2000F1EE10FA40F3098336EEC77A66EE695A3F
:106D300087EE266AC5EE856AB7EE007AB4EEC76ABA
:106D4000F1EE10FA88BFB0EE476AB5EEC06AF1EE18
:106D500010FA76EE876AB8BFB0EE6A6A66EE266A07
:106D60000CE6264A92ED007AF0EEE76AF4EEC76A86
:106D7000F1EE10FA7FF7A5A8214A92ED007AF0EE25
:106D8000CC6AF4EEC76AF1EE10FA7FF79AA81D4AB2
:106D900098ED007AD2ED006AB0EEC77AB4EEE67AEA
:106DA000F1EE10FA7FF58DA801220399C4F86C1159
:106DB00084F86821FFF789B8593A00201CAD0020FB
:106DC00040AD0020F8660020F0AC0020BCCD0020D3
:106DD000BECD0020C0CD00207C5D0020D4AD0020C1
:106DE000D43B0020D6AD0020C0AD0020B468002008
:106DF000DCAD0020D0AC0020D8AC002004AD0020D9
:106E000000AD002008AD0020D93A00208F49904BFA
:106E100091F801908F4902930D781B688E4E4FF4C4
:106E20007A71B1FBF3F3C3EB431803EB88034FEA2A
:106E3000C3081FFA88F84745B6F9060001F0FE8539
:106E4000DBF88810BBF93CE0DBF86C304A1C07EE3D
:106E500090EA7344012ACBF88820CBF86C30F8EE26
:106E6000E77A01F0F885DBED1E5ADBED206A07EECC
:106E7000102A37EEE56AB8EEC75A012F86EE057A7A
:106E800037EE257A77EEC77A8BED1F7AE7EE866AC2
:106E90008BED1E7AF0EE667ACBED216ACBED206A9F
:106EA00002F01084DBF89C10BBF93EE0DBF8703098
:106EB0004A1C07EE90EA7344012ACBF89C20CBF8D9
:106EC0007030F8EEE77A01F0E185DBED235ADBED77
:106ED000256A07EE102A37EEE56AB8EEC75A012F89
:106EE00086EE057A37EE257A77EEC77A8BED247A2F
:106EF000E7EE866A8BED237AF0EE667ACBED266AB2
:106F0000CBED256A02F00884DBF8B010BBF940E055
